:020000040800F2
:1000000000500020C56C0108656D01087950010899
:10001000656D0108656D0108656D0108000000004F
:10002000000000000000000000000000656D0108F5
:10003000656D010800000000656D010823F30008EC
:10004000656D0108656D0108656D0108656D010844
:10005000656D0108656D0108C92A0108C72A0108F4
:10006000656D0108656D0108656D0108656D010824
:10007000B1F20008A1F2000891BB0008656D01080B
:1000800091F2000881F20008656D0108656D0108B4
:10009000656D0108656D0108656D0108C52A0108D7
:1000A000656D010869B90008656D010879B9000836
:1000B0005DB900086D8300085D830008757600084F
:1000C000797600086D76000871760008656D010884
:1000D000656D010889BB000881BB000879BB000879
:1000E00031F30008656D0108656D0108000000002E
:1000F0000000000000000000000000000000000000
:0C01000000000000000000005FF808F1A3
:100110002DE9F04FAE4B93B01F789946002F6BD06E
:10012000AC4B1868002801F0AC870FF09DF8AA4C82
:1001300020680FF039FA002801F0A38720680FF03B
:1001400030FA0928A54C01D03F2849D14FF00008CA
:1001500046462768A24D2FB1A24829683A4618F0B2
:10016000C1FE10B9A84606B92E469F4B10359D42D8
:10017000F1D3C6B1D6F800E0D8F800C023681EF865
:1001800003501CF80300A8420DD15A1C954938B9F8
:100190002D2B05D8914D2A602025CD54885402E09E
:1001A000CD542260EAE723680BB146450FD08F4853
:1001B00012F0F4F8464507D856F8100B12F0EEF896
:1001C000092008F035FDF5E70DF0E2FD0027236872
:1001D0009F42ACD2834BD85D08F02AFD0137F6E789
:1001E0002368002B41F0D286042841F023877D4804
:1001F00012F060FA01F045BF7D4E751E06F1010850
:1002000055F8093C002B01F0618655F8090C0FF0F8
:10021000CBF9002801F03D8655F8090C0FF0C1F923
:1002200015F8053C0446013B042B04D8DFE803F035
:10023000070C111B1F0024283BD1012336E04D2859
:1002400014BF0023022331E03C2814BF0023032302
:100250002CE040284FF000039EBF05F8043C05F851
:10026000030C042322E005F8020C05231EE015F818
:10027000042C15F8033C9A4209D2531C5D4905F839
:10028000043C482303FB07131A44107242E015F89C
:10029000022C691E5A4013F1FF3303D311F8010BEE
:1002A0004240F8E794420CBF0623002305F8053CC2
:1002B00030E0DFF870A19AF8003013F0040229D181
:1002C000232C55F8091C1AD1012389F80030424B20
:1002D00049481960494B5A7310221A733D4A5860B5
:1002E0001960996046480433136012F057F80DF016
:1002F0004FFD9AF8003043F002038AF80030414B7A
:100300001B78A34201BF404A404B1A60404A04BFD9
:10031000404BDA6015F8053C062B7FF476AF15F8F4
:1003200003EC482303FB07E33B4A05F1FF3A03EBE9
:10033000020E15F8023C394A1FFA83FB4FF0000CFD
:1003400006AC572BCDF80CA007CACDF810E084E816
:100350000700ADF814B0ADF816C0ADF820B0CAEB88
:100360000E0A00F06A8500F29980372B00F0BD84F8
:100370005CD82D2B00F0198414D8252B00F0F683BF
:1003800004D8232B00F0688100F06BBD292B00F00E
:10039000F8832B2B40F06585039515F8012C204B35
:1003A00001F0B2BC312B00F0008508D82F2B40F0B3
:1003B0005885DFF874A00024D34600F0D7BC332B57
:1003C00000F04984352B00F07D8100F04ABD00BF6C
:1003D000DC3A0020F4150020343100209431002054
:1003E00054BE01086431002044C001085CC4010807
:1003F0006A1500206015002075F60008B003002083
:100400008CC401089A360020EFBEADDEF04F00200C
:100410000400FA0500ED00E06815002074A0010852
:1004200050310020DB3A0020381F0020432B00F021
:1004300024841DD83C2B00F0EC8011D8392B40F0DF
:100440001085B64B15F8012C1A7016F8012C1A718C
:100450006A78DA70EA1C0392AA785A7101F0C9BC72
:100460003E2B00F0C580412B40F0FB840023F9E3D4
:100470004A2B00F0C78009D8442B00F0ED84482BAC
:1004800040F0EF8407F042FF01F0B3BC4E2B00F0C8
:10049000BB83512B00F0AD8200F0E3BCD22B5CD0CB
:1004A00020D8CD2B00F084820FD8C92B00F0B68263
:1004B00003D8C82B64D000F0D4BCCA2B00F0B380A2
:1004C000CC2B00F0498100F0CCBCCF2B00F08D810B
:1004D000C0F07982D02B00F06382D12B00F0D08263
:1004E00000F0BFBCDA2B00F03F8218D8D42B00F00C
:1004F000DB813ED3D62B00F0CB81D92B40F0B184E9
:1005000003A80CF0D1FC864C208003A80CF0CCFC96
:10051000608003A80CF0C8FCA08001F06ABCEF2B3F
:1005200057D012D8DB2B00F03682DC2B40F09984B8
:100530007C4B15F8012CCDF80C801A7016F8012CA4
:100540005A706A789A7001F054BCF22B00F0ED8179
:10055000FA2B00F0438200F084BC734B1B785907E0
:1005600001F1478415F8010C03950AF0BBFB01F07B
:1005700040BC03A80CF098FC6C4B188001F039BC0F
:10058000CAF3470ABAF1120F01F235840024544528
:1005900007D203A80CF088FC09AB23F8140001343F
:1005A000F5E752460023534507DA09A931F813004D
:1005B0005F4921F813000133F5E7122A05D05C4B9F
:1005C000002123F812100132F7E70124594B00F003
:1005D00045BC594C03A8D4F800A00CF065FCAAF85F
:1005E000020003A824680CF05FFC208001F001BC2D
:1005F000524B15F8012C03969A7016F8012C5A707C
:1006000001F0F7BB03A80CF04FFC4D4B188401F030
:10061000F0BB4C4B15F8010C1B680395987711F053
:1006200059FD01F0E6BB474B1A68531E02F1090160
:10063000039A501C0390104610F8024B03F8014F28
:10064000039050788B42987202F1030003909278E5
:100650001A75EDD101F0CDBB15F8011C03951329D6
:1006600001F3C983384C16F801EC20680396002387
:10067000364A02EBC30292F805C0F4451DD1127947
:1006800000EB810300F82120039A511C039112789A
:100690005A70039A511C039112789A70039A511C54
:1006A000039112780021DA7020680EF0B7FD284B14
:1006B00080F00100187001F09CBB01331C2BD7D1D6
:1006C00001F099BB15F8012C03950B2A01F39383D4
:1006D00016F8010C1F4B04281968039601F38B834D
:1006E00006235A438B1858716878CDF80C808854CB
:1006F000039A511C039112785A70039A511C03916A
:1007000012789A70039A511C03911278DA70039A46
:10071000511C039112781A7101F06BBB98140020E0
:1007200010260020A4170020DB3A0020FE0E002037
:100730009C130020B533002010160020B10E0020BD
:10074000B003002080270020F422002054A40108D8
:1007500006000020F81F0020BAF1090F41F34B8377
:10076000DFF8F8B315F8013CDBF80040039523707F
:10077000039B04F1030E5A1C03921B780022637042
:10078000039B022A03F10101039118780CBF4FF07B
:10079000FF0C4FF0640C604528BF60460132032A0D
:1007A0000EF8010FECD19A1C03925A780333642A95
:1007B00028BF64220393E2714B7812A8A370039BB5
:1007C0005A1C40F83C2D1B78E3700CF06DFBBAF11D
:1007D0000A0F608101F00D83039BDBF80020591C98
:1007E00003911B78137201F004BB03A80CF05CFBAF
:1007F0006FF4AF628318DFF868A3C62B98BFAAF81E
:10080000100003A80CF050FBC14C208003A80CF092
:100810004BFB608003A80CF047FBA08003A80CF002
:1008200043FBBC4BBC495880039BBC4C5A1C0392F5
:100830001A4612F8030B03929A7808704A701A1D30
:100840000392DA780633E27213F8022C0393B44B66
:1008500003A88AF80B20D3F82CA00CF025FB039BEF
:1008600000EB80005A1C4000AAF8000003921A46D0
:1008700012F8021B03925A7821702271DA1C03923B
:100880009A78E2701A1D0392DB78637101F0B1BAB5
:10089000002403A80CF008FBA24B23F81400013439
:1008A000082CF6D101F0A5BABAF10F0F41F0A382DE
:1008B00015F8014C0395072C01F29D82DFF8A4A2E4
:1008C00003A8DAF800B00CF0EFFA0E235C432BF823
:1008D000040003A8DAF800B00CF0E6FAA344ABF881
:1008E000020003A8DAF800B00CF0DEFA039BDAF895
:1008F0000020A34414441A46591CABF80400039189
:1009000012F8021B03A80392A1715A78E271DA1C53
:1009100003929A7822721A1D0392DB7863720CF0AC
:10092000ADFAC4F80A0001F064BA15F8013C039569
:100930000F2B01F360827C4916F8010CC3EBC30254
:100940008B1888546A785A70AA789A70EA78DA70A4
:100950002A791A716A795A71EA1D0392AA799A71F1
:100960000EF089FE01F045BA704B03951C6815F82E
:10097000013C12A82370039B5A1C03921B786370DE
:10098000039B5A1C40F83C2D1B78A3700CF08CFA8A
:10099000E08001F02EBA66480CF019FF01F029BA88
:1009A000644B1B785B0701F124820AF0B3F91AE06B
:1009B000604B1B785C0701F11C825F4B4FF4C872DF
:1009C0001A8001F016BA5B4B1B78580701F11182AF
:1009D0005A4A137843F0040300F015BF554B1B78B7
:1009E000590701F1088209F003FF09F0F7FF01F050
:1009F00000BA4B4B93F83020012A01F2FC8115F824
:100A0000012CCDF80C8083F8332016F8012C83F8E4
:100A100031206A7883F8322001F0EBB915F8012C07
:100A2000464B1AB11A7842F0020202E01A7822F01C
:100A3000020212AC44F83C6D1A7016F8012C404BBF
:100A400020461A700CF01AFADFF81CA1CAF8000050
:100A500020460CF013FACAF8040020460CF024FAE1
:100A6000384B188020460CF01FFA374B2C4A188060
:100A700092F8343043F0020382F8343001F0B9B90F
:100A800012AC15F8011C44F83C5D204601910CF0B5
:100A9000F5F9009020460CF0F1F9834620460CF061
:100AA000EDF9824620460CF0FFF920460CF0FCF9E7
:100AB000039B019901330393009A99B9234B1020AA
:100AC00083E8040809F04AFE1C4A137843F0010346
:100AD0001370BAF1000F01F08C811D4BC3F800A018
:100AE00001F087B9102941F084811A4B83E804088A
:100AF000BAF1000F02D0164BC3F800A01548164BF0
:100B00000222011D1A7007F021F901F072B900BF2D
:100B100046240020A9390020EC270020981400204A
:100B2000B00300201A31002058320020C00F0020EE
:100B3000B8E60108DB3A0020C60E0020882F00200E
:100B4000F80F0020F60F0020F40F0020B010002056
:100B50007C270020080F0020020F0020F03000202A
:100B600074360020081F0020FC0F0020CA4C03A888
:100B7000C4F800C00CF082F923681843206001F02B
:100B800038B903A80CF090F9C44CE08003A80CF02D
:100B90008BF9039B20815A1C03921B7803A8A37234
:100BA0000CF082F9A08101F024B912ACDFF8F4A2B4
:100BB00015F8013C44F83C5D20468AF808300CF0FA
:100BC00073F9AAF8140020460CF06EF9AAF8100088
:100BD00020460CF069F9039BAAF812005A1C0392F4
:100BE0001B788AF80A30049B9B1A012B41F3018180
:100BF00020460CF059F9AAF8160020460CF054F9DA
:100C0000AAF8180001F0F5B815F801AC0395BAF18F
:100C1000110F01F3F08016F8013CA14C12A804F862
:100C20001A3040F83C6D0CF03FF940F2ED23984249
:100C300005DD40F6CA039842A8BF184601E040F21D
:100C4000EE20A0F2EE20192390FBF3F004EB4A040F
:100C5000607001F0CEB815F8012C924B0395DA7252
:100C600001F0C7B8039A511C039111788D4A995429
:100C70000133082BF6D101F0BCB812AC44F83C5D4E
:100C8000DFF814A215F8012C874B2046CAF800C0E3
:100C90001A700CF0F3F8DAF800301843039BCAF826
:100CA00000005A1C03921A787E4B20461A720CF0F0
:100CB000FBF8DFF80CA2AAF8350020460CF0F4F897
:100CC000AAF8370020460CF0EFF8AAF839002046C1
:100CD0000CF0EAF8DFF8C4A1AAF8060020460CF0F0
:100CE000E3F8AAF8080001F084B807239AFBF3F3AD
:100CF000C3EBC3039A4541F07E80039A049B9B1A81
:100D0000062B41F37680531C039312780023674C23
:100D100004EBC304A1788A4217D1A27003A80CF097
:100D2000C3F8039BA0805A1C03921A4612F8021BB8
:100D30000392A1715A78E271DA1C03929A78627276
:100D40001A1D0392DB782372D7E70133052BDED11E
:100D500001F051B82BF824000134102C8AF802104D
:100D60008AF803300AF1040A01F04380039A049BD5
:100D70009B1A032B41F33D8003A80CF095F8039BCD
:100D8000B0F5B47F03F1010203921A4612F8021B78
:100D900003925B784FEA8402DCDB00230BEB020159
:100DA0002BF802304B8001F026B8BAF1080F0395FA
:100DB00015F801BC41F01F80BBF11F0F01F31B8030
:100DC00003A80CF071F8044603A80CF06DF8039B1F
:100DD000DFF8F0E0194604F03F0444EA80145A1C9E
:100DE0000EEB8B000392448011F8024B03915A786A
:100DF00002F00F0242EA04120EF82B20DA1C0392D2
:100E00009B7843700FF01AFC00F0F3BF19465A1C90
:100E1000039211F8022BD81C0391597803909B7808
:100E20000F2B00F2E887052A0ED8052900F2E38788
:100E3000062000FB02121E495354039BC3EB0E0213
:100E4000022AE3DC00F0D5BF062A40F0D487072948
:100E500000F2D187174AEFE7174B01241C7000F00E
:100E6000CCBF562B00F0618600F2C280362B00F01A
:100E7000078666D8242B00F06B852FD8032B00F053
:100E8000B68121D8012B00F0A381022B40F090877E
:100E900020460A490422E9E360310020981400202A
:100EA000EC14002074360020503100209A360020C7
:100EB0000C1F0020301F0020D8390020C4C40108B6
:100EC000B0030020781F0020052B00F0A681C0F0A1
:100ED0009A81222B40F06C870024CEE32E2B00F069
:100EE000E3851FD82A2B00F049852C2B00F049857B
:100EF000282B40F05D87DFF8B4A32046BAF806102F
:100F00000BF0FBFF2046BAF808100BF0F6FF069B2B
:100F10009AF80A20591C06911A702046BAF80C104B
:100F200000F0E0BE322B00F07085342B00F0C88357
:100F3000302B40F03D87DFF878A30AF1800B00F0FA
:100F4000CFBD452B00F09A861FD83B2B00F0918334
:100F500009D8382B00F000853A2B40F0298720462D
:100F6000BF4B00F0F7BC402B00F05285422B00F045
:100F70005A853D2B40F01C87BA4B069A9978501C35
:100F8000069011705A7800F0BCBE4D2B00F01F8502
:100F90000CD8472B00F03586C0F01A86492B40F05C
:100FA0000787B14B2046198C00F09CBE502B00F0F7
:100FB0004B86522B00F05D864F2B40F0F986069B46
:100FC0004FF0000A5A1C069283F800A0069B2046A8
:100FD0005A1C069283F800A0069B51465A1C0692A2
:100FE00083F800A00BF075FF2046514600F051BE7B
:100FF000732B00F0C68300F290806A2B00F0CA8346
:1010000011D8662B00F0AA8104D8642B00F013815C
:10101000652BA7E0682B00F0488200F2558220463D
:101020009249102222E36E2B00F070820DD86C2BB7
:1010300000F05A8240F2D5838D4B204619680BF0A0
:1010400048FF20468B4B00F074BC702B00F0F182FF
:10105000C0F0B482722B40F0AB86DFF858B2DFF8F4
:1010600058A22046BBF810100BF047FFBAF800104A
:1010700020460BF042FFBAF8021020460BF03DFF6D
:10108000BAF8041020460BF038FF7B4B20465988F5
:101090000BF033FF794B069A1978501C06901170AB
:1010A0000699DFF808A24A1C069200220A705978B5
:1010B000069B581C06901970069B9AF80B10581C3A
:1010C00006901970069B9BF80B10581C069019701F
:1010D000069B2046591C06911A70634B0A21DB6A55
:1010E000B3F9003093FBF1F189B20BF006FF069BD8
:1010F0009AF80020591C06911A70069B9AF8042051
:10110000591C06911A70069B9AF80320591C0691E7
:101110001A709AF8052000F0F4BD7E2B00F0E585EA
:1011200015D8772B00F01A8307D8752B00F09B8217
:1011300000F26B834FF0000AF5E27C2B00F0AC85E7
:1011400000F2BA85782B40F0338600223BE1F02B89
:1011500000F0E4832FD8A02B00F0ED83A42B00F047
:101160009F83962B40F02486454B204619880BF030
:10117000C4FE444B2046198889B20BF0BEFE424B98
:1011800020461B68C3F3C001C3F38002890041EA13
:101190004201C3F340021143C3F3401241EAC201CA
:1011A00003F0100319430BF0A8FE384B0021B3F8ED
:1011B00000E00B4682E0F52B00F0A885FE2B00F046
:1011C0009F83F12B40F0F485314B03F1700143E133
:1011D000069A511C069100211170069A511C069125
:1011E0001370069B5A1C0692132200F08DBD069BBD
:1011F0005A1C069201221A70069B9A1806920D221A
:101200001A7000F036BD2046224904220BF057FE2A
:10121000214B2046197800F065BD20461F490B225E
:101220000BF04DFE20461E4908220BF048FE2046DA
:101230001C4907221AE2069B20465A1C0692E72206
:101240001A70194B1A78069B591C06911A70069B46
:1012500004215A1C069200221A7000F01ABD00BF29
:1012600050270020B10E0020B0030020F003002022
:10127000A8100020D40F0020A9390020EC2700205E
:10128000D0390020FC1500208C170020622F002090
:1012900059320020C9C40108D93A0020CEC401083F
:1012A000DAC40108E3C4010850310020981400207A
:1012B000791F00207436002046240020AA4AD05608
:1012C000421C0BD04FF2FF721A41D20706D54EFADC
:1012D00003F2D20742BF01228240114301330C2B9B
:1012E000ECD1A24B0022D3F800E00123A0489340A8
:1012F000184018B113EA0E0F18BF19430132202A03
:10130000F3D19C4B8E461B7858079B4B48BF41F04E
:10131000010ED3F83CA0002319461846012202FA18
:1013200003FC1CEA0A0F05D01CEA0E0F1CBF82400A
:101330001143013001331C2BF0D120460BF0C9FDC5
:101340008E4B1A78069B591C06911A70BDF9143001
:10135000962B40F04E852046894BEAE2894B4FF0B0
:10136000000A1B89B3F5806F8CBF4FF0030B4FF061
:10137000000B854B204633F91A100AF1010A41FA95
:101380000BF189B20BF0B9FDBAF1030FF1D14FF0B7
:10139000000A7E4B204633F82A100AF1010A0BF0AE
:1013A000ACFDBAF1030FF4D14FF0000A784B2046A0
:1013B00033F82A100AF1010A0BF09FFDBAF1030F6E
:1013C000F4D100F016BD0E2303FB02FADFF8E4B1FE
:1013D0000092DBF80010204631F80A100BF08DFD6A
:1013E000DBF800302046534459880BF086FDDBF8CB
:1013F00000302046534499880BF07FFDDBF8003025
:1014000053449979069B581C06901970DBF80030FC
:101410005344D979069B581C06901970DBF80030AC
:101420005344197A069B581C06901970DBF800305B
:101430005344597A069B581C06901970DBF800300B
:1014400020465344D3F80A100BF043FD009A0132B2
:10145000082AB8D100F0CDBC069A13F8010C541C30
:1014600006941070069A1878541C06941070069A08
:101470005878541C06941070069A9878541C069458
:101480001070069AD878541C06941070069A187931
:10149000541C06941070069A58790733541C8B42DA
:1014A00006941070D8D100F0A4BC4FF0000A394B5C
:1014B000204633F81A100AF1010A0BF01EFDBAF1AA
:1014C000080FF4D100F095BC4FF0000A324B1B78A6
:1014D0009A4580F28E84314B204633F81A100BF077
:1014E0000CFD0AF1010AF1E7DFF8CCA02046BAF8BA
:1014F00000100BF002FDBAF8021020460BF0FDFCC4
:10150000BAF904300A2193FBF1F129E04FF6FF7A92
:10151000234B069A1B88511CFF2BA8BFFF23069163
:101520001370204B204619685145A8BF514621EA47
:10153000E17189B20BF0E1FC1B4B204619880BF0DE
:10154000DCFC1A4BDA7A1A4B19683AB10A23594370
:101550005145A8BF514621EAE17101E001F30F01B5
:10156000204689B2BEE300BF80A00108842F00207E
:10157000C0F11F0ADB3A0020B00300201831002020
:10158000F8150020C8160020CE0F0020782F00206C
:10159000A0270020242500209436002000340020BD
:1015A000AC140020A8140020AC10002098140020D7
:1015B000F00F0020081F00205C2F0020A74B1A68A6
:1015C0001178069A501C069011701A685178069A84
:1015D000501C0690117000221968DFF880A2114497
:1015E00008790699013201F1010E032ACDF818E0BD
:1015F0000870F1D1DAF800302046DA79069B591CE0
:1016000006911A70DAF800309A78069B591C0691F8
:101610001A70DAF80030DA78069B591C06911A70B5
:10162000DAF8003059890BF068FCDAF800301A7AE1
:1016300067E300238A4A1168C85C06994C1C06942B
:10164000087011681944887A06994C1C0694087031
:1016500012681A44117D069A0133501C0A2B069019
:101660001170E7D1C5E320467E492F220BF027FCFD
:10167000BFE37B4B1B689A7F43E37B4B1B6813F8EC
:10168000240003EB840A07F01BFA069B4279591CDD
:1016900006911A70069B9AF80120591C06911A703F
:1016A000069B9AF80220591C06911A70069B9AF81C
:1016B00003200134591C142C06911A70DDD198E3D3
:1016C000002106224A43694B069C186804F1010C6C
:1016D000831893F805E0CDF818C084F800E0805C2A
:1016E000069A0131541C06941070069A5878541CBE
:1016F00006941070069A9878541C06941070069AF6
:10170000D878541C069410701A79069B0C2903F1A2
:10171000010006901A70D4D16BE30AF1010ABAF104
:101720001C0F00F06683524A0123D26B03FA0AF3BE
:101730001342F2D05FFA8AF007F0C2F9D0F800B095
:10174000584617F0C6FB5946024620460BF0B7FB39
:10175000069B5A1C06923B221A70DEE70024444A7C
:101760000123D26BA340134207D0E0B207F0A8F9DF
:10177000069B4279591C06911A7001341C2CEED13B
:1017800037E30123069A511C069113700133092B8C
:10179000F8D12EE3374B069A1B78511C03F0020355
:1017A00006911370344BDFF8F4A01A78069B20469C
:1017B000591C06911A70DAF800100BF08AFB2046CB
:1017C000DAF804100BF085FB2C4B204619880BF03F
:1017D00094FB2B4B204619880BF08FFB2046294B9E
:1017E000A7E0294B204619880BF087FB274B2046A2
:1017F00019880BF082FB1E4B069A93F83430511C6B
:1018000003F0010306911370F3E215F8013C039510
:101810000BB91F4A02E0102B03D11E4A92E80204C2
:1018200002E04FF0000A5146069A501C06901370D1
:1018300020460BF04EFB204651460BF04AFB164B60
:10184000204619680BF045FB204600210BF055FBA4
:10185000204600210BF051FB0BE200BFF0300020CE
:10186000802700208CA00108F4220020F81F00200F
:10187000B0030020882F0020F80F0020F60F002072
:10188000F40F0020C01000206A1000206C1000200F
:10189000B0100020080F00207C270020FC0F002043
:1018A000069BB94A581C0690104692F850101970C1
:1018B000002390F85020934280F29B82B34A06990D
:1018C0009C5C01F1010ECDF818E00C7002F11001E2
:1018D0005C5C069901F1010ECDF818E00C7002F184
:1018E00020015C5C0699303201F1010ECDF818E060
:1018F0000C70995C069A0133541C06941170D8E759
:101900004FF0000AA24B204633F81A100AF1010AE0
:101910000BF0F3FABAF1040FF4D16AE2DFF8A8A2EF
:101920002046DAF8003059880BF0E7FA2046DAF85A
:1019300000301988D6E1974B204619680BF0C9FA98
:10194000954B204619680BF0C4FA2046934B01E0F2
:101950002046934B19689CE1924B069A1978501CCB
:1019600006901170069A1979501C06901170069A0B
:10197000D978501C069011705A79C2E18A4B1A78B6
:10198000BFE1DFF830A2069B9AF80820591C0691A7
:101990001A702046BAF814100BF0AFFA2046BAF8C5
:1019A00010100BF0AAFA2046BAF812100BF0A5FAA4
:1019B000069B9AF80A20591C06911A702046BAF81C
:1019C00016100BF09AFA2046BAF818108AE14FF078
:1019D000000A764B1B789A4580F20B82744B13F801
:1019E0001A1003EB4A02069B0AF1010A581C0690E2
:1019F00019705178204601EB810101EB810101F260
:101A0000EE2189B20BF079FAE3E76A4BDA7A78E1F2
:101A10000023684A995C069A0133501C082B0690F3
:101A20001170F6D1E5E1604B20461A78069BDFF88D
:101A300058A1591C06911A70594B19680BF049FAB4
:101A40005C4B20461A7A069B591C06911A70BAF80C
:101A500035100BF052FABAF8371020460BF04DFA59
:101A6000BAF83910DFF83CA120460BF046FA2046C0
:101A7000BAF806100BF041FA2046BAF8081031E126
:101A8000DFF848A10AF1280B9AF8022000234A49FE
:101A9000C95C8A4200F046820C333C2BF7D10AF134
:101AA000080ADA45F0D1A4E14FF0000A434B204682
:101AB00033F80A100AEB030B0BF01FFA069B9BF896
:101AC0000220591C06911A70069B9BF803200AF10C
:101AD000040A591CBAF1400F06911A70E6D188E148
:101AE000BAF80110204601F03F010BF006FABAF8EF
:101AF0000110204689090BF000FA069A1AF8013CF9
:101B0000511C1B0906911370069A1AF8013C511CCE
:101B100003F00F0306911370069B1AF8042B591C4F
:101B2000DA4506911A70DBD163E10022244B0620CE
:101B300000FB0230002306994C1C06940A7006999B
:101B40004C1C06940B700699C45C013301F1010E24
:101B5000062BCDF818E00C70EDD10132062AE5D144
:101B60000023069A511C069106211170069A511CF9
:101B700006911370134A995C069A0133501C082B86
:101B800006901170EDD134E1B00300200104002073
:101B900042040020E8F7FF1FECF7FF1FF0F7FF1FDC
:101BA000603100209814002050310020943600202D
:101BB000EC14002074360020C4360020381F0020AA
:101BC0000C1F0020301F0020101600209A36002025
:101BD00011F08EF9069B40F002005A1CDFF804A3B6
:101BE00006921870BAF8001020460BF072F9DAF875
:101BF0000C1020460BF06DF906F080FA01462046E5
:101C000047E003A80BF03AF98246204651460BF014
:101C100060F9DDF818B0079CB24BCBEB0404802CC4
:101C2000DB68A8BF80240AEB04029A4288BFCAEB93
:101C3000030406F01DFB50465946224611F08CF96C
:101C4000069B18440690D4E0069B5A1C069201227B
:101C50001A70A54B069A93F83310501C0690117019
:101C6000069A93F83110501C0690117093F83220A8
:101C700047E0069B5A1C0692002245E020469B49FD
:101C80000B220BF01CF9204600210BF022F9204614
:101C900000210BF01EF9ACE0DFF884A22046BAF870
:101CA00000100BF02AF92046BAF802100BF025F9C3
:101CB0002046BAF8041015E08D4B1A681178069A80
:101CC000501C069011701A685178069A501C0690A4
:101CD00011701A689178069A501C0690204611706F
:101CE0001B68D9880BF009F983E0824B069A1978B2
:101CF000501C06901170069A5978501C069011706D
:101D00009A78069B591C06911A7072E07A48002155
:101D1000C02217F09AF84FF0000EF346774C724A43
:101D200092F89E309E4537DA637AD90730D5227A09
:101D3000734B33F91230002B2ADDE0686E4B4FEA0B
:101D40000B124168B0F808C003EB020AAAF806C0FB
:101D500099504FF0000A012000FA0AF010EA0C0036
:101D600001D0504604E00AF1010ABAF1100FF2D195
:101D7000134498800220D8724820A3F808C09872B3
:101D800003F108029B680BF1010B53601023937160
:101D90000EF1010E0834C2E75A4B5FFA8BF119704D
:101DA000069B581C06901970012382F8143120E01C
:101DB000194655480BF014FD0146002800F0D48068
:101DC0004A880698514B079C93F800E0241AC2F306
:101DD0000B039C42A8BF1C464968120448BF0EFB77
:101DE0000311224617F0CEF8002C06DB069B1C449C
:101DF0000694012401E04FF0FF34ADF82240002C9E
:101E000044D0069B55F8090C0793414B06930DF0FF
:101E100060FB069B079C55F8090CE41A24238DF8F7
:101E200024304D238DF82530BDF9223009A9002B2F
:101E3000B4BF21233E238DF82630BDF82030052283
:101E40008DF828308DF827400DF0F6FB9DF828A07E
:101E50009DF82730002C8AEA030A0EDD224655F849
:101E6000090C06990DF0E8FB069B1C44A34204D024
:101E700013F8012B8AEA020AF8E755F8090C5146D3
:101E80000DF0B8FB55F8090C0DF01EFB002305F80A
:101E9000053C154B93F8142152B1002255F8090C5A
:101EA00083F814210DF06FFB55F8090C11F0FAFCC2
:101EB000184B1B7853B155F8090C0DF064FB0DF06D
:101EC00075FC08F06BFC144A144BDA60012F06F124
:101ED000480605F1480508F1480800F0D2800127BE
:101EE000FEF78EB91C000020B0030020CEC401080C
:101EF000C00F0020A4170020282200204C0400203E
:101F000024250020DC330020B5850008183100208E
:101F1000D9390020D83900200400FA0500ED00E08E
:101F200010260020069B2046591C06911A70BAF80C
:101F300004100AF0E2FF069B9AF80620591C06914D
:101F40001A70069B9AF80720591C06911A70069B76
:101F50009AF80920591C06911A70069B9AF80820D5
:101F6000591C06911A709AE54748BDF914100BF0F8
:101F700037FC00283FF43FAF444B03991B7852468F
:101F80000BF004FC039B5344039332E70C2803D16A
:101F90003F4810F003FA49E00A2801D00D2864D127
:101FA0003C4D3D4810F0FAF92846232116F083FFF6
:101FB00008B1401B206023687BB35A1EA95C20290E
:101FC00001D11346F8E7334A00212360D154334B43
:101FD000334DD3F80080D5F800A02E4F504616F0B0
:101FE00078FF064651463246384616F07BFF2D4AAA
:101FF00020B9BB5D43445B78580703D01035954248
:10200000E9D306E0954204D2701CEB683844984747
:1020100002E0254810F0C2F900231E4800213022BA
:10202000236016F012FF99F8003053B30BF0B0FEA6
:10203000FEF77DB80C28ABD07F2804D1FEF777B827
:102040002F2B3EF674A8A0F12002D2B25E2A3EF6F3
:102050006EA813B920283EF46AA85A1C22600D4AC3
:10206000D05406F0E5FDFEF762B87F28E8D1094AB2
:10207000013B00210D482360D15410F08FF9FEF789
:1020800056B813B0BDE8F08FD9850008183100208C
:1020900061C401086431002062C9010840030020C6
:1020A00054BE010844C001086CC4010888C401087A
:1020B0002DE9F04FA24C97B02368A24F5D6AA24B66
:1020C0009B783BBB2368A14ED3F82490A04B1FFA0A
:1020D00089F51D80284614F02DF89E49834614F09A
:1020E00081F89D4B804618600021706814F00EFA4C
:1020F000A0B19A4B736011E098470028E2D10DF02F
:10210000DFF8974B1B68EB1A1844964B1B68643337
:102110009842D7D2FB68002BEED1F0E740467168B9
:1021200013F058FF0146404614F010F9D6F800A00D
:1021300080465146584613F04BFF0146404614F086
:1021400051F80146504613F045FF306014F036FA5E
:102150007E4C80B2844B2D1AB081A3F800905D8034
:1021600004F10E007B68984748B9804B804D1A688F
:10217000049312F0020F40F0098100F001BE7D4D82
:10218000B4F90E3028462B60B4F9103029466B6044
:10219000B4F91230AB60784B1A7808F0B9F9774B84
:1021A0005A88984672B9764F3B88002B00F0A7807A
:1021B00098F80030DFF8D081049308F10C044FF058
:1021C000000961E0277D183477B9B8F8020013F0F0
:1021D000B1FF644BE1191A6824370AF0CBFE6C2F6B
:1021E000F3D15A4B01221A75002755F8270013F036
:1021F000A5FF242101FB07410AF089FE17F03EF8F4
:1022000045F827000137032FEFD1CCE7D4F800C001
:1022100008936146CDF818C0079013F0D9FE089BCB
:102220008346184613F08AFF0146584614F08EF88C
:10223000DDF818C00146604613F0CCFE0346079A4D
:10224000194660601046069313F0C2FE01465846D8
:1022500013F0C8FFA16813F0BDFE069BE060236089
:10226000A060DFF820B1002345F80A304AF80B30AF
:10227000059B012B26D009F10109B9F1030F08F1E3
:10228000040804F1140447D03B8855F82900B3F53D
:102290007A7F059302BF0023C8F800302361D8F885
:1022A00000304FEA890A0344C8F8003013F046FFB3
:1022B00023690133012B2361A8D1002360602060D2
:1022C000A360CEE72069012807DD013813F036FF4F
:1022D0000146E06814F03AF800E0002017F094F9A5
:1022E000049A72B10590104613F028FF059B014631
:1022F000184614F033F920B14FF47A733B80002371
:1023000012E0D8F800304FF47A7203F5FA7393FBB9
:10231000F2F34BF80A30AEE73888012801D10DF00E
:1023200033F83B88013BE9E7164955F8232051F87B
:102330002310521A45F823200133032BF4D114E75C
:1023400034270020D4160020D0030020040A0020E7
:10235000D0390020BD378635D430002083F9223EA5
:10236000B839002088300020420400208C1700205B
:10237000D8380020782F0020DA3A0020901700206B
:10238000C00E0020D00A0020880A0020904B1B7845
:10239000002B00F0F5840CF093FFD6F8D8308D4C6C
:1023A000C31A0693D6F8DC30C6F8D8001F78059318
:1023B0004FF0000A4FEA4A030793002F3AD055F82E
:1023C0002A0013F0BBFE8346069813F0B3FE824941
:1023D00013F008FF00218146606814F097F858B1A7
:1023E000384613F0ABFE7D4913F0FCFE01464FF07A
:1023F0007E5013F0ABFF60604846616813F0EAFD61
:102400000146484613F0A2FFD4F8008081464146B9
:10241000584613F0DDFD0146484613F0E3FE014641
:10242000404613F0D7FD206014F0A2F86C4A079BD9
:10243000D05204E055F82A10694A22F81A100AF11D
:10244000010ABAF1030F04F10C04B3D16449B1F8E5
:1024500002A0B1F800900FFA8AF252430FFA89F302
:1024600003FB03228B8864210993BDF9243003FB0D
:10247000032301FB03F25B4B1B895B4392FBF3F3EA
:10248000523B0B93049B1A68110706D5564B1968EB
:1024900019B1596809B19B687BBB544B197801F09D
:1024A000100000F0FF0360B312F0200329D001F008
:1024B000020202F0FF0322B34D4B1B78042B1FD9FD
:1024C0004C4B1B88B3F5967F1AD34B4BB3F90400E2
:1024D00013F034FE494B0446188813F02FFE484988
:1024E00013F034FF0146204613F072FD454913F006
:1024F00079FE00248046012306E00023012401E048
:1025000000231C464FF0000806980D9313F012FEAE
:10251000314913F067FED6F804513B4E0490306801
:1025200013F00CFE294613F05DFE0790706813F05F
:1025300005FE294613F056FE0890B06813F0FEFD24
:10254000294613F04FFE2849834607988B680F6889
:102550004D6801460A9313F045FE06460898014669
:1025600013F040FE0146304613F034FD594606464E
:10257000584613F037FE0146304613F02BFD17F096
:1025800043F80D9B0C90002B44D040461F4913F09C
:10259000E5FF28B14046114913F01AFD8046F4E7E3
:1025A00040461B4913F0BCFF28B140460B4913F0CD
:1025B00011FD8046F4E74FF07C51404613F012FEC7
:1025C0000BF020F8002113F005FD064623E000BFC4
:1025D0000C390020E40A0020BD378635DB0FC940E6
:1025E000CE0F0020C8160020A0270020882F002032
:1025F000F80F0020F40F00205C2F0020C0100020F6
:102600000000204135FA8E3C782F0020DB0F494036
:10261000DB0F49C00026002C00F0A180384613F0E3
:102620008DFD0746284613F089FD05460A9813F0EC
:1026300085FD39460446384613F0D4FD29468046C8
:10264000284613F0CFFD0146404613F0C3FC214657
:102650008046204613F0C6FD0146404613F0BAFC02
:10266000A349804613F07AFF002878D0404616F040
:10267000CBFF01464FF07E5013F068FE804638468F
:10268000414613F0AFFD41460746284613F0AAFD28
:1026900041460546204613F0A5FD964C804621682C
:1026A000384613F09FFD61680A90284613F09AFDA2
:1026B0000A9B0146184613F08DFCA1680A9040461B
:1026C00013F090FD0A9B0146184613F083FCE16865
:1026D0000A90384613F086FD21690746284613F014
:1026E00081FD0146384613F075FC61690546404698
:1026F00013F078FD0146284613F06CFC0A9B054652
:102700001946184613F06EFD29460746284613F071
:1027100069FD0146384613F05DFC16F075FF014671
:10272000284613F05FFD00F10048A169404613F010
:1027300059FD002113F04EFCE1690746404613F0B5
:1027400051FD002113F046FC216A0546404613F076
:1027500049FD0146304613F03DFC064601E00025E8
:102760002F460B9B262B00F286800FFA89F013F080
:10277000E5FC81460FFA8AF013F0E0FC0446BDF94F
:10278000240013F0DBFC49468046484613F02AFD3E
:1027900021468246204613F025FD0146504613F09F
:1027A00019FC41468246404613F01CFD0146504646
:1027B00013F010FC4E49824613F0D0FE00285AD088
:1027C000504616F021FF01464FF07E5013F0BEFD3B
:1027D00082464846514613F005FD51468146204643
:1027E00013F000FD51460446404613F0FBFC414BFC
:1027F00082461A6A20461146D3F81C800A920B932F
:1028000013F0F0FC41460990504613F0EBFCDDF864
:1028100024C00146604613F0DBFB0146384613F046
:10282000D9FB0B9B07469B6950461946099313F049
:10283000D9FC0A9A82461146484613F0D3FC014659
:10284000504613F0C5FB0146284613F0C3FB414632
:102850000546484613F0C6FC099B804619462046AB
:1028600013F0C0FC0146404613F0B2FB014630466F
:1028700013F0B0FB0646059B4FF00009D3F8048027
:102880004946404613F06AFE1B4C002838D00C988D
:102890001A4913F045FE002838D03946404613F057
:1028A000A1FC049913F09EFC0146D4F8080113F032
:1028B00091FB2946C4F80801404613F093FC0499A3
:1028C00013F090FC0146D4F80C0113F083FB314661
:1028D000C4F80C01404613F085FC049913F082FC07
:1028E0000146D4F8100113F075FBC4F810010DE097
:1028F0000AD7233C24260020040A0020C2B8B23E96
:10290000C4F80891C4F80C91C4F81091059B98681C
:10291000064B1B785B0705D4054B1A6844F61F630A
:102920009A4207D94FF07E5105E000BFDB3A002004
:1029300018150020A64913F055FC3946804613F0BF
:1029400051FCD4F8081113F045FB0146079813F029
:1029500041FB29468146404613F044FCD4F80C1153
:1029600013F038FB0146089813F034FB3146074654
:10297000404613F037FCD4F8101113F02BFB01463E
:10298000584613F027FB4FF07C518246049813F011
:1029900029FC05464846294613F024FC29460646EC
:1029A000384613F01FFC29468046504613F01AFCA7
:1029B000884B8246D3F800B0874B3146D3F800905D
:1029C000864B09F100401F68854B1D6813F00AFC17
:1029D00041460790384613F005FC079B0146184610
:1029E00013F0F6FA51460790284613F0FBFB079BBD
:1029F0000146184613F0ECFA0146584613F0EAFA7D
:102A0000744B314618600990584613F0EBFB514661
:102A10000790384613F0E6FB079B0146184613F073
:102A2000D9FA41460790284613F0DCFB079B014684
:102A3000184613F0CDFA0146484613F0CBFA664B20
:102A4000414618600890584613F0CCFB5146079059
:102A5000484613F0C7FB079B0146184613F0B8FA27
:102A600031460790284613F0BDFB079B01461846E8
:102A700013F0B0FA0146384613F0ACFA574A514603
:102A800010600790584613F0ADFB41468246484619
:102A900013F0A8FB0146504613F09CFA31468046DD
:102AA000384613F09FFB0146404613F091FA014669
:102AB000284613F08FFADDF824C0494B61461860B0
:102AC0000546604613F08EFB089A064611461046EE
:102AD00013F088FB0146304613F07CFA079B06464C
:102AE0001946184613F07EFB0146304613F072FA81
:102AF00029460646284613F075FB0146304613F07A
:102B000069FA16F081FD01464FF07E5013F01EFC6D
:102B10000546304B2946186813F064FB2D4B2946B7
:102B200018602D4B2F4E186813F05CFB2A4B29467A
:102B300018602A4B186813F055FB284B294618607B
:102B4000274B294D186813F04DFB254B18600CF0EE
:102B50006BFE296AE8690AF0D3FC244913F042FBB2
:102B600016F08CFB3080A86900F100400AF08BFC65
:102B700001461F4813F02CFA1C4913F033FB16F0E2
:102B80007DFB29687080E8680AF0BAFC174900F1FB
:102B9000004013F027FBD4F8141113F01BFA16F0C1
:102BA0006DFB83B213F4004F16BF00F56160B38074
:102BB000B0802C462E6A0F4D3046D5F8181113F010
:102BC000CDFC0D4B1A78C8B142F0080218E000BFE6
:102BD000000020412C000020182600201C26002088
:102BE000202600205C2F0020242600204C3D0F448E
:102BF000DB0FC93F040A0020882F002022F00802C2
:102C0000954F1A70B7F9000013F098FA8146B7F99A
:102C1000020013F093FA8046B7F9040013F08EFA1D
:102C200021680746484613F0DDFA6168824640464F
:102C300013F0D8FA0146504613F0CCF9A168824649
:102C4000384613F0CFFA0146504613F0C3F9A16994
:102C50008246484613F0C6FAE1698346404613F0BF
:102C6000C1FA0146584613F0B5F939468346304655
:102C700013F0B8FA0146584613F0ACF9E16806467D
:102C8000484613F0AFFA21698146404613F0AAFA8C
:102C90000146484613F09EF961698046384613F0B4
:102CA000A1FA0146404613F095F9059B00F1004753
:102CB0005B78012B18D1694B1B7858070ED4D5F8D7
:102CC0001C01402390FBF3F3C01A13F037FA31468E
:102CD00013F080F913F04CFCC5F81C01D5F81C0169
:102CE000402390FBF3F001E05D4B188913F026FAC6
:102CF0000146304613F06CF9D5F8241106460498C5
:102D000013F068F90146049813F020FBD5F8204130
:102D100080462146304613F05BF90146404613F0E9
:102D200061FA0146204613F055F9C5F82001064620
:102D3000504616F0A3FAD5F828514A4C29780AF0E3
:102D400093FB236818442060384616F097FA2978D8
:102D50000AF08AFB636818446060304616F08EFA09
:102D600069780AF081FBA3683F4A18440699136802
:102D7000A060194411603D4A13680133136003E0F9
:102D800000232B606B60AB60394BB3F90610394BF5
:102D90001F687A8991420EDBB1F5FA6FFD79BFBFEA
:102DA0008B1A6B43A2F5FA6593FBF5F5ACBFC5F141
:102DB0006405643500E064252F4B0022B3F810E071
:102DC0002E4B1B6804932E4B1E680593284B4FEA2D
:102DD000420833F912C0CEEB0C03002B05DDB3F52E
:102DE000FA7FA8BF4FF4FA7306E0CCEB0E03B3F5FD
:102DF000FA7FA8BF4FF4FA73022A49D0049C2478C2
:102E00001CB1A342CCBF1B1B0023642093FBF0F931
:102E10001C4C6FF0630B34F819A00BFB093B09F154
:102E2000010934F919400FFA8AF9C9EB040404FBCB
:102E30000BF494FBF0F41448544420F80840BC18F8
:102E4000247964206343114C93FBF4F364339BB205
:102E50006B4393FBF0F048E0CE0F0020DB3A0020FC
:102E6000C816002064270020BC39002060270020FD
:102E700000340020F030002074360020C00F002005
:102E80008027002078240020642F00200CFEFFFF04
:102E9000049844781CB1A342CCBF1B1B00236420C0
:102EA00093FBF0F0DFF80CA36FF0630909FB003B24
:102EB0003AF9104001303AF91000002BA0EB040061
:102EC00000FB0BFB9BFBF9FB0498C4EB0B0490F994
:102ED00004B0A3480BFB04F48480B879B8BF5B420C
:102EE0004343A04893FBF0F0643033784FF064091B
:102EF000434393FBF9F39C4C022AA354B37A9B4CB3
:102F000000FB03F393FBF9F3A354337D944C00FBD4
:102F100003F090FBF9F0964B9854964B0ED1F44584
:102F200083F802900DDB944B5A8A0493914214DB90
:102F3000B1F5FA6FA8BF4FF4FA610FE0F4459D5464
:102F400004DA34F808305B4224F808300132032AEE
:102F500006F101067FF43AAFE5E71146891A4FF40E
:102F60007A735943C2F5FA62B1FBF2F1642391FB23
:102F7000F3F2824F6FF0630037F8126000FB02112A
:102F8000013237F9122030B2121A514391FBF3F398
:102F90003344E3807A4B724D1B8859063FD5794BF9
:102FA0000A20B3F9043093FBF0F0774B1B88C01A6A
:102FB00000B213F0C3F8754913F014F906460AF08D
:102FC00095FB074630460AF01DFB0646B5F90200A0
:102FD00013F0B4F88046B5F9000013F0AFF83946A5
:102FE000814613F0FFF831468246404613F0FAF866
:102FF0000146504612F0ECFF13F0BAFA3946288029
:10300000404613F0EFF831460746484613F0EAF819
:103010000146384612F0DEFF13F0AAFA6880049BDE
:103020005B4D9B7B002B4FD0AB89B5F83011B1FBCA
:10303000F3F1584B481C1B7880B2A5F832011BB342
:10304000B5F934A10023524E0FFA80F906F59B78AA
:1030500038F9132006F59F7E0AFB02F292FBF9F283
:1030600034F813C03EF813702EF813C0C7EB0C07EA
:10307000174428F813700133042BE4D1454B002288
:103080001A70A6F8341104E0B5F83431013BA5F804
:1030900034313F4A0023B2F93401002812DDB2F97D
:1030A00032613D49A1F1080232F9132031F81310C1
:1030B000424392FBF6F28A1A24F813200133042BC0
:1030C000EFD101E0A2F83431344B01221A70344BB5
:1030D0009B680BB133489847334F344E3B682848C0
:1030E00013F0080F71D0A188DFF8CCE001F10E03D6
:1030F0009BB21C2B234BB3F9043061D802885207D2
:103100005ED50A2293FBF2F2BEF80030D21A92B2D8
:1031100093B20FFA83FE1EF1B30FBCBF02F5B47376
:103120009BB21AB2DFF894E0B32A214A9EF800E07D
:10313000C8BFA3F5B4731268C8BF9BB21EF0080FD6
:10314000127942D052B25242534332681BB2127AC1
:1031500053431E2293FBF2F3CB1AA38035E000BF4A
:10316000642F00200CFEFFFFA02F0020300B00205A
:1031700024300020843000207436002052240020A7
:10318000622F00205C2F0020000F002035FA8E3CBB
:10319000040A0020960F0020420B0020970F002009
:1031A000D41600204A0B00208C1700208027002016
:1031B000C00F00206A240020FE0E0020882F00206F
:1031C0000A2293FBF2F3AEF800309E4B1B68DA0242
:1031D0006BD5B0F8008008F400681FFA88F8B8F1E1
:1031E000000F4ED1984B1B785B074AD54FF4006017
:1031F00007F0C4FA31688B7F022B944B04BF012285
:1032000083F84821D5F84C2118BF83F848811089EC
:103210004FF47A7343438E48008893FBF0F38D4854
:103220005B429BB290F800E0A5F850310D460021BA
:10323000D67810780EB1B04204D8BEF1030F03D88F
:10324000022901D10026D6702E780132864238BF7D
:10325000287015F8016B7D48B60100F5A97C2CF8A3
:10326000116000F5AC764FF0000C26F811C000F5A7
:10327000AF7626F8113001310329D9D1012380F826
:103280006431754B1B881D051AD46F4B1B7803F0F6
:10329000040303F0FF069BB96C4D95F864317BB1D4
:1032A00007F02EFD85F864610AE00388180507D54C
:1032B000654B1B78590703D54FF4006007F04EFAB1
:1032C0003B68624D13F0140F6FD0634B1B8803F4FF
:1032D0000273002B69D0614B1B7803F0100303F0DD
:1032E000FF0643B15E4B95F965211968638801FBC0
:1032F0000233638059E05B4B5B4A1B685B48D978BB
:103300009B7809B3B2F906E0B0F90010C1EB0E02E8
:10331000002AB8BF52429A420CDD554A8E451660CB
:103320004FF0010285F86621E288C8BF5B42134472
:10333000E3803AE095F866313BB34E4B85F8666121
:103340001A684D4B1A6020E0B0F90000B2F906206F
:10335000121A82EAE270A0EBE27098420ADD0223C0
:1033600092FBF3F2454B1A60454A0123137085F82E
:1033700066310AE095F866313BB13E4B85F866113F
:103380001A683D4B1A603E4B19703E4B3E49B3F9EB
:103390000020334B1B6813440A884988934203DB9F
:1033A0008B42A8BF0B461A46E280384B384E1B783A
:1033B0009BB12D4BB3F90620364B5B8A9A420CDC4D
:1033C0003378012B01D0192B01D1B2792AB90E2BF8
:1033D00003D0082B1CBF0023A380D5F8683193F8D5
:1033E0000280B8F1000F61D01B4B1B889A075DD09B
:1033F000294B2A49D3F82090484613F09BF800281F
:1034000050D148460AF03FF8104BD3F86C1112F037
:10341000E9FE15F033FFB0F5617FA8BF4FF461708E
:1034200012F08CFE1E4912F091FF0AF0EBF8814673
:10343000404612F083FE494612F0D4FE15F01EFFFE
:1034400080B230E0842F0020DB3A0020040A002004
:10345000D03900206C250020622F0020882F00200A
:1034600088270020C00F002000340020980F002083
:1034700084270020A81000207C270020C0390020CD
:103480008C2700209A0F00204624002006000020F0
:103490005031002074360020242600208FC2753C55
:1034A000EFB6B0440020E3881844E0803B689B06F8
:1034B00040F19A80B44B1B8803F03003002B00F0DE
:1034C0009380B24B1B78DF0740F18E80B04BB3F98D
:1034D00004000A2390FBF3F012F030FEAD4912F025
:1034E00081FE07460AF08EF8804638460AF0FEF85C
:1034F000A94B07461B68DA78A84B002A3DD0DFF8B5
:10350000A0A2B3F90200BAF8029007920FFA89F16B
:10351000401A069304F008FC079A5146C2F1000BCA
:103520005845069B03DB9042A8BF104600E0584672
:1035300000EB090AB1F80090B3F900000FFA89F323
:103540001FFA8AFAC01A0692A1F802A004F0ECFB56
:10355000584504DB069A9042A8BF10468346D944DA
:103560008F4B1FFA89F9A3F800900FFA8AF012F036
:10357000E5FD83460FFA89F008E0B3F902000693EF
:1035800012F0DCFD069B8346B3F9000012F0D6FD75
:1035900039468246584612F025FE4146069050466E
:1035A00012F020FE069B0146184612F011FD7D49DF
:1035B00012F0CCFE12F0DCFFDFF828924146A9F8A9
:1035C0000000584612F00EFE39468046504612F072
:1035D00009FE0146404612F0FDFC724912F0B6FEAB
:1035E00012F0C6FFA9F802006F4B5A89049B0093A2
:1035F0006E4B1F68059B18686D4B19686D4B1B68F7
:10360000B8476D4B6D49DB7804936D4B1F78032FE2
:1036100016D9B6F804E0BEF5FA7F11D2B4F9040069
:10362000B1F904C00028B8BF4042CEF10002131A1D
:103630009C4504DB0EEB00036345A8BF63468B800B
:10364000604B1B6813F000600FD196F90280E3888D
:10365000C8F10002B1F90480B1F80290B1F800A0FD
:1036600008FB02F8584D044674E196F902B04FF099
:103670000008CBF10003B1F904B046460BFB03FB95
:1036800043464A88B1F800A0DFF85C91BB423ED2C5
:1036900010B20793069212F051FDD9F8081012F0FB
:1036A000A1FD05900FFA8AF012F048FDD9F8041038
:1036B00012F098FDDDF814C00146604612F08AFC55
:1036C0000590584612F03AFDD9F80C1012F08AFD18
:1036D000DDF814C00146604612F07CFC12F048FF91
:1036E000079B80B20FA921F813000FFA86FE01B2E2
:1036F0007145069A04DC0FFA88FE714502DB3046FC
:1037000006464046013309F110098046BEE72F4BBB
:10371000C8EB060A1A681FFA8AFA12F4805FDFF80B
:10372000CC90984664D02A4B1B7813F0040F294B99
:1037300008BF1A8A188A284B08BFA5F830221B68D0
:10374000264AD788DA883CB2811A8C42244B03DCA3
:103750001E88B9F8004005E00244944205DBB9F840
:1037600002605C88A5F8307247E0B5F930228A42E1
:10377000D7BF1E885C88B9F800403746C4BFB9F887
:103780000260274639E000BF622F0020882F00200A
:103790005C2F002035FA8E3C040F0020160F00200D
:1037A000120F002000002041D00300203C03002025
:1037B000F0300020101600201C15002028300020BA
:1037C0006C250020842F0020800B00207036002004
:1037D000DB3A002074360020C00F002000340020A7
:1037E00010260020D4390020740B0020462400202D
:1037F000E788B9F80260B9F80040B6B21FFA84FB56
:10380000CBEB06040FFA8AFA24B2A245B04B2ADDAC
:1038100001221A70204612F091FC0646504612F022
:103820008DFC0146304612F091FD82460026A94BE0
:103830001B789E420FD20FAB33F91600059312F09E
:103840007DFC514612F0CEFC15F018FD059B23F8C7
:1038500016000136EBE7022094FBF0F00BEB0004BE
:10386000A4B226460AE000221A7002239AFBF3FA59
:103870000BEB0A04CAEB0606A4B2B6B2D8F80030C5
:10388000B9F8042003F480530993B5F93032B9F83C
:1038900002B00593904BB9F800901B8A8F4D0693A8
:1038A0008F4B4FF000081B6807938E4B19885B887D
:1038B0000891884991F800A04FEA4A0AD04500F0E3
:1038C00030810FA938F801C038B20C920B93CDF8B3
:1038D00028C012F033FC844951F8381012F082FCF1
:1038E00012F046FE21B28842DDF828C00B9B0C9AEC
:1038F00003DB31B28142A8BF01468C4404991FFA10
:103900008CFC25F802CF0FFA8CFC19B1944517DA1C
:1039100094461AE0099989B107990698C988411A0D
:103920000598884206DCCC450EDB08998C45A8BF7B
:103930008C460AE09C4503DA9C4606E0CC4503DB56
:10394000DC45A8BFDC4600E0CC46A5F800C008F185
:103950000208B3E7BC42DFF8A0B137D218B2069331
:1039600012F0ECFB55F80C1C12F03CFC05900FFA21
:1039700089F012F0E3FB55F8041C12F033FC059AB1
:103980000146104612F026FB05900FFA8AF012F05D
:10399000D5FB55F8081C12F025FC059A0146104687
:1039A00012F018FB0590404612F0C8FB55F8101BAA
:1039B00012F018FC059A0146104612F00BFB12F0AB
:1039C000D7FD069B2BF814000134C3E7BBF80010A9
:1039D0000122BA420BB207D23BF9121001328B42DC
:1039E000B8BF0B4699B2F4E7404A96F80180508878
:1039F00083423F4BC8BF091A1B68C8BF89B203F492
:103A000080520B923B4A03F01003B2F90640324A4F
:103A10000C93168A324AD8BF002112680592314AA7
:103A2000B2F80090B2F802E01FFA89F207922F4A2A
:103A30001FFA8EF5B2F800C006959588264A1FFA3F
:103A40008CF3528A0A9308922B4AABB2099302EB89
:103A500047030D930D9B9A4263D013880B9F5B1A0B
:103A60009BB222F8023B07B3B8F1000F09D1059FC2
:103A7000B7F806A0CAEB060B5C4502DDB24454451C
:103A80000CDBB4421BB203DD734514DA734645E028
:103A9000AB4214DB4B45A8BF4B463FE0B442CCBF22
:103AA000BDF81830BDF81C3038E0049F4FB132F932
:103AB000023CAB4203DB8342A8BF03462EE02B4609
:103AC0002CE01BB2634519DB8342A8BF034616E016
:103AD000892F00206C25002074360020222500202C
:103AE000C00F002010260020740B00204624002068
:103AF000703600200034002024250020634622F880
:103B0000023C089B9C42A5DA0C9B13B1BDF8243003
:103B100004E0B8F1000F9DD1BDF8283022F8023C36
:103B200098E7B7490A788B4602F0040202F0FF03D7
:103B30003AB1B44B1B78013BDBB2182B00F2208169
:103B40000BE0B14A12789342F3D2B04931F8130036
:103B5000AF4921F813000133F5E701229A40AD4B3C
:103B60001340002B00F00C81AB4BAC491B88AC48D8
:103B700013F4807F08D0AB4B1A88ADF83C205A88EC
:103B80009B88ADF83E2013E0A74B1A88ADF83C2087
:103B90005A889B88ADF83E20A44AADF840301268A0
:103BA000D40407D5B1F90640028A944202DA5B4296
:103BB000ADF840309E4D4FF47A72B5F902304FF4B3
:103BC000616403F5E163534393FBF4F3A3F5FA73E4
:103BD000ADF85430B5F9003003F5E1635A4392FB78
:103BE000F4F28B4BA2F5FA721B88ADF85620A3F2C3
:103BF000DC53ADF842300A88038AD21AADF844206B
:103C00004A88D21AADF846208A88D21AADF84820E0
:103C1000CA88D21AADF84A200A89D21AADF84C20C7
:103C20004A89D21AADF84E208A89D21AADF85020AE
:103C3000CA89D31AADF8523000237E4A002122F8F7
:103C400013100133082BF8D17B4B7C491B687C4D4A
:103C500005937C4B1B6804937B4B1B78C3EBC3031E
:103C600001EB0308414573D00B7833B11533DAB259
:103C700001239340059A134066D0049B11F806EC8B
:103C80000E2707FB0E37B7F90020B7F90230642082
:103C90009B1A11F9022C9BB25A4392FBF0F211F8D5
:103CA00005AC4FEA530911F8034CC9EB02024FEA85
:103CB0004A0616A892B211F801CC064414B936F897
:103CC0001C0C0CE0B5F9000036F91C6CB04208DAA7
:103CD0000444844203DBA6423046A8BF2046288025
:103CE00008E007DD041BB44203DB8442A8BF04469E
:103CF00026462E80D7F80A40012000FA0AF020421A
:103D0000B5F9006011F9040C12B200FB06F04FF097
:103D1000640690FBF6F014BF4FF0FF34012490428C
:103D20000ADB4FFA8CF25A4392FBF6F2C9EB02021D
:103D300012B28242A8BF02463E4B33F81E9002FBED
:103D4000049423F81E4000E02B800235073189E7F8
:103D50003C4B3E4E1F6800250E2303FB057393F971
:103D6000064036F9023FE8B26343642493FBF4F45F
:103D700034800BF0A9FC01352044082D3080EBD1B4
:103D80002A4E2C4C33682F4D13F0200F33D00020D7
:103D90000BF09AFC2080074601200BF095FC264B87
:103DA00060801B681A0626D5294B214AD3F8543265
:103DB0001B78012B4ED12968B2F9003091F914E03B
:103DC0004FF0320C03FB0EF393FBFCF31FFA83FE60
:103DD00091F90630B2F902205B4253436FF0310192
:103DE00093FBF1F193FBFCF30EEB0102B918734462
:103DF000218018446080D5F800E0002344E000BF33
:103E0000DB3A0020503100206C2500201A310020C0
:103E10002425002099209801622F002000340020E2
:103E200074360020642F00202830002070360020D7
:103E30005C2F0020F0030020842F0020B3240020FA
:103E4000360C0020C8320020AC240020EE030020F5
:103E5000040A0020D5F800E0B2F902309EF90610FD
:103E60005943322391FBF3F1394421809EF91470B8
:103E7000B2F9001001FB07F292FBF3F21044B9E72C
:103E80000133082BE25310D00E2101FB03E134F97A
:103E90001300B1F900205F009042B1F90210EFDB8E
:103EA0000AB28242A8BF0246EAE7A34F97F90C3054
:103EB00093B93B78013B182B73D8DFE803F03772D6
:103EC00072507272724972727272725A7272727235
:103ED00072506672725A3700DFF884924FF0000811
:103EE00039F9020F12F02AF9944B242101FB083111
:103EF00009F00DF815F0C2F92B680E2202FB08320A
:103F000080B2A9F80000B2F9003000B29842B2F9CC
:103F1000022003DB13B28342A8BF034608F1010865
:103F2000B8F1080FA9F80030DAD1C2E7BB7913B1B4
:103F30000020618908E09BF8003003F0040303F0DF
:103F4000FF00002BF4D101460DF064FB012529E0B0
:103F50000020E1880DF05EFB0120218905E00020B2
:103F600021890DF057FB618901200DF053FB0225DB
:103F700018E00225A81E34F81510C0B201350DF066
:103F800049FB082DF6D106250CE00325E81E34F880
:103F90001510C0B201350DF03DFB072DF6D10425FB
:103FA00000E0002533689B0602D43B78052B0AD13C
:103FB000284621880DF02EFB681CC0B261880DF0E8
:103FC00029FB0235EDB23368DF0206D45C4C94F86D
:103FD000783373B10BF092FB0BE05A4F0024281991
:103FE000C0B237F8021F0DF015FB0D2CEED00134D6
:103FF000F5E7554B1878002840F0B98133681D0368
:1040000040F1B581514D2B78033B052B1ED8504B09
:104010009B7833B1012B09D104F068F9C0F17F001E
:1040200004E0D4F87C0303689B689847D4F8803395
:1040300094F884231344B3F5807FA8BF4FF48073B2
:104040008342D4BFC4F88033C4F880032B78023B8A
:10405000092B00F27C81DFE813F00A0015004C0008
:1040600085009B00B400C600340151015C010023AF
:10407000C4F88033C4F88833364B1B68C4F88C33DB
:10408000032363E1334B1A68D4F88C3364339A42C8
:1040900040F25D81402006F09FFE002840F05781ED
:1040A0004FF040082C4BD4F88823254F985C1E46CF
:1040B00080B105F057F9D7F88033B8F1010803F162
:1040C000FF33C7F88033D7F8883303F10103C7F80B
:1040D0008833E7D1D4F88823194BB25C002A40F02A
:1040E0003681C3F888234FF0FF32C3F88C230423B2
:1040F0002CE126230093194B492003F10C02019374
:1041000002925021A3F10A02023305F0EFFC0028CD
:1041100040F01D8133684FF0FF3213F080030FBF72
:10412000C4F88833C4F88803C4F88C23052304BF7B
:10413000C4F88C23072309E1503100205C0C0020D7
:10414000040A002006340020DC3A0020E0030020AE
:10415000E10300201815002084A10108EEA1010848
:10416000EE030020834A0223002100930191029173
:10417000482002F1080305F0B9FC002840F0E78070
:104180004FF0FF33C4F88C33C4F888030623DDE016
:10419000794B072603F10C02019302920096A3F1DA
:1041A000080247200021043305F0A0FC002840F05D
:1041B000CE804FF0FF33C4F88803C4F88C332E70E0
:1041C000C5E06E4A0523002100930191029153201E
:1041D00002F1080305F08AFC002840F0B880C4F81A
:1041E00088030823B2E0402006F0F6FD002840F0E6
:1041F000AE80D4F888330D2B00F2AF80DFE803F0F7
:10420000070B0E12171E282C303438454D515C48D0
:1042100005F0D0F84FE05B485B4916E05B485C492D
:104220005C4A46E05C4B5D4819785A7841E05C4B4B
:104230005C4893E8060008331B682BE05A4B5B4848
:104240001A780C2353435A4AD15C05F0B3F832E094
:10425000584B59481988F8E7564B58485988F4E79D
:10426000574B58481969F0E7574B58481989ECE7FC
:10427000D4F89033D80403D5554B56481978E4E761
:10428000554B0C22C3F8882315E0514B534819793C
:104290005A79DB7805F08EF80DE05148B4F89413A4
:1042A000D3E73368190506D5494B4E481989B3F948
:1042B000062005F07FF8D4F888330133C4F888333A
:1042C00045E0494B1B689A0115D5B4F89833424E26
:1042D0008BB9D6F89C330E200F93444B0FA91B6863
:1042E000109305F0F5F84FF48053A6F896330A239F
:1042F0002B7005F045F905F0CDF828E094F8A033CF
:10430000002BF6D0384B1B689B01F2D409232B708D
:10431000F1E7374B1A68D4F88C33C8339A4203D983
:104320001D4B9E788EB904E006F09AFD0028F7D167
:104330000DE0D4F87C030AF081FE94F8A133C4F8B0
:104340007C63022B01D104F013FC01232B7006F0D7
:1043500071FD60B101232B7009E006F081FD00289A
:10436000F5D04FF48053A4F896330A23EEE717B044
:10437000BDE8F08FACA30108C4A3010810A4010894
:10438000CCC50108E6C50108E3C40108FBC5010866
:10439000CEC40108DAC40108E10300200FC60108F9
:1043A000E8F7FF1F20C601081831002034C60108B5
:1043B000F4300020462400203EC601084DC6010806
:1043C000D41600205CC60108C81600206CC601087F
:1043D0009814002076C60108040A002083C601084C
:1043E0009CC60108A7C60108842F0020B839002008
:1043F000181500209B492DE9F04F0A689A4C02F5E8
:104400009C4320332360994B89B01E788946B6B10E
:10441000974909688A4240F2FC80013E1E70F8E02C
:10442000072D96BF934B2946E95C934B93481B6835
:104430009847032D0AD904EB4505A88001368F4B18
:10444000F5B21A781946AA42EAD81EE00028F2D03E
:104450008B4A4FF47A7332F8251002EB8502401A2A
:10446000584353885B1A90FBF3F040F6C90300F5FC
:104470007A70984205DC40F2EE239842B8BF1846A5
:1044800001E040F6CA0080B2D5E742F201067D4B5A
:104490001B681E40B6FA86F67B4B76091A6836B959
:1044A00094F8293084F82830784B5878187094F8AC
:1044B00028701FB1754B1F7887F001070F2384F810
:1044C0002A306C4B91F800A0B3F816B01B8B032177
:1044D000019394F82B30DFF8C881B3FBF1F101EBC5
:1044E0004101591AC9B202910025554554DADFF845
:1044F000B4E13FB3AEF1700131F81500584502D375
:104500000199884222D95EF825005749824203D298
:104510005F4931F815001DE0E8B20493039205915C
:1045200004F06CFA032D039A049B13DC05994FF0F9
:10453000010C91F82AE00CFA05FC2EEA0C0E81F829
:104540002AE007E0BBF1000FDDD1584602F5967175
:104550004EF82510CEB9029928F81100424991F879
:10456000BCE0BEF1000F04D1022B0ED9012081F86E
:10457000BC00B8F80010B8F802000844B8F80410FD
:10458000084480B20321B0FBF1F0414908F106086C
:1045900021F815000135A8E794F82A203A49A2F13C
:1045A0000F067242724184F8BD203A4B92B13A4AEA
:1045B0001268550103D5334A1268D0050AD40A6837
:1045C0009A60DB68D21AC82A1ED9324B012283F8BE
:1045D000212019E02D4A0120507010700A68996856
:1045E000DA605B68521A9A4282BF2A4B002283F833
:1045F00021200025554507DAE8B204F0FFF9244BE5
:1046000023F815000135F5E794F82B30013384F8D1
:104610002B301C4E3368D90405D51F4B1B68DA07B5
:1046200001D410F0D9FC134BD9F80070D87A01935B
:10463000002839D0164A5B7B013832F810001BB1D4
:10464000C0F53B60083080B200B2A0F57A70B0F5DA
:104650007A7FA8BF4FF47A7020EAE07011F06EFD07
:104660000E4957E0B8390020DC0D00201415002059
:1046700010150020743600205400002094360020CD
:10468000FE150020703600201815002004000020C0
:10469000003400201C150020842F002000007A44E4
:1046A000080E0020500E002033681B043BD5D4F8C0
:1046B000C030AC4DFB1A002B35DB07F59C43203393
:1046C000C5F8C030A84B95F8C4105A79A74B0131F2
:1046D00033F81230019A9BB2127B93FBF2F301F094
:1046E0000F0285F8C4202A4482F8C5300346A04A48
:1046F000825C0130134410289BB2F8D11BB293FBAB
:10470000F0F000B26428A8BF642020EAE07011F045
:1047100015FD984911F01AFE974911F063FD11F04B
:104720004DFF964B18803368954D13F4807F00F051
:10473000FE80944BDFF850929F4205D999F80220F1
:1047400012B9012289F8022099F80220002A00F00B
:10475000EE808D4A95F8008092F821708B4A07F11F
:10476000FF3E9246DEF10007116847EB0E07002F6F
:10477000C1F38063C8F38008029314BF4FF0000BAD
:104780004FF0030B99F82020052A00F2CA80DFE8D9
:1047900002F0034A5D8594B1B8F1000F36D07C4A2F
:1047A0001268D0880FF022FD012809D1794A7A4990
:1047B0001268B1F80510642000FB0122C9F810202E
:1047C000029B53B1744A12793AB110F0C5FF03222B
:1047D00089F820204FF47A7235E0002F40F0A18054
:1047E0006C4AD9F810101068674A88420AD90392B7
:1047F00010F0B2FF039A032182F8201040F6B8317E
:10480000D161BFE7012182F82010BBE7029B4FF482
:10481000806013B105F0B2FF01E005F09FFF0022B8
:10482000C9F810207DE0002F59D15B4AD279012AC6
:1048300002D010F091FFA5E710F08EFF032289F857
:10484000202040F6B832C9F81C209BE727B105228A
:1048500089F82020012000E03846B8F1000F0ED082
:10486000019B4E491A8A4C4B0A804A808A809A786A
:1048700093F803E04FF0020B42EA0E22CA80454A49
:104880001168D9F81420914202D8B8F1000F45D12F
:1048900047F23052C9F81C20032221E02A7842F066
:1048A00002022A7010F098FB3A4AD9F81C101268DC
:1048B0000A44C9F81820042212E0364A9FB1116850
:1048C000D9F8182091422CD9354A92781AB9DAF8D9
:1048D0000020D00725D42A7822F002022A7005226F
:1048E00089F820204EE71268D9F81C100A44C9F84C
:1048F000182016E0274A28491268B1F805106420EC
:1049000000FB01224FF48060C9F81020002289F8D2
:10491000202089F8032005F021FF33E700287FF4E9
:1049200031AFBBF1000F02D058460AF02DFD184BF5
:104930001A4F1B68D8880FF059FC019BB7F9022069
:104940001B8A824603F10B0191422BDB0B3B934206
:1049500028DCB7F90020914224DB9342CCBF00232E
:10496000012320E0DC0D0020AE140020BE14002046
:10497000A10E00200000C84200C07F44AC100020FF
:10498000DB3A0020404B4C001C150020842F0020F7
:10499000C00F002018150020A93900200034002085
:1049A000040000200023BAF1000F0FD18D4A1268D5
:1049B000110111D58C4AD27872B92A7852070BD5D9
:1049C00023B18A4A137843F0200303E0874A13781F
:1049D00023F0200313700CE0854A00238548136000
:1049E0005360854A00210360116043605160836019
:1049F00091602B78580739D53368D90636D57B4B6B
:104A00001B78DA0632D47D4B9B789BB1BAF1000F4C
:104A100018D194F8D730DFF8EC8173B1784B1A686D
:104A2000D8F8DC309B1A002B07DA10F0D5FA88F89A
:104A3000E0A01BE0BAF1000F10D110200AF0A4FC96
:104A4000012311E094F8D73043B16D4A4FF47A71E5
:104A5000126801FB03236B4AC2F8DC3094F8E030A3
:104A600023B10AF07BFC002384F8E030019B002294
:104A7000B3F812E0B3F814C0134694F8D59094F844
:104A8000D60037F912109B087145C4BF63F07F034D
:104A9000DBB201326145B8BF43F04003042AF0D1D4
:104AA00094F8E12057499A4205D191F8E220F92A79
:104AB00004D8013200E0002281F8E22084F8E130DD
:104AC0004E4B9A789846EAB9464B1B68DB0708D5E7
:104AD000BAF1000F16D12B78D80713D510F0C8F80B
:104AE00010E02B7859070DD5464B93F828304BB181
:104AF0003D4BDB7833B910B110F06EFA02E0BAF139
:104B0000000FF9D094F8E230DFF8F8A0142B40F051
:104B1000988098F8023019F1000918BF4FF0010988
:104B20003BB39AF8E1305F2B0DD12B7803F00403EF
:104B300003F0FF0B13B110F04FFA04E00B200AF062
:104B400023FC8AF8E2B0B9F1000F12D094F8E130FA
:104B50007D2B0ED12B7803F0040303F0FF0A13B171
:104B600010F03AFA05E00B200AF00EFC254B83F812
:104B7000E2A02B7803F0040303F0FF01002B60D1C7
:104B800094F8E1301F4A572B10D14FF47A73A2F8F2
:104B9000E43033681A0601D503F06EF91A4B1B682E
:104BA0005B074ED5194B0A221A804AE0306840074D
:104BB0002ED55A2B2CD192F8E6302BB1012382F856
:104BC000E61082F8E7303CE092F8E83083F0010329
:104BD00082F8E8300BB10C2000E00D200AF0D4FB85
:104BE0002FE000BF842F00201C150020882F0020FC
:104BF000982F00206C2F0020C830002004000020D7
:104C000018150020DC0D00208C170020D239002060
:104C10005D2B00F0CB845B2B00F0CA845E2B00F090
:104C2000C984562B01D106F06BF898F80230002B9E
:104C300000F0908494F8E1306F2B40F0858410F000
:104C400017F833685B0736D594F8E830B249B34AB1
:104C50008BB12B7858070ED5019BB7F906005B8AFC
:104C6000984208DD136813F0010302BF3220A1F857
:104C7000EC0081F8E8301368DA030DD594F8EE20E3
:104C8000A54B2AB993F8E62012B93222A3F8EC20FA
:104C9000012384F8EE300EE094F8E6309E4A53B1DA
:104CA0002B7803F0040303F0FF0123B9012382F8FA
:104CB000E61082F8E7309A4B4FF000091B689F1C02
:104CC00003F152083A787B7817F8010C9A4209D21E
:104CD00039460AF07FFA28B117F8022C01239340D5
:104CE00049EA030904374745ECD18C4BC3F80090DF
:104CF0008C4B1B785BB1894BDFF844B21A6898463D
:104D000012F0020FDFF83C9240F00082F8E1864B8F
:104D10001F6807F148087A78BB7838789A4228D219
:104D2000791C0AF057FA20B378790C2202FB004272
:104D3000D2F8F830BB421CD0C2F8F870397902F1D1
:104D4000F00382F8F01000215960FA785A70FA786E
:104D50000C2A4FF0010204BF9A700322DA7094F813
:104D6000202118BF99700123834022EA030384F8AD
:104D7000203106374745CED16C4B6D4FD3F800A09C
:104D80006C4B4FF000091B68029394F82830039392
:104D900097F80080B8F1000F00F0A981D7F8033030
:104DA000029AD31A002B0CDB02F5FA73C7F8033012
:104DB00094F82021012303FA09F322EA030384F87B
:104DC0002031039B002B00F0928117F8012C7B7897
:104DD0000432D2B2002B40F04681574B33F91220F7
:104DE000019B1B8A03F1C8018A4202DD97F802B0D9
:104DF00016E0C83B9A4204DA97F802C0CCF1000BE7
:104E00000EE094F82021012303FA09F322EA0303B8
:104E100084F82031029B03F5FA73C7F8033066E18A
:104E200094F8203143FA09F3DB0700F16081BBF10C
:104E3000000FCCBF022001200AF0C8FA08F1FF33AE
:104E4000252B00F24C81DFE813F026002B00350003
:104E50003F00500056007F009000A100A600AB006C
:104E60004A013F004A0056007F00900062008B001C
:104E70009C00BF00C400C900FB0000010501F60052
:104E8000CE00D300D800DD00E200E700EC00F10026
:104E9000B000B500BA00504601215A46FA2304E09A
:104EA0005A460AF10100022164230FF075FA0AF054
:104EB00073F914E10AF1030003215A4664230FF049
:104EC0006BFA0AF005F90AE10AF105000D215A46CC
:104ED00064230FF061FAB8F10D0F00F000810AF1C0
:104EE00004000E215A466423BAE00AF106000521A7
:104EF0005A46FF23B4E0114B0F2118685A4601307F
:104F0000C8230FF049FAB8F10F0F00F0E8800B4BFF
:104F100012211868A2E000BFDC0D0020842F0020C1
:104F2000F4220020DC3A0020F81F0020F03000209E
:104F3000CD0E00201815002000340020802700200E
:104F40008C170020622F0020B04B102118685A46A1
:104F50000B30C8230FF020FAB8F1100F00F0BF801B
:104F6000AA4B132118680A3078E0A84B1121186861
:104F70005A461530C8230FF00FFAB8F1110F00F0A0
:104F8000AE80A24B14211868143067E09F4B0921B2
:104F90001868023062E09D4B0A2118680C305DE011
:104FA0009A4B0B211868163058E0984B242118684A
:104FB000073053E0954B2521186811304EE0934B94
:104FC000262118681B3049E0904B152118680330E2
:104FD00044E08E4B162118680D303FE08B4B1721B3
:104FE000186817303AE0894B1C211868043035E006
:104FF000864B1D2118680E3030E0844B1E21186846
:1050000005302BE0814B1F2118680F3026E07F4BC5
:1050100020211868193021E07C4B212118680630C6
:105020001CE07A4B22211868103017E0774B2321BF
:1050300018681A3012E0754B1B21186808300DE013
:10504000724B18211868093008E0704B1921186854
:10505000133003E06D4B1A2118681D305A46C823DF
:105060000FF09AF93BE0012B39D1694BB87833F94D
:105070001230B3F5617F05DB40F633029342A8BFDF
:10508000134601E04FF46173B8F10C0F27D14FF4D0
:10509000966292FBF0F0A3F5617393FBF0F35D4928
:1050A0005FFA83FB0A785A4519D0BBF1030F34BF6E
:1050B0005A4600220A70584908FB021257490A60F2
:1050C0000AF06AF80AF04EF80AF002F8404659462B
:1050D0000AF0B5F80BF10100C0B20AF077F994F8C4
:1050E0002021012303FA09F3134384F8203109F145
:1050F0000109B9F1040F07F10C077FF449AEFAE595
:105100003368DF0512D5464BDB787BB1DBF8003026
:1051100098070BD5B9F8007017F001070BD1414B78
:1051200001201F605F6005F029FB05E0012005F00C
:1051300015FB012700E00027D8F80030590710D5EB
:105140007FB1012005F00AFBB9F8003003F002033B
:105150009BB24BB9334A02201360536005F00EFB3B
:1051600002E0022005F0FAFADFF8C0A0B9F800303A
:10517000DAF80820BAF80C1013F0030F14BF5161CD
:105180001161DBF8002012F00A0F30D0D8F80020AF
:10519000D2060DD55F070ED4042005F0EFFA224B9E
:1051A0000A22B3F9043093FBF2F3A4F8223102E0AF
:1051B000042005F0D3FAD8F80030980607D5B9F8DE
:1051C0000030590606D4402005F0D8FA02E040200D
:1051D00005F0C4FAD8F800305A0641BF124B0A2233
:1051E000B3F9043093FBF2F348BFA4F82431DBF8A1
:1051F00000309B061CD4D8F800301F0540F1B08069
:105200004FF4807005F0BAFAAEE000BF80270020AE
:1052100000340020D8130020F4300020F0300020AB
:105220001C150020982F00205C2F00204415002022
:10523000B14B1B78980756D5B04B1B78042B52D92D
:10524000D8F8003013F400730FD0B9F80030D90645
:105250003DD4102005F092FA202005F07FFAA848EE
:10526000011D02F073FD02232DE0B9F8007007F074
:105270001007BFB23FB11020019305F06FFA019BF8
:10528000012784F82631D8F800305A0513D5D4F810
:1052900028219C485189B0F900209B4B002AB8BFB7
:1052A00052428A4207DAB0F90220002AB8BF5242BD
:1052B0008A42C0F2B081B9F800309B0608D52020A0
:1052C00005F04CFA002384F82631012700E000277E
:1052D00094F83431BBB90E200AF056F88A4B0122FB
:1052E00083F834210FE0B9F8003003F03003002BCD
:1052F00081D0102005F032FA202005F02FFA00238B
:1053000084F8263102E0002F3FF475AF00221746E3
:105310007E4B002023F817007D4B191D03F10A0E68
:1053200021F81700002142F80E109644CEF8040030
:10533000CEF8081023F8170003F1320E5A3342F862
:105340000E10D15096441344CEF80400CEF8081045
:10535000586099601432002F7FF44DAF0127D7E7D2
:105360004FF4807005F0FAF96A4B1B78082B01D0D6
:105370000E2B02D1402005F0F1F933685E051AD5F5
:1053800094F8B8311BB92B7813F0040F03E0D8F868
:10539000003013F4002F0AD05F4B00221A704FF434
:1053A0009E700EF0C9FF30B103F0C2FBF7E70FF0BB
:1053B00057FB03F0DDFB2B78580705D5DAF80030F2
:1053C000BAF804205A6138E0D8F8002094F8D800E0
:1053D000D1075EBF514A43F00103137010F0AEFED7
:1053E0004F4910F0FFFE08F081F94E4B0146186A54
:1053F00011F0B4F818B92B7823F001032B700FF0DB
:105400001FFE494B18B9494A1288632A06D902225D
:105410001A702B7823F001032B7005E02A78D2074D
:1054200056BF022218701A7009F04AFF404B1B68E1
:10543000C01A002801DB03F053FB012384F8BA31C2
:1054400094F8BB31304E23B3DBF800305F0720D532
:10545000D8F800301D0703D4082005F07FF918E0C4
:10546000B9F8005005F00805ADB295B9082005F06F
:1054700085F9304B1A68304B1A60304BDB88A6F840
:10548000BC31204BDB88A6F8BE312D4B1D602D4B67
:105490001D6094F8BB311C4D002B00F0D880DBF868
:1054A0000030D80640F1D380D8F80030990206D4F5
:1054B0004FF4007009B0BDE8F04F05F04FB9B9F8EE
:1054C000004004F40074A4B2002C40F0C0804FF4FB
:1054D000007005F053F9174B1A68174B1A60174BF9
:1054E000DB88A5F8BC31074BDB88A5F8BE31144B2F
:1054F0001C60144B1C60AAE0882F0020F80F0020CD
:10550000B0100020642F0020DC0D0020D4390020D2
:10551000120F00205031002098360020DB3A002086
:1055200035FA8E3C2426002040150020F815002076
:105530005C150020A81000207C27002000340020EB
:105540008427002088270020B9F1000F02D07E2B8D
:105550003FF475AB94F8E130972B06D13D4B4FF4F7
:10556000C872A3F8EA20FFF76CBBA72B06D13A4A12
:10557000137843F004031370FFF763BB0022BB2BC7
:10558000079201D1022303E0B72B04D14FF6FE733B
:10559000ADF81E301BE0BE2B01D1022303E0BD2B72
:1055A00028D14FF6FE73ADF81C3010E0012002E068
:1055B000022000E003205FFA80F808F1FF30C0B25B
:1055C00005F090FB404609F001FFFFF73ABB234B83
:1055D000BDF81C101B681A880A441A80BDF81E10FA
:1055E0005A880A445A8005F08BFB002384F8E23085
:1055F000FFF727BB792B04D1194AD37823F0010395
:1056000006E07A2B7FF41DAB154AD37843F00103F3
:10561000D370FFF716BBB9F8002092063FF558AEDD
:105620002020019305F0AAF80E4A019B11685268E8
:10563000C3F82C1103F5967003F59871C3F8302167
:1056400002F084FB019B012783F8267140E609B034
:10565000BDE8F08FDC0D0020882F00201016002000
:105660003C310020FC0F00202DE9F04F89B00FF0F5
:10567000F7F9B84B1E78002E41F03E81B64D2B68ED
:10568000580541F13981B54CDFF804832368DF8880
:105690002379002B00F0D681D8F80020A368D31A14
:1056A0007C2B40F2CF81237BA2600133237306F170
:1056B0002400DFF8A892C0B20FF086F909F10E03BA
:1056C00033F916004FF47A735843A54B01361B8902
:1056D00090FBF3F000B20FF065F9032EE7D1302014
:1056E0000FF072F9B9F914000FF05CF90FF064F9DA
:1056F00099F80C30990732D141F28833D9F8082053
:105700009A4219D910200FF05FF9D9F818006426D1
:1057100090FBF6F000B20FF045F921200FF054F99C
:10572000D9F8180090FBF6F306FB13000028B8BF69
:10573000404200B20FF036F914200FF045F9894BC2
:10574000B3F904000A2390FBF3F00FF02BF91C20AF
:105750000FF03AF900200FF025F90FF02DF9237B17
:105760005A0740F04A8102200FF02EF97B4B4FF090
:105770000509D8696423323090FBF3F000B20FF0D2
:1057800011F9794B0320B3F906600FF01DF996FB70
:10579000F9F6764BB6B21B785B070AD538460EF0A1
:1057A00025FD20B92B6813F0100F18BF002630B26A
:1057B00004E06F4B9889B0FBF9F000B20FF0F2F8FB
:1057C0002B689F0765D5DFF8CCA16A4E9AF80030A8
:1057D00032884FF0640909FB02325B00B2FBF3F33D
:1057E000278C06203F01BFB247EA0327BFB2C3F3AD
:1057F00003231F430FF0E8F838B20FF0D3F8238CDF
:105800009AF8001001339BB293FBF1F201FB1233C3
:10581000238494F82E30012B05D139200FF0D4F8D1
:10582000B6F9000019E036886E235E43152796FB13
:10583000F7F63A20B7B20FF0C7F8B7FBF9F630B277
:1058400009FB16760FF0AEF83B200FF0BDF8B0B2B2
:10585000461D0A2096FBF0F000B20FF0A3F82820B6
:105860000FF0B2F8236B0A2093FBF0F000B20FF0B8
:1058700099F804200FF0A8F83D4B9B8913B103F071
:1058800055F803E03C4B186880F3100000B20FF0AD
:1058900089F83A4B1B689E0640F1A580384F3B784B
:1058A00098071BD511200FF08FF8A08E4FF4F366E8
:1058B0007043344B90FBF3F000B20FF073F81920F3
:1058C0000FF082F8A08E4643642096FBF0F696FB1C
:1058D000F0F300FB136000B20FF064F83B78E68E43
:1058E00013F0020F08BF002601200FF06DF830B250
:1058F0000FF058F809200FF067F800200FF052F869
:10590000214B94F838601A88B2F5967F0AD9134B68
:105910001B7B03F00F03072B04D842F20F7696424D
:1059200028BF164605200FF04FF894F82D300BB91C
:1059300030B239E0A6F1200010F000FC134910F05D
:1059400005FD0021064610F0EBFD28BB4FF07C5111
:1059500024E000BFDC3A002070360020C00F002099
:10596000C81600205C2F0020642F0020DB3A0020A6
:1059700098140020AC140020A81400208C170020DC
:10598000882F0020A0860100080000206666E63F00
:1059900018150020610000204FF03F41304610F004
:1059A00019FB10F0E5FD00B20EF0FCFF3B78990703
:1059B00004D494F83930BE4E012B04D1012384F86D
:1059C0003930BC4815E0BC49706A10F00BFC10F08F
:1059D000CFFDB9490090B06A10F004FC10F0C8FD8A
:1059E0000190684605E0B54A92E803008DE803009F
:1059F00068460EF0F9FF0EF0DFFF237B282B21D144
:105A0000AB4B0022D8F800001A734FF47A73B0FB46
:105A1000F3F74FF03C0917200EF0D6FFB7FBF9F66D
:105A2000B6FBF9F009FB1060000200B20EF0BAFFFD
:105A300018200EF0C9FF09FB167000B20EF0B2FF7D
:105A40000EF0BAFF94F84430994E002B00F05F81BD
:105A500009F036FCB36C9A4AC31A9342074640F2E7
:105A6000C180002386F84E3086F85030954B96F86A
:105A70007C101B88DAB21B0A86F86A2086F86B3025
:105A800086F8602086F86130B26FD8F800309A1A34
:105A90004FF47A734B439A420DD38B4B1B68B36719
:105AA0008A4B1B78013B012B9FBF102386F84E3099
:105AB000022386F85030226B0A21854B92FBF1F2CB
:105AC0001B6884F8682093FBF1F3121284F86920B4
:105AD000804A84F86C3012781B1284F86D3094F888
:105AE00038309207724884F8973003D42D2380F819
:105AF000983075E0D4F83CA0774ADFF8E8919AFB3B
:105B0000F2FB09FB0BA14FF00608042B08FB01F187
:105B10008CBF3323322380F89830704B0BEB8B0B08
:105B200091FBF3F60BEB8B0B4FFA86FE03FB161182
:105B30000EEB8B06206CB6B284F88760360A84F8C8
:105B4000886090FBF2F609FB060908FB09F898FB50
:105B5000F3F24FF0640C91FBFCF103FB128393FB17
:105B6000FCF384F88910091284F88A1051B206EB0C
:105B7000860202EB820201EB820292B284F88C2050
:105B8000120A84F88D2084F88E30A28E1B1284F8BD
:105B90008F30242353434FF47A7293FBF2F384F84B
:105BA0008430C3F3072384F88530B4F8AA304FEA71
:105BB000DA7A84F890301B0A84F89130E38EC00FB3
:105BC00003F5FA739BB284F892301B0A84F8933081
:105BD000B4F8AC3084F886A084F88B0084F899304F
:105BE000334B9F64324C94F8AE80B8F1000F0DD166
:105BF000D4F8B40009F0D8FC012807D90228384E9F
:105C000000F030860EF0C0FE0123B370D4F8B86007
:105C1000274B002E7BD093F8AE203AB140F6B73137
:105C2000D3F8C020BA1A8A4216D870E0012283F84D
:105C3000AE20D3F8C420D3F8B4001278022A04D8D6
:105C4000043002210EF08AFE02E0022109F046FC37
:105C5000002384F8C83058E093F8BC20AAB9C3F8F0
:105C6000B82083F8AE20D3F8C420D3F8B40012785B
:105C7000022A04D8043001210EF070FE02E0012156
:105C800009F02CFC0EF080FE3FE0013AD2B283F81E
:105C9000BC2093F8C81093F8C9002ABB01304A1CF5
:105CA00083F8C90083F8C820D3F8B4002BE000BF04
:105CB000C00F0020FC0F00208096184B38A401086C
:105CC0003F0D0300AC14002018150020FA15002029
:105CD000A8140020882F00208096980040420F00D2
:105CE00008000020806967FF324612F801EB01309E
:105CF0000EEB0106714683F8C900D3F8B40083F8AF
:105D0000C860C3F8B82009F075FCC4F8C070B34C83
:105D1000B34E94F8CA303768002B00F0B781D4F83E
:105D2000CC30002B00F0B28194F8D030013B012B35
:105D300000F2AC81D4F8CC00DFF8A08209F034FC8A
:105D4000E0B1D8F8CC0009F02CFC98F8D1308146AD
:105D50007E2BD6F800A00ED102231B2888F8D03065
:105D600009D1D8F8CC0009F01FFC20B90123C8F8EC
:105D7000D4A088F8D83084F8D190DBE7D8F8D420C4
:105D800033689B1A41F65832934220D9032388F88E
:105D9000D0307BE1934A32F8130010B903464FF438
:105DA00003600133B0F5C06FDBB27DD020D9B0F510
:105DB000006F00F0878033D9B0F5036F40D184F8CD
:105DC000D930894BDFF814821B6899063FD494F8C8
:105DD000D81094F8D930002900F056813268D21BCF
:105DE000012AD7D984F8D930002384F8D8304DE17E
:105DF000B0F5007F40D007D8B0F5807F49D0B0F52E
:105E0000887F00F09080E6E7B0F5806F00F0AC800E
:105E1000B0F5826F00F0F680B0F5047FDBD121E0B1
:105E2000B0F5E26F00F09380B0F5E46F00F094807D
:105E3000B0F5E06FCFD184F8D930B4F90E108FE00F
:105E4000B0F5046F7BD0B0F5026FC4D104E1674BAD
:105E50001B789A07BBD5B8F8341024234B43642130
:105E6000123313E084F8D9302B689B07AFD5604B11
:105E70000A211B8859431EE084F8D9302B68DFF8CB
:105E80005C811905A3D5D8F830300A2193FBF1F1D4
:105E9000F4E084F8D930544BDFF840811B685A078E
:105EA00095D5D8F81810E9E084F8D9302B681B058F
:105EB0008DD5504B19680EF01DFD484B002283F81C
:105EC000D82084E74849454A096884F8D9308906CA
:105ED0007FF57DAF4549097888077FF578AFD90709
:105EE00010D5136C192283EAE371A1EBE37101EB86
:105EF0005101B1FBF2F1002BACBF41F0004141F088
:105F000040410DE0D36B192283EAE371A1EBE37109
:105F100001EB5101B1FBF2F1002BB8BF41F0804120
:105F20004FF4006087E084F8D9302F4BDFF8AC8065
:105F30001B685A077FF54BAFD8F814109EE084F821
:105F4000D9302D4B0A21B3F90430594373E084F85A
:105F5000D930B4F9101003E0B4F9121084F8D93034
:105F60002C2391FBF3F166E084F8D930234B42F205
:105F700011711A7842F2107312F0010F08BF19461E
:105F800093071F4B48BF02311B88500748BF04319D
:105F9000DA0748BF0A31980748BF14311A0648BFCC
:105FA0002831D80548BF28315A0748BF643118073F
:105FB00048BFC8319A0548BF01F5C871980648BF67
:105FC00001F57A71DA0648BF01F5FA61580648BF53
:105FD00001F57A614FF480602DE000BFC00F002012
:105FE00018150020C4C701088C170020882F002036
:105FF000AC140020A81400205C2F0020DB3A002005
:10600000622F002084F8D930B74B1B6813F02008AA
:1060100017D0B64B1A7812F0020F14BF4FF47A71F2
:10602000002112F0010F14BF4FF4FA6300230B4458
:1060300094F8381019440EF05DFC002384F8D83031
:10604000C5E62B6819067FF5C2AE41460EF052FC3C
:10605000A74B83F8D880BAE684F8D930A24BDFF892
:1060600090821B689A067FF5B2AEA04B1B789B0707
:106070007FF5ADAEB8F83630642159430EF03AFCE6
:10608000002388F8D830A2E684F8D93094F8DA30C2
:10609000DFF85C92002B00F0E180D9F8DC30002BB7
:1060A00000F0DC80D6F80080D9F8E030C3EB0803BC
:1060B000632B40F2D380DFF850A241200EF000FCA9
:1060C000BAF902000A2790FBF7F080B20EF0EFFB5E
:1060D000BAF9000090FBF7F080B20EF0E8FBBAF9D5
:1060E000040090FBF7F080B20EF0E1FB0EF0B0FB85
:1060F00099F8E47017F0010738D07B4B1A689B467B
:1061000012F0200F7FD0794B1B78990708D599F8AA
:106110003830052B34BF4FF002094FF0030901E07E
:106120004FF0010947200EF0CBFBE06B0EF0AEFB09
:10613000206C0EF0ABFBA08E6427B0FBF7F0C0B272
:106140000EF092FBDBF80030DFF8A4A113F0140F7F
:106150000ABFBAF83600DAF8E80078430EF096FB8A
:1061600094F8380049EA8000C0B248E0614B1B88CF
:10617000DA0518D4D8060DD499060DD45A060DD4D4
:1061800018070DD4D9070DD413F0020F14BF03273D
:10619000012708E00D2706E0092704E0042702E0B4
:1061A000082700E00227544B93F80090534BC9F3A3
:1061B0008009DB781BB149F002095FFA89F95320A5
:1061C0000EF07EFB4E4B188800EB800000EB800049
:1061D000800080B20EF06BFB00200EF068FBB4F87C
:1061E000EC00FE23584340F2FF3390FBF3F0C0B2C3
:1061F0000EF03AFB00200EF037FB49EA87000EF064
:1062000033FB0EF025FB94F8E470DFF8E490C7B997
:106210004F200EF055FBD9F8F0000EF037FBD9F8FF
:10622000F4000EF033FB38460EF030FB01200EF088
:106230001BFB2E4B187800F001000EF015FB0EF042
:1062400007FB94F8E4300A210133DBB2B3FBF1F22F
:1062500001FB1233C4F8E08084F8E43094F8F8309D
:10626000002B00F04983274B1B68002B00F0448370
:1062700009F026F844F61F621D4B0746D3F8FC30A0
:10628000C31A934240F2388302200EF0B7FA002876
:1062900078D049F60742144B48F603491B682D682D
:1062A00013F0080F18BF91465A0744BF49F400592C
:1062B00049F008099B0644BF49F4804949F0200988
:1062C00015F00205C9F3090820D00D4BB4F830A031
:1062D0001D8802F04FFB05EB850505EB8505AD003C
:1062E000ADB2C0B215E000BF8C170020882F00208F
:1062F000C00F0020622F0020DB3A00201C15002078
:10630000AC140020243400205C2F00204FF6FF7ACC
:1063100064206A460023ADF80C30ADF81230ADF8B9
:106320001430ADF81630ADF81830ADF81A30ADF8BD
:106330001C30564BCDF80090CDF80490CDF8088075
:10634000ADF80E50ADF810A08DF81E000DF1180E2E
:10635000154603CD7545186059602A4603F10803B8
:10636000F6D128681860A988AA7999809A71484B53
:1063700001227C211F20DA710DF0E0FE0DF0C6FE37
:106380000DF0B2FE03200EF039FA002863D0414B25
:10639000D6F800A01B78002B00F0A2823E4A012B09
:1063A000B2F800E040F29D82022B508800F09A8201
:1063B000032BB2F804C000F09782042BB2F80680D9
:1063C00000F09482052BB2F8089000F09182062B21
:1063D000558900F08E82072B918914BFD289002243
:1063E00040F2FF3BB4F8EC30ADF81220C3EB0323CE
:1063F00093FBFBF300228DF814206A468DF81530CC
:10640000224BADF804E0CDF800A0ADF80600ADF8E1
:1064100008C0ADF80A80ADF80C90ADF80E50ADF89C
:1064200010100DF1100E154603CD7545186059601A
:106430002A4603F10803F6D12868F4211860AA88D7
:1064400016209A80124B2322DA710DF077FE0DF0A0
:106450005DFE0DF049FE06200EF0D0F9002800F098
:10646000CE800E4B1A68994612F0200F00F0C780BC
:106470000B4B1B78980715D594F83830052B34BF93
:106480004FF002084FF003080EE000BF3735002040
:106490002F35002094360020003400208C17002077
:1064A000882F00204FF0010808F00AFF226CE38ECD
:1064B00003924FF6FF724FF47A755D43B4F80031E2
:1064C000049503EB83035B00ADF81A30C34BADF8C2
:1064D0001420ADF816208DF81C806A466D4698464B
:1064E000E16BB4F834E094F838C0009000200190DB
:1064F0000291ADF818E08DF81DC00DF1180A96460E
:10650000BEE80300D64518605960724603F10803DF
:10651000F5D1DEF80000DFF8D8B21860BEF804202C
:1065200018219A801E208BF807100DF007FE0DF041
:10653000EDFD0DF0D9FD08F0C3FE8646E38E4FF465
:106540007A725343D9F80020D94612F0140F1EBFB7
:10655000A34A4FF00A0CD2F8E8204FF00A0B18BFFC
:106560000CFB02FC9F4A08BF9C46B2F90420CDF800
:1065700000E092FBFBF2AE46E06B216C039300233C
:10658000ADF81430ADF81630ADF81830934B0190DB
:106590000291CDF810C0ADF81A20724603CA5245D8
:1065A00018605960964603F10803F6D11068682117
:1065B000186021231C2089F807300DF0BFFD0DF075
:1065C000A5FD0DF091FDD4F8F020D4F8F4308DE85D
:1065D0000C00002302932B4603CBC9F8080018686F
:1065E000C8F8041031232721C8F808000C2089F8C6
:1065F00007300DF0A3FD0DF089FD0DF075FD0A20AB
:106600000EF0FCF8002846D0764DD6F80090B5F98B
:1066100000000FF093FD74490FF098FE73490FF0DE
:10662000E1FD8046B5F9020040420FF087FD6E495A
:106630000FF08CFE6D490FF0D5FD0646B5F904004C
:106640000FF07CFD68490FF081FE68490FF0CAFD2C
:106650006D460023049305930693604B0296CDF894
:106660000090CDF80480039006AE2A4603CAB242D9
:1066700018605960154603F10803F6D11068272108
:1066800018605B4B1E221C20DA710DF057FD0DF0D7
:106690003DFD0DF029FD0B200EF0B0F8002800F0B4
:1066A000DE80544B0025D3F8008018F020090AD072
:1066B000A08E0FF0C1F900224F4B0FF04DFB0FF0F1
:1066C00033FC064600E02E4618F0140F0AD0D4F82A
:1066D000E8000FF0B1F90022474B0FF03DFB0FF03F
:1066E00023FC07E0B9F1000F03D0E08E0FF022FD8C
:1066F00000E000203B4B0A22B3F9043093FBF2F296
:106700003E4B92B2B3F90630B3F57A7F05DBB3F5B1
:10671000FA6FA8BF4FF4FA6301E04FF47A73ADF853
:106720001020A3F57A73642253434FF47A7293FBDB
:10673000F2F3ADF81230294B6A46E8469A460196C4
:1067400000950290039504AE154603CDB54218603E
:1067500059602A4603F10803F6D12868244E1860D0
:10676000142001464A23F3710DF0E8FC0DF0CEFC35
:106770000DF0BAFC224BB1461D78224B05F0040502
:1067800005F0FF02002D0CBF4025C0251B78013B02
:10679000DBB2102B97BF1C494FF0000B5B1893F82E
:1067A00008B01A4B1B8899071ABF002645F0100540
:1067B000012613F4027F18BF022613F0100F18BF32
:1067C000062613F0200F18BF10261AB3104BDB78E3
:1067D000002B14BF0522042222E000BF3735002021
:1067E000C00F00205C2F00200000204135FA8E3CB5
:1067F0002F3500208C170020000059400034002065
:10680000DB3A00205031002038A40108622F00201C
:106810001C1500200EF014FC002814BF02220322D5
:1068200000238DF8072003228DF805308DF808200D
:1068300000968DF804B08DF80650B8E803008AF889
:106840000820CAF80000CAF804100920322189F88B
:1068500007300DF073FC0DF059FC0DF045FCC4F849
:10686000FC7049E0B3782BB1C4F8B07086F80280B0
:10687000FFF7CCB9D4F8B030FB1AB3F57A6FFFF458
:10688000C5A90123D4F8B400B37008F08AFE064607
:10689000D4F8B40008F085FE76067FF4B7A98A28FC
:1068A00003D08E280ED0FFF7B1B9154B1B689806A0
:1068B0007FF5ACA994F8AE30002B7FF4A7A904F1C2
:1068C0007D0306E094F8AE30002B7FF49FA904F11D
:1068D0004C03C4F8B8302D2384F8BC30FFF796B9C8
:1068E0009E4600204FF0000C4FF000084FF00009CA
:1068F000002500210A4673E509B0BDE8F08F00BF0E
:106900008C1700202DE9F04F87B06C4C02916C4938
:1069100022880E680546C2EB26135B435200C2EB89
:10692000E602B4F902601B135643B4F90420B4F92B
:106930000A0053439B1303EBE62606EB86038033E2
:106940001B12B6F5FA384FEAE67704934B6847F125
:10695000FF39A8FB08AB039308FB09F3B4F908203F
:106960000BEB430BE389A6610593D31708FB03F1F7
:1069700002FB0911A8FB02230B44C1171F030AFBEA
:1069800001F300FB0B33AAFB00011603194447EA8D
:106990001257020A42EA016292194FEA2123E6885D
:1069A0007B410032A2FB060143F5004306FB0311C5
:1069B0004B100093CB170193DDE900231343B4F888
:1069C00010E0B4F80CC06DD00FFA8EF0C1170AFBBE
:1069D00001F1AAFB002300FB0B11BDF914600B446D
:1069E000F71708FB07F106FB0911A8FB06670F4420
:1069F00079047004801841EAD6315941039B0FFA9B
:106A00008CF8C3F5801E7246D317002212184FEA85
:106A1000CE764FEAC3774FEAC8034B4147EA5E0799
:106A2000B61A67EB030740F63543A6FB030103FBE9
:106A30000711DDE900230FF0E1FDB4F916204E1334
:106A400002FB06FE470B47EAC147D31707FB03EEDD
:106A5000A2FB07235643734407FB0366A2FB0723ED
:106A60003344560E46EAC3168219B4F914604FEA4D
:106A7000636741EB07037143F71700FB0717A6FB9A
:106A800000013944C60C46EA413692194FEAE14703
:106A90004FEA1221B4F912207B4141EA036113014C
:106AA0000B4400E000230DB11B0A2B60029B13B1C5
:106AB0001A46049B136007B0BDE8F08F70170020E2
:106AC000DC100020704770476B4B6C4A2DE9F04F8B
:106AD0005E8994684FEA062AB4EB0A0A9C884FF054
:106AE00000054FEA04481C894FF0000BA4FB0A671D
:106AF00065EB0B0B04FB0B77F40944EA476418EBD6
:106B000004065C884FF000094FEAE7154FEAC438E5
:106B1000DC8849EB050787B0CDE90467A4FB0A6769
:106B200004FB0B77340A44EA076418EB04064FEAC7
:106B300027259C894FF0000949EB0507CDE900673F
:106B4000AAFB046704FB0B77F40D44EA472414F511
:106B5000FA664FEAE75545F10007B6F5FA6F77F1A7
:106B60000003CDE90267964666DADDE90489A4FBF5
:106B7000046704FB05F34FF0050C07EB4307A6FB86
:106B80000C230CFB07335F104FEA3206B8EB060804
:106B90004FEA920646EA837669EB07099F10DDE922
:106BA0000023921B63EB0703CDE90023DDE90267B5
:106BB000334A4FF0FF33964277EB0303CDE9048964
:106BC00027DA40F6AC520023A4185D4104FB05F31C
:106BD000A4FB04456FF0060205EB4305664202FB89
:106BE0000566A4FB0223334418EB020649EB0307B6
:106BF000CDE904670B26A4FB062306FB0533DDE97C
:106C000000455B104FEA3202A41A65EB0305CDE99B
:106C10000045DDE902450AFB0BF3AAFB0AAB0BEBCF
:106C2000430B4FEADA7242EA4B02A41A4FEAEB73C3
:106C300065EB0305CDE90245DEF80C40009B019DA4
:106C4000A4FB032304FB05334FEA525848EAC32848
:106C50004FEA6359DDE90423B8EB020269EB030351
:106C60009946D30B43EA494300B1036009B1029B43
:106C70000B6007B0BDE8F08F04170020DC10002087
:106C800024FAFFFF2DE9F041324C334D62892B8A03
:106C9000B4F904809A1A2389B4F902E05A43B4F98A
:106CA0001230D613B4F91420DB02324493FBF2F213
:106CB00032440A26E2615643A2F57A6202FB02F3ED
:106CC000B4F90EC002FB0EFE02FB08F2B4F90C8010
:106CD0001B130CFB03FC03FB08F31B1403EB6232D6
:106CE0000232E388921002F5004253434CF25032D4
:106CF000B4F920704FEAEE2EB4F900400EEBEC2C04
:106D00000CEB8404BC406D690234A5EBA4043A4149
:106D100062434FEAD3384EBFB2FBF8F35400B4FBE2
:106D2000F8F340F6DE3448BF5B001A125243624368
:106D30000A4C08365C43241404EB224202F6CF626C
:106D4000361103EB221300B1036001B10E60BDE800
:106D5000F08100BF18170020DC10002043E3FFFF84
:106D600013B50C4B04465B681B20022101AA98470F
:106D700070B19DF804209DF8053043EA022303F525
:106D80004E5310334FF48C7293FBF2F32333238072
:106D900002B010BDEC160020034B1A7E02F0FF007B
:106DA0000AB100221A767047DC10002037B5104B6C
:106DB00004465D68187806216A46A847A8B19DF880
:106DC00000209DF80130012043EA022323809DF832
:106DD00002209DF8033043EA022363809DF80420DB
:106DE0009DF8053043EA0223A38003B030BD00BF05
:106DF000EC16002013B5104B04465B683B200621BF
:106E00006A469847A8B19DF800209DF801300120FE
:106E100043EA022323809DF802209DF8033043EAD1
:106E2000022363809DF804209DF8053043EA022385
:106E3000A38002B010BD00BFEC160020054A08B5C3
:106E4000138801339BB21380034B187804F022FAA5
:106E5000002008BDFC150020F417002008B54FF4F1
:106E600080400EF06FFA012801BF044B4FF48042BE
:106E70005A61034B08BF587608BD00BF00040140AB
:106E8000DC10002010B5074C236818690EF05AFA80
:106E900030B123681A69044B5A61044B01221A76F7
:106EA00010BD00BFF816002000040140DC100020D7
:106EB000F8B50E461746084C4FF48055656140F012
:106EC00080000DF031F83846002132460CF0FEFF0C
:106ED00025610120F8BD00BF000C014070B50E46D1
:106EE000054C4FF4805565610DF01EF830460DF0ED
:106EF0001BF82561012070BD000C014070B5104CDD
:106F00000546192008F003FAA368152000219847C8
:106F100010B9022008F072FAA36845F01801162093
:106F20009847A368002117209847A36801213D20B6
:106F30009847A3683E200121BDE87040184700BF74
:106F4000EC160020F0B5274D85B0AB7E002B46D166
:106F5000254C2368002B42D01A68244E12B1B16927
:106F60000A43B2619A889868ADF8002002228DF831
:106F70000320694604228DF802200BF030FEB3692D
:106F8000002743F00103B36123680126187B197DB4
:106F90000BF010FE2368164993F9150008F07CFAEF
:106FA0002368144A1B695361029308230DEB030005
:106FB0008DF80D308DF80C708DF80E600EF092F992
:106FC000236801A85B7D8DF806708DF804300323DB
:106FD0008DF805308DF807600CF05AFFAE7605B0DD
:106FE000F0BD00BFDC100020F816002000100240A9
:106FF000856E00080004014070B505461B4CFFF784
:10700000A1FFA36880216B209847642008F07FF9D6
:10701000A368072168209847642008F078F9A368DE
:1070200000216B209847642008F071F9A3680121C2
:107030006B209847A36818211B209847A36810214C
:107040001C209847A36829461A209847084AA36835
:10705000117819209847A368102137209847A36812
:1070600038200121BDE87040184700BFEC16002011
:107070004606002010B50446FFF764FF4FF4805326
:10708000238110BD70B50546154CFFF75BFFA36863
:1070900080216B209847642008F039F9A368032108
:1070A0006B2098470F4AA3681178192098470F2042
:1070B00008F02DF9A36829461A209847A3681821DB
:1070C0001B209847A36810211C209847A368022121
:1070D00037209847A36838200121BDE87040184741
:1070E000EC1600204606002010B50446FFF72AFFE4
:1070F000064B5B7813B1012B03D010BD4FF4006336
:1071000001E04FF48053238110BD00BFE81600203A
:1071100010B54000204CC0B220702048204C0170B7
:10712000204800210170012020701F4C23601F4C5B
:1071300023601F4B1A701F4A1F4B107019701F4994
:10714000086811461A4630B383889C0515D4038815
:10715000DB050DD44FF480530488A40502D5013B10
:10716000FAD112E08BB103889BB243F480730380A1
:1071700083889BB243F4407383804FF48053087834
:1071800010B1013BFBD100E013B9BDE8104055E65A
:10719000107880F0010010BDFA170020F8170020C9
:1071A000F617002000180020FC170020041800200B
:1071B000F91700200818002009180020F0170020F7
:1071C00007B5F7216B4606227620FFF7A1FF9DF851
:1071D00000309DF801101B0343EA01139DF80210D3
:1071E000094A43EA111353609DF803309DF80410D7
:1071F0001B0343EA01139DF8051043EA11131360C2
:1072000003B05DF804FB00BFDC10002007B50021CF
:1072100001AB03227720FFF77BFF9DF805309DF837
:1072200004001B0243EA00439DF80600184303B024
:107230005DF804FB08B5FFF7E9FF014BD86008BD16
:10724000DC10002008B5FFF7E1FF014B986008BD96
:10725000DC1000200F4B13B51B780F4C0BB1637E75
:10726000B3B1032201AB7720F621FFF751FF9DF860
:1072700005309DF804201B0243EA02439DF80620D6
:107280001343064AB2F92020C2F10802D3406361D9
:1072900002B010BD0B000020DC10002018170020E9
:1072A0000A4B13B51B780A4C0BB1637E63B1022203
:1072B00001AB7720F621FFF72BFF9DF804209DF806
:1072C000053043EA0223238202B010BD0B000020E8
:1072D000DC10002030B505460C46134629462246F0
:1072E000BDE83040682013E713B5062204460121AB
:1072F0001C206B46FFF70CFF08B39DF801309DF88A
:107300000020042143EA022242F38D0292FBF1F2B3
:107310009DF8023022809DF8032042EA032242F3C6
:107320008D0292FBF1F29DF8043062809DF80520F9
:1073300042EA032343F38D0393FBF1F3A38002B0EE
:1073400010BD13B506220446022118206B46FFF734
:10735000DFFEB8B19DF800309DF801209B0803EBDB
:10736000022323809DF802309DF803209B0803EB45
:10737000022363809DF804309DF805209B0803EBF1
:107380000223A38002B010BD314B2DE9F3411B78DD
:107390000546002B3BD0002426462746A046013454
:1073A0005320322108226B46E4B2FFF7B1FE08B940
:1073B000002049E09DF801209DF80030202C03EBCF
:1073C00002231BB29DF8032098449DF8023003EB82
:1073D00002231BB21F449DF805209DF8043003EBE7
:1073E00002231BB21E449DF8073003F07F0301D037
:1073F000002BD4D198FBF4F897FBF4F796FBF4F646
:10740000144BA5F800806F80AE80DC761CE0532022
:10741000322106226B46FFF77BFE0028C8D09DF87C
:1074200001209DF8003003EB02232B809DF8032000
:107430009DF8023003EB02236B809DF805209DF838
:10744000043003EB0223AB8002B0BDE8F08100BF43
:10745000FE160020DC10002013B502AB03F8012D4E
:107460004000214AC0B21070204A0020117020490B
:1074700001220A701F4908701F490B601F490B60E9
:107480001F4B20491A700A701F4B204A1870106851
:107490001A4630B383889C0515D40388DB050DD4C8
:1074A0004FF480530488A40502D5013BFAD112E0C1
:1074B0008BB103889BB243F48073038083889BB2B3
:1074C00043F4407383804FF48053087810B1013B3C
:1074D000FBD100E013B9FFF7B1FC02E0107880F0B7
:1074E000010002B010BD00BFFA170020F8170020FD
:1074F00000180020F617002004180020FC170020B8
:10750000F91700200818002009180020F0170020A3
:107510007620F42131229FE77720482101229BE742
:1075200077205821012297E7064B002193F820206D
:10753000054B9201343259767720F42102F0FC0297
:107540008AE700BF18170020DC100020034B002240
:107550005A767720F4212E227EE700BFDC1000202F
:1075600003460A466820194676E737B505462A21BC
:1075700000221C20FFF770FF0E2102221C20FFF7C3
:107580006BFF0F2103221C20FFF766FF2B21122225
:107590001C20FFF761FF164A02249369154843F047
:1075A000040393612023ADF8043004230DEB0301A1
:1075B0008DF806308DF807400BF011FB22462C2188
:1075C0001C20FFF749FF2D2101221C20FFF744FF5B
:1075D0002E2100221C20FFF73FFF2A2105221C201C
:1075E000FFF73AFF4FF480732B8103B030BD00BF2B
:1075F000001002400008014010B504460F21082287
:107600001820FFF729FF182010210E22FFF724FF72
:107610004FF48053238110BD134B10B51B780446E3
:107620002D21532008227BB1FFF716FF31210A22BA
:107630005320FFF711FF2C210C225320FFF70CFFE2
:1076400053203821902209E0FFF706FF31210A225A
:107650005320FFF701FF53202C210A22FFF7FCFEE5
:107660004FF48073238110BDFE16002003F01ABF73
:1076700004F03EB803F016BF04F03AB8034B13F819
:10768000012D5A70024A9342F9D1704760060020DA
:107690004C06002001238370704710B50EF04EFD9C
:1076A000002104460EF05AFF08B1204601E004F123
:1076B000004005490EF04AFE04490EF093FD06F025
:1076C00015F8034B186010BD8096184B35FA8E3CA8
:1076D00030000020F8B5A14B0446187818B10128F5
:1076E00000F06281A0E2242C9D4D0CD006D80A2C1B
:1076F00000F0D9800D2C00F0D6801EE12A2C06D097
:107700002C2C04D019E128706870A87049E1954BC1
:1077100069782F780020924A58542FBB1978D77077
:10772000472921D1597850291ED19978472907D165
:10773000D978472904D11979412901D10121D17082
:107740009978884A522903D1D1784D2900F06E8268
:107750009978844A472907D1D178532904D11279DD
:10776000562A04BF0322EA70EA787D4E022A39D0F5
:10777000032A4CD0012A40F08580BA1E072A00F265
:107780008180DFE802F004080F131A257F2A0CF02D
:1077900003FC686076E01B78532B73D16B685B4207
:1077A0006B606FE00CF0F8FBA8606BE01B78572B68
:1077B00068D1AB685B42AB6064E01B78302B6A4BEE
:1077C0001A788CBF42F0020222F002021A7059E0CD
:1077D00000200CF041FC287354E000200CF03CFC2D
:1077E000E8814FE0072F06D0082F4BD101200CF085
:1077F00033FC708246E001200CF02EFC41F218436D
:1078000058434FF47A73B0FBF3F030823AE0022F22
:1078100007D0032F0AD100200CF01EFC534B187028
:1078200030E000200CF018FC30752BE02AD93A1F0C
:107830009210337D0132D2B2013B02EB8303DBB203
:10784000102B1FD8F91EC2F1010201EB8202D2B245
:10785000012A0BD0042A11D100205E1E0CF0FCFB83
:10786000434B00229855434B9A5507E0424A5E1E0F
:10787000002093550CF0F0FB404B9855404A13689C
:1078800001331360364B2A2C18BF9A7807F1010791
:107890004FF000000CBF012254402F7068700CBFE5
:1078A0005A759C707DE0687D002843D0FFF7E6FEA6
:1078B0002C4A2B4C13785278402B85BF373B1B0149
:1078C0001B01DBB298BF03F0F003402A8CBF373AAC
:1078D000303AD2B21344AA78DBB29A42294B26D16D
:1078E000294921221A70E0780A68012802F1010270
:1078F0000A600AD002281CD172221A70228A234BF5
:107900001A80628A224B1A8013E067221A70164B83
:107910001B789B070ED51F4B62681A60A2685A60DD
:10792000227B1D4B1A70E2891C4B1A8002E03F2219
:107930001A70002000236B7533E06B78687D0E2B86
:107940009FBF074A591C5170064A98BFD454044A35
:1079500030BB93785C40947023E000BFEC2700209C
:10796000F8100020F0330020882F002000040020B1
:107970003104002021040020010400201104002013
:10798000302400204C06002028240020F40F002082
:10799000C0100020FC0F0020F80F0020F60F002080
:1079A000002000F00100F8BDA44E0023B27D082A9B
:1079B00000F23A81DFE802F0050F141A2530557005
:1079C0007A00B52C02D1F375012307E09C4A1368B5
:1079D0000133136028E1622C08BF0223B37523E151
:1079E0000323B37534767476B4761DE10423B3753E
:1079F000737EB27E2344DBB273761344B376F4769F
:107A000012E10523B375737EB27E2344DBB2737635
:107A10001344B376B48307E10623B375737EB08B4A
:107A2000B27E2344DBB240EA04207376B0F5AC7F2B
:107A30001344824DB376B0830BD9FFF71FFE814B01
:107A40003E221A70804A00205368A87501335360A3
:107A5000F8BD0023EB83002840F0E6800723AB75D8
:107A6000F8BD737EB27E2344DBB273761344B376E3
:107A7000F38BB3F5AC7F3EBF704AD21882F820403A
:107A8000B28B013A934204BF6C4A072103F1010310
:107A900008BF9175F383C7E00823B375737EA342D3
:107AA00000F0C280654B0122DA7509E0B375FFF77B
:107AB000E5FDB37E614DA342624906D03F230B70C2
:107AC000614A536801335360AEE0604AE87D136851
:107AD0000133136010B13E230B70A5E021230B701E
:107AE000EB7E062B41D004D8022B07D0032B23D0EA
:107AF000F8BD122B59D0302B67D0F8BD50236A6ADD
:107B00000B70534B5A60AA6A1A602B6B4FF47A724F
:107B100093FBF2F34F4A138095F878214E4B1AB13C
:107B20001A7842F0020202E01A7822F002021A7079
:107B3000012386F8793169E053230B7095F82530DD
:107B4000DF0705D595F82430DC1E6342634100E071
:107B5000034603F0010286F87821002B56D13E4AF5
:107B6000137823F00203137050E04F230B7095F845
:107B70002B30D90705D595F82A30DA1E53425341E8
:107B800000E0034603F0010286F8782123B9324A67
:107B9000137823F00203137096F84F202F4B1A70BE
:107BA000B6F84C202E4B1A8030E056236A6B0B70CF
:107BB0002C4B1A8042F21072AB6B93FBF2F32A4A01
:107BC0001380012385F87A3120E095F82420492399
:107BD0000B70102A254B88BF10221A70244A19787E
:107BE00000238B420ED2157A224C1D55557A224C19
:107BF0001D55D57A214C1D5512F80C5F204C1D5592
:107C00000133EEE71F4A13680133136096F87921B8
:107C10000A4B92B193F87A217AB1002183F8791155
:107C200083F87A111046F8BD0020F8BD1279432A76
:107C30007FF48EAD0222EA708AE5F8BDF8100020CC
:107C40003C2400204C060020CC27002028240020C3
:107C5000FC0F0020F60F0020882F0020F80F0020D6
:107C600008000020F40F0020C010002000040020B5
:107C7000181100200104002011040020210400201C
:107C800031040020302400200449054B09680022FB
:107C900018705A6199611A77704700BF1815002053
:107CA000CC270020F8B5101A0D461F460EF046FAF4
:107CB0000446781B0EF042FA174B079E19680EF027
:107CC00091FA2146054620460EF08CFA29460746D1
:107CD00028460EF087FA014638460EF07BF911F07F
:107CE00093FC0E490EF07EFA0EF068FC069B2946C6
:107CF000186004F1004005F003FC09490EF072FA27
:107D000008490EF067F90EF033FC0028BCBF00F5FF
:107D10000C40A0303060F8BD300000202C7D8E3F3C
:107D2000A00CB34500A00C4644F25063984203DD1A
:107D3000A0F50C40A0387047034B9842BCBF00F53B
:107D40000C40A030704700BFB0B9FFFFF7B5036823
:107D5000174C184D23600B68174E63600068FFF7DF
:107D60009CFC95E80300154B0196009394E80C00E9
:107D7000FFF798FF3668124B60681E606B68114F02
:107D8000C01A0EF0DBF9104B19680EF02BFA0EF04A
:107D9000EFFB2A68236878609B1A3B600B4B1E60E0
:107DA0000B4B1B68DA880B4B1A8003B0F0BD00BF89
:107DB0000C290020FC0F0020182900201429002085
:107DC000542900201C290020300000204C290020CC
:107DD000040F00204829002070B5044600790EF0F9
:107DE000A9F91E490EF0B2FA1D4D1E4E2860A07B67
:107DF0000EF0A0F919490EF0A9FAEE6068606079FA
:107E00000EF098F918490EF0A1FA184D2860E07BA1
:107E10000EF090F911490EF099FA6860607E0EF04C
:107E200089F913490EF092FAEE60A860A0790EF07D
:107E300081F90D490EF08AFA0E4D2860207C0EF073
:107E400079F906490EF082FA6860A07E0EF072F9A8
:107E500007490EF07BFAEE60A86070BD0000C842D2
:107E6000242900200000FA44000020413429002089
:107E700000007A445829002010B50E4C23789B0747
:107E800017D50D4B1B78042B13D90C4A0C4B1068DB
:107E9000526818605A60FFF700FC0A4B0A22B3F9D7
:107EA000043093FBF2F3084A1380237843F0010374
:107EB000237010BD882F0020F80F0020FC0F002039
:107EC000B01000205C2F0020682900202DE9FF4120
:107ED000654B044633F9103064492BB902280CD0A5
:107EE000634B1B88980708D0624B002223F81420AC
:107EF000614B1B8821F81430B2E031F8143023B9FB
:107F00005E4A02EB8402C2F87C3101339BB221F855
:107F100014301BB2002B1CDD022C584A58480BD1E0
:107F2000B0F90800202590FBF5F5D2F8840100EBAC
:107F30004510C2F884010CE030F92400802590FB44
:107F4000F5F502EB8402D2F87C0100EBC510C2F813
:107F50007C014C4A1768BA7A934240F08180474AC4
:107F6000022C02EB8402D2F87C01424E90FBF3F328
:107F7000C2F87C314FF0000221F8142007EB040214
:107F800092F803E003BF5D42ADB214219DB218BF69
:107F90000A21BEF1000F61D0002D5FD036F8142009
:107FA000002A5BD028B20FFA82FC604556D080EAE6
:107FB000E0728CEAEC78A2EBE072A8EBEC78C8EB0C
:107FC0000202002812B209B22F4803DDBCF1000FF3
:107FD00003DC1DE0BCF1000F1ADA8A420CDD022C32
:107FE000BA7904D1818802F580720A440EE030F833
:107FF000141040320A4415E049428A4214DA022C35
:108000000DD1BA7902F140018288521A82800BE0C8
:10801000002AB8BF52428A4206DD022C04D030F852
:108020001420203A20F8142030F914203F5D9211DA
:10803000BA4203DB7245A8BF72461746134A12685C
:10804000120308D5142001A98DF804400293ADF85D
:108050000C7001F03DFA0E4B1B681F5526F81450AA
:1080600004B0BDE8F08100BF642F0020620B002047
:10807000622F00205C0B0020540B0020F810002021
:10808000782F0020500B0020560B00207036002067
:1080900080270020094A137818441346C0B210F014
:1080A000800F18BF80381070054A197813789942EC
:1080B00001BF00231370014A13707047451600205A
:1080C0004416002010B50A4B0A4A1B7842609C18DF
:1080D000094A046012789A4225BFD31A0B60C3F193
:1080E000800300232EBF4B600B604A6010BD00BFB1
:1080F0004516002046160020441600201FB568468D
:1081000002A9FFF7DFFF044B02981B6803440398A2
:10811000184405B05DF804FBB00900202DE9F04FCC
:1081200089B0019300238246994602910392039AF3
:10813000934205DA029A52F8232001339144F6E77C
:10814000019B4D46002B56D10AF0D2FE002852D199
:1081500001987DE00222404E8DF81C201A0C4FF44D
:1081600080578DF81D2006201A0A8DF81E208DF8E4
:108170001F300AF0E1FE776106200BF0D5FE374B89
:1081800001223761D0461A7077612646002007A980
:1081900004220BF09BFE029F4FF0000B039B9B45BC
:1081A0001EDABC4657F8042B4FEA8B03002A48D04E
:1081B000B24236D332465AF803100020CDF814C02C
:1081C00004930BF083FE049BDDF814C05AF80320DF
:1081D00032444AF80320DCF800309E1BCCF80060E3
:1081E0001D4B4FF480521A611D4A2D1B13681C440D
:1081F000019B146053B34DB3194B1B68DCB22A19B1
:10820000B2F5807F174A88BFC4F58074D26898BFE2
:108210002C4693429ED3144A00231370134A1370C2
:1082200014E00020D8F800100BF050FE57F8043C82
:10823000D8F80020F61A1344C8F80030002347F895
:10824000043C0BF1010B08F10408A7E7C5EB09009A
:1082500009B0BDE8F08F00BF000C0140AD0900205F
:10826000B00900201C000020441600204516002004
:1082700030B50B4C0B4D22782B7885B09A420CD040
:10828000684602A9FFF71EFF0123684602A90222E1
:10829000FFF744FF00232B70237005B030BD00BFF3
:1082A000451600204416002030B50E4D0E4C2A789D
:1082B000237885B09A4211D0684602A9FFF702FFE1
:1082C000002302A902226846FFF728FFFFF7E2FE1B
:1082D00020782B781B1A5842584100E0012005B045
:1082E00030BD00BF4516002044160020054A064B4D
:1082F00010781B7883422EBF181AC0F18000C01876
:10830000704700BF451600204416002038B50E4CBB
:108310004FF4805545F208200AF00EFE65610620F4
:108320000BF002FE094B01222561C7201A7065611E
:108330000BF0FAFD064A002325611370054A1370FD
:10834000054A136038BD00BF000C0140AD09002094
:108350004416002045160020B009002001480249BB
:1083600003F0B8BA00080040E8250020014802499F
:1083700003F0B0BA00040040C025002010B5044648
:108380000021102210F061FD0F232371054BA36023
:108390002823237363730123A37300232380638043
:1083A00010BD00BF0000A040014B33F82100704712
:1083B0008012002003788B4283BF034B03EB410103
:1083C000088D0020704700BF801200200022134655
:1083D00070B5264914180C4494F8404083EA0423ED
:1083E000082413F4004F4FEA430318BF83F481536A
:1083F00004F1FF3418BF83F0010314F0FF049BB2B3
:10840000EFD10132192AE4D100F1190200F11A0565
:108410000A440D4492F8406095F8402002EB062291
:1084200092B29A4221D1114B93F86150E2B2AA4222
:1084300018D2431C03EB4203DBB2CA1801330B44CE
:1084400092F8402093F8403003EB02239BB24FF4A4
:10845000AF625343064A1B1303F5487322F81430E6
:108460000134E3E7012381F8623070BD80120020FF
:10847000A812002003788B420BD9074B89001A7889
:10848000064B1944486E02B1400800F5777080B27F
:1084900070470020704700BF9736002080120020F0
:1084A00007299DBF034B03EB8101B1F89400002025
:1084B000704700BF80120020034B03EB4101B1F86D
:1084C000B400C008704700BF8012002008B5084BF8
:1084D00003EB8101D1F8D4000DF02CFE05490DF01D
:1084E00081FE05490DF076FD0EF068F880B208BDFA
:1084F000801200200000203F00005C44024B03EB90
:108500004101B1F81C01704780120020024B03EBBF
:108510004101B1F84001704780120020024B03EB8B
:108520004101B1F8400170478012002000207047DF
:1085300040F6CA03F0B5184F40F2EE25F98A40F232
:10854000ED2699420A46A8BF1A463F8AB142CCBFDF
:1085500011462946BB42A8BF3B46B742D8BF2B466F
:108560001924A1F2EE21A3F2EE2391FBF4F193FB87
:10857000F4F3C9B2DBB20022032A0CBF0D461D463C
:10858000CCBF0124002400F8124000EB4204013269
:10859000122A6570F0D1F0BD7436002000234FF42C
:1085A0007A72C252C21804334FF4FA61102B518010
:1085B000F5D170470388C3F30B03022B03D126299F
:1085C00008D101207047012B04D1A1F14B0358427F
:1085D00058417047002070470388C3F30B03022BF8
:1085E00003D1272908D101207047012B04D1A1F123
:1085F0004C0358425841704700207047B0F80D10A6
:10860000154B164A934206D21A88C2F30B028A42CD
:1086100003D01033F5E7002200E01A46037903F097
:108620003003102B10D0202B04D09BB9B0F80F30A2
:1086300050680DE00A4BB0F80F1093F858310C2039
:1086400000FB0310536803E09268B0F80F30106825
:10865000184470470020704798E4010878E7010843
:108660008012002010B5044606F02AFE40F6B8310C
:108670000E4BD3F85C21C3F85C01821A8A4284BF96
:10868000002283F8602193F860210AB9202C0CD1D4
:1086900013441F2A054983F8614103D1012381F85E
:1086A000813110BD013281F8602110BD801200209F
:1086B00070B5054606F004FE334CD4F88431C4F896
:1086C0008401C31AB3F5FA5FC4F8883182BF00236E
:1086D00084F88C3184F88D3194F88C312BB9A12D2C
:1086E00002BF294A012182F88D1194F88D11264A82
:1086F00031B1D118EDB2013381F8405082F88C319C
:1087000094F88C5194F88E31AB423CD11E4B93F8C7
:108710008F31052B02D0062B03D02FE00020FFF76E
:1087200055FE94F841301E2B28D100200246C1B2DC
:108730006B1E99421ADA214491F840300821DBB2CD
:1087400083EA0206F60744BF83F01803C3F3460327
:1087500001F1FF3154BF5B0843F0800311F0FF01CA
:10876000C2F34702ECD101301A46E0E7234493F804
:1087700040309A4202D10320FFF728FE002384F8FC
:108780008D3184F88C3170BD8012002010B5044604
:1087900006F096FD41F288310F4BD3F89021C3F8D3
:1087A0009001821A8A4284BF002283F8942193F8B0
:1087B0009431094A0F2B0DD8591CC9B21344102902
:1087C000E4B283F895410CBF0123002382F8941191
:1087D00082F8A53110BD00BF8012002010B50446FC
:1087E00006F06EFD41F288310E4BD3F8A821C3F894
:1087F000A801821A8A42C3F8AC2184BF002283F800
:10880000B02193F8B0210749142A134418BF01324C
:1088100083F8B14112BF81F8B021012381F8C6313C
:1088200010BD00BF8012002038B5044606F048FD98
:10883000274A2749D2F8C831C2F8C801C31AB3F58C
:108840007A6F84BF002382F8CC3192F8CC3133B9EF
:10885000A82C3BD181F8CD31A1F8CE3106E0022B16
:1088600002D181F8D04101E0242B02D8D11881F83F
:10887000D14192F8D01101330231DBB249008B4271
:10888000134D82F8CC3118DAB5F8CE31E0B283EA74
:108890000020082310F4004F4FEA400018BF80F476
:1088A000815003F1FF3318BF80F0010013F0FF0384
:1088B00080B2EFD1A2F8CE0138BD01318B4201BFA9
:1088C000002385F8CC31012385F8CD3138BD00BFB8
:1088D0008012002010B5044606F0F2FC40F6AC51C0
:1088E000114BD3F8F821821A8A42C4BF002283F8C0
:1088F000FC2193F8FC212AB90F2C13D10A49C1F8A5
:10890000F80101E0182A0DD8511CC9B219290648EE
:1089100083F8FC11134483F8FD410CBF01230023AD
:1089200080F8163210BD00BF8012002038B50F4B02
:10893000D3F82802B3F8244280F31000201A0DF077
:10894000FDFB0B490DF04EFC054620460DF0F6FBF5
:10895000014628460DF0FAFC0DF00AFE6428A8BF77
:10896000642020EAE070C0B238BD00BF8012002051
:108970000000C84210B50949094B91F81C021A7849
:10898000B1F82C3291F81B1202FB1034081A642340
:1089900063435043B3FBF0F0C0B210BD801200201F
:1089A0006100002038B5144D95F82F3205EB4303D4
:1089B000B3F83E0280B2A5F846020DF0BBFB05F508
:1089C000127104F0A4FA95F8183203EB43140DF079
:1089D000F5FD44F6FB7380B200FB043495F81932C0
:1089E000C3EB0333B4FBF3F395F81A42B3FBF4F390
:1089F000A5F82C3238BD00BF8012002010B5174AF0
:108A00004300D118032891F86C1203D8144C246841
:108A1000E40503D511B1022915D010E0022802D9CE
:108A2000032802D00BE00F4B05E00D4B1B6813F43D
:108A3000805F0C4B01D0188A10BDD88A10BD0A4B3C
:108A400033F8100010BD134493F86D0200EB800062
:108A500000EB800000F2EE2080B210BD80120020FA
:108A600070360020743600200034002008B506F06F
:108A700027FC074B022283F89422D3F89822C3F8EC
:108A80009002C3F8A422012283F8BD2208BD00BFD2
:108A90008012002008B506F013FC084B022283F870
:108AA0009422D3F8A42200F5B71000F5587002F212
:108AB000DC52C3F89002C3F8A42208BD8012002043
:108AC0000022064B03EBC2031979814201D11846FB
:108AD000704701321C2AF4D10020704754A40108C9
:108AE00010B5124C94F8C032012B10D009D3022BD0
:108AF00012D1D4F8C422B4F8C812D3684B40D36062
:108B00000AE0D4F8C432B4F8C8221A6104E0D4F8F8
:108B1000C432B4F8C8225A6106F0D2FB00F5F42042
:108B200000F59070C4F8DC0210BD00BF8012002078
:108B300038B50D4C0546D4F8E032834207D106F033
:108B40007DFA04F538700021482210F07EF9D4F83F
:108B50002833AB4207D1284606F070FA03480021BB
:108B6000482210F072F938BD80120020A8150020AC
:108B70002DE9F743012006F093FA0346002B4CD071
:108B80001C7800220C21514325480D18095660B26B
:108B9000814202D12A895ABB02E00132052AF1D171
:108BA000204AD2F8E0421CB1D2F82823AABB012403
:108BB0001A791D4B002503EB820303228DE8240064
:108BC00001212A46D3F8E03006F08BFC4FF048082C
:108BD00008FB04F4134F814607F53876264438B174
:108BE0003046294642463C4410F02FF9C4F8E09242
:108BF0000C490C4691F87023042A0CD81046531CDB
:108C0000DAB20A4B03EBC0039888C007F4D581F8A9
:108C100070230233B2E784F8702303B0BDE8F08319
:108C2000C43600208012002054A401089A36002087
:108C3000074BD3F87433597A4A1CD2B219445A728A
:108C40008872197A914202D8184606F00DBB704717
:108C5000801200200FB407B5074904AB53F8042B6A
:108C6000D1F874030549019304F0FEFA03B05DF8EE
:108C700004EB04B0704700BF80120020F920010807
:108C800007B5064B06480093064B07490193074A70
:108C9000074BFFF7DFFF03B05DF804FBDAC4010800
:108CA000E4C70108E3C4010805C801080AC80108AF
:108CB000CEC4010870B5224890B0FFF7CBFF002466
:108CC000E0B208A904F03CF89DF82430002B32D023
:108CD0000F980DF02FFA01461A480DF037FB0DF0F2
:108CE00047FC0C9B4FF47A7603FB00F202F59C5292
:108CF0000832B2FBF6F10E9D019005FB00F20A204E
:108D0000009591FBF0F502F59C520832B2FBF6F2A9
:108D100000FB1511039192FBF0F100FB112205926B
:108D20000D9A0491B2FBF6F202950692064821468E
:108D3000089AFFF78FFF01340F2CC1D110B070BD1E
:108D400011C80108002474495AC801082DE9FF41DF
:108D5000314C324E94F87A53B4F8787306EB8505AB
:108D6000D5F800116425B7FBF5F02D4BD4F898E247
:108D7000B4F82C221B78009181B205FB10702546B7
:108D8000019180B24FF47A71BEFBF1F10290254857
:108D9000FFF760FF244B25481968254B0027B1FBDE
:108DA000F3F1FFF757FF234BD3F80080FBB206EB3C
:108DB0008302D2F81011E9B101249C4014EA080F93
:108DC00016D0220714D01C4A0B20D25C00FB0323D0
:108DD000124A1A4802EB8303D3F83021FFF73AFF17
:108DE000022C05D1164B997A11B11648FFF732FFC4
:108DF0000137DBE7144809F0D1FA144B144C1988F9
:108E0000144BB5F87C231B1B134892B21B1104B002
:108E1000BDE8F0411EE700BF8012002054A4010805
:108E20006100002091C8010864000020EAC8010820
:108E300040420F008C17002068000020FAC801088B
:108E4000C816002002C9010862C90108D0390020F3
:108E500098E4010878E7010806C9010830B585B033
:108E600004460D46FFF7CAFB002855D0237903F0CE
:108E70000F02052A34D8DFE802F00305080A0D0FB7
:108E800001782EE090F900102BE0018829E0B0F97C
:108E9000001026E0016824E06946006804F06AF9E1
:108EA00001461E48FFF7D6FEB5B3237913F0C00F75
:108EB00032D1D4F805000DF041F9694604F05AF9B1
:108EC00001461748FFF7C6FED4F809000DF036F941
:108ED000694604F04FF901461148FFF7BBFE1BE05D
:108EE000002113F0C0030CD0402B15D162790D4B3B
:108EF00003EBC203D3F8E03153F82100FFF7AAFED9
:108F00000AE00948FFF7A6FE35B10848D4F8051075
:108F1000D4F80920FFF79EFE05B030BD8CDB0108B8
:108F200085DB010854A4010852D901083AC9010897
:108F30002DE9F843002581462C46124E04EB041718
:108F4000F319D3F84882494640460FF0FFFF68B155
:108F50000D484146FFF77EFE06F5127038440021A9
:108F6000FFF77CFF094809F019FA01350134A72CF5
:108F7000E3D125B9BDE8F843054809F00FBABDE8CB
:108F8000F88300BF54A4010853D7010862C901083F
:108F900041C901082DE9F74F05460FF09AFF064633
:108FA00020B101281CD12B782A2B19D1674809F050
:108FB000F5F90024664D04EB0417EB19D3F84812B9
:108FC0006448FFF747FE05F5127038443146FFF755
:108FD00045FF0134604809F0E1F9A72CEAD1B2E07D
:108FE00028463D210FF067FF002800F0A7800346C8
:108FF0001C4613F8012D202AFAD0641B0130834649
:109000009BF800300130202BF9D04FF0000ADFF838
:1090100040810AEB0A1308EB030606F51276D6F830
:109020000090019348460FF054FF8446494662463B
:109030002846CDF800C00FF055FFDDF800C0019BB9
:1090400000286FD1E2B262456CD1357908F5127A09
:109050009A4415F0C0030AD0402B61D104467679BA
:10906000F60008EB060393F8E421234636E0584661
:109070000FF084FF0446584603F0E6FF0746D6F893
:1090800005000DF05BF8014638460DF05DFA00284A
:1090900046D0D6F809000DF051F8014638460DF0DB
:1090A00049FA00283CD005F00F03052B1AD02746BB
:1090B00018E0B0B908EB0601D1F8E0118DE80C001A
:1090C00051F8240059460FF0C9FE9DE80C00B0FA93
:1090D00080F0400908B1274601230134E1B29142F2
:1090E000E7D3EBB15046FFF789FA78B105F00F05E9
:1090F000052D0BD8DFE805F0030305050709077008
:1091000004E0078002E0076000E00760494613487A
:10911000FFF7A0FD5046002103B0BDE8F04F9DE6EB
:109120000F4806E00AF1010ABAF1A70F7FF46FAF0A
:109130000C4803B0BDE8F04F09F030B9284603B041
:10914000BDE8F04FF4E603B0BDE8F08F50C9010868
:1091500054A4010853D7010862C9010865C9010870
:1091600070C9010841C901082DE9F047304B86B0AC
:109170009B780746012B01D004464AE00FF0A9FE78
:109180000546064603A96846FEF79CFF039B049A22
:10919000029713442B443F2B059519D900236846A9
:1091A00003A90322FEF7BAFF039B3BB9049B2BB92B
:1091B000204A13705370059BABB301E0FEF76AFFC2
:1091C000039B049A059E134433447F2B2BD8029FA4
:1091D000DFF860903946CA461AF8024BC4F180089D
:1091E000B04528BFB0460AEB04004444E4B242460E
:1091F0000FF0C8FE802C89F8004014D1C8EB060699
:10920000504607EB080132460FF0BCFE89F80060BB
:1092100009E0254614F8011B21B1074B186806F038
:10922000E9F9F6E7ED1B284606B0BDE8F08700BF78
:10923000E103002044160020800D00200FB407B584
:1092400004AB53F8042B05490020019304F00CF8FB
:1092500003B05DF804EB04B0704700BF059400084C
:10926000304B10B51C68304B1B6823602F4B1A68BD
:1092700062605A689B68A260E3602D4B1A682261A5
:109280005A689B686261A3612A4B1A68E2615A6856
:109290009B6822626362284B1A8822855A886285FD
:1092A0009A88DB88A285E385244B1A6822865A684F
:1092B00062869B68A386224B1A88E2865A889B881E
:1092C0002287224622F83A3F1E4B197800238B4210
:1092D00006DA1D4830F81300013322F8020FF6E7D2
:1092E0001A4B1B88A4F86430194B1B88A4F866300D
:1092F000184B1A68A4F86C205A689B68A4F86E2072
:10930000A4F87030144B1B68A3660BF033FA134BB0
:1093100060671B88A4F87830114B5B89A4F85E3035
:1093200010BD00BF4C370020B8390020303000207D
:109330003C30002048300020642F0020782F00208F
:10934000CE0F00206C25002024250020C61400200C
:10935000C8330020A0270020D80F0020AC10002028
:10936000F003002008B5104B01469B78012B13D168
:109370000E4B1878421CD2B21A70120648BF002257
:10938000184448BF1A708170FEF7B0FF3F2809D912
:10939000BDE80840FEF788BF054B1868BDE80840E7
:1093A00006F028B908BD00BFE103002044160020E4
:1093B000800D00200FB437B506AC54F8045B48208C
:1093C000FFF7D0FF2020FFF7CDFF2A4623460B49A9
:1093D0000020019403F048FF04460A20FFF7C2FF73
:1093E000074BC4F1FF241A6804F57F04FD341444CC
:1093F0001C6003B0BDE8304004B07047059400081D
:10940000840D00200846ADE770B54720FFF7AAFF9E
:10941000174B1B681B0307D5164B174A5B68106870
:109420001B68C01A01F0BEFD144E154C154D307866
:1094300001F0B8FD23682868C01A01F0C3FD636815
:109440006868C01A01F0BEFD0F4B188801F0AAFD34
:109450000E4B188801F0A6FD0D4B188801F0A2FDF7
:10946000337823742B68A3606B68E36070BD00BF22
:10947000940D00204C370020B8390020F80F002050
:1094800038370020FC0F0020F60F0020F40F0020DA
:10949000C01000200A4A138801331380094A136858
:1094A00001331360084A138801339BB2202B01BF9C
:1094B00000231380054A138808BF013313807047C7
:1094C0009A0D0020A00D00209C0D0020CC3800201B
:1094D00038B5294B05461B780C46093B012B4AD869
:1094E0004520FFF73FFF2846FFF73CFF0E2D33D006
:1094F00003D83DB10D2D07D038BD142D20D0FF2D40
:1095000032D038BD20682BE0637820789BB180F0A2
:109510008000FFF727FFA568E8B2FFF723FFC5F338
:109520000720FFF71FFFC5F30740FFF71BFF280EBB
:10953000FFF718FF04E0FFF715FF606801F042FD38
:109540002078FFF70FFF606801F03CFD2489E0B24E
:10955000FFF708FF200A0BE0206801F023FD606898
:10956000BDE8384001F01EBD0448FFF7FDFD0020B6
:10957000BDE83840F6E638BDE003002062D50108BA
:109580002DE9F04FBC4B8BB018880093DFF818839F
:10959000002840F0B18098F80030012B05D198F8F0
:1095A0000100A0F1200460426041B44D00F00100D0
:1095B0000BF062F8FFF754FE2C6849202646FFF7AF
:1095C000D1FEAF4B04F11C09186801F0EBFC56F812
:1095D000040B01F0E7FC30460AF032FE04F1100003
:1095E0000AF02EFE1027A74E01233268BB4013421B
:1095F00003D0D9F8000001F0E5FC0137132F09F181
:109600000409F0D1A04F04F128000AF009FE3B88BC
:10961000B4F92E00B946C01A01F0C4FC336813F443
:10962000805F08D0994BB4F864001B88181AC0F307
:109630000D0001F0B7FC3368990403D5B4F8660057
:1096400001F0B0FC33685A0503D504F16C000AF050
:10965000E7FD33681B0502D5A06E01F0B3FC33684B
:109660005F0402D5606F01F0ADFC3368180403D5C8
:10967000B4F8780001F096FC274604F130000AF0B7
:10968000CFFD04F136000AF0CBFDB9F8003037F910
:109690003C0F4FF00109C01A01F084FC7C4B1B7891
:1096A000994509DA37F9020FB4F93C3009F101099B
:1096B000C01A01F087FCF1E73368990505D5B4F9C4
:1096C0005E00A0F2DC5001F07DFC2A6871486A60FF
:1096D000AA60121A9110704A4A43531C032293FB4A
:1096E000F2F202EB42029A1A7C2303FB02032B6084
:1096F0006A4B01221A70DCE1694B6A4A1B681168E7
:109700008B4206D00AA941F8203D00201360FFF7E4
:10971000DFFE009B98F800101B8898F801000B44AE
:10972000013BB3FBF0F200FB12338B4280F08C81E3
:10973000524F01200AF0A0FFFFF792FD50203E6833
:109740007D68FFF70FFEBA683B6810681B687A688F
:109750000344106806F11C09A3EB400001F032FC41
:109760006A68736802A89B1A0293AA68B36805F135
:109770001C0B9B1A0393EA68F36810249B1A04934A
:109780000AF05EFD2A69336902A89B1A02936A698E
:1097900073699B1A0393B369AA699B1A049301F036
:1097A00071FB384801210368A1401942019006D09D
:1097B000D9F80000DBF80030C01A01F003FC0134D6
:1097C000132C09F104090BF1040BEAD106F1260070
:1097D00005F12601002331F9024F30F9022F121B47
:1097E00002AC44F823200133042BF4D103214FF0C1
:1097F000000A02AB53F821304FEA8A025FFA82FA7C
:109800006BB103F108000F2802D84AF0010A06E004
:109810008033FF2B94BF4AF0020A4AF0030A11F189
:10982000FF31E6D250464FF0000BFFF79BFD5C4640
:109830000DF108090AF00300022815D0032835D0DD
:10984000012850D134B9D9F8003004461B015FFA21
:1098500083FB48E0D9F80000002400F00F0040EA44
:109860000B00FFF77FFD3EE02CB3D9F80000C0F3FA
:10987000031040EA0B002FE09C0D00204C37002025
:10988000A00D0020940D002046240020980D0020FB
:109890006C25002058370020DF7BEFBDDA0D00205B
:1098A000D8330020D0380020E103002044B999F8D3
:1098B0000100FFF757FD99F80000FFF753FD12E094
:1098C000D9F80000C0F3033040EA0B00FFF74AFD6F
:1098D000D9F80000C0F30710FFF744FDD9F80030B5
:1098E0001B015FFA83FB09F1040906AB99454FEAB6
:1098F0009A0A9FD1012C02D15846FFF733FD019BF4
:109900001B6813F480541FBFB6F86420B5F86410C8
:109910000124521A18BF02929A040AD50AAA02EB2D
:109920008401B5F86600B6F866200134121A41F8D1
:10993000202C580513D502AA02EB840C06F16A0EFE
:1099400005F16A0000223EF9021F30F902BFCBEB9D
:1099500001014CF822100132032AF4D10334190515
:1099600008D50AAA02EB8400A96EB26E0134521A1D
:1099700040F8202C5A0408D50AAA02EB8400696F2B
:10998000726F0134521A40F8202C18040AD50AAB21
:1099900003EB8402B5F87810B6F8783001345B1A1E
:1099A00042F8203C002C20DD012C03D1029801F06C
:1099B00009FB1AE0631E002002AA52F8232040008F
:1099C000C0B20AB140F0010013F1FF33F4D2FFF747
:1099D000C9FC4FF0000B02AB53F82B0008B101F0AB
:1099E000F1FA0BF1010BA345F5D1302003210AF068
:1099F0009FFE362003210AF09BFE324B3C20197853
:109A00000AF096FE019B1B68990506D5B6F95E0023
:109A1000B5F95E30C01A01F0D5FA3A682A487B6879
:109A20007A60121A9110294ABB604A43531C0322E0
:109A300093FBF2F202EB42029A1A7C2303FB02032D
:109A40003B60234B01221A70224B1B681A0630D54B
:109A5000214C224D22682B689A420BD162686B68B8
:109A60009A4207D1009B1B88102B11D11C4B1B88DD
:109A70005B060DD14820FFF775FC206801F0A2FAC3
:109A8000606801F09FFA23682B6063686B600EE0EA
:109A9000144A124B11782A7C914208D1124A9968D3
:109AA0001068884203D15268DB689A4201D0FFF700
:109AB000ABFC98F80230012B01D1FEF7F5FB0BB09F
:109AC000BDE8F08F6C25002058370020DF7BEFBD0C
:109AD000DA0D002070360020B0100020383700204A
:109AE000CC380020F80F0020FC0F00202DE9F74FA4
:109AF0000E9FC2EB030B4D4C0D9B002914BF4FF082
:109B000006094FF00409FF1A6368824601331646BE
:109B100035D122684A4580F08580DFF82C8101919B
:109B200058F822000FF0D5F90B3001F055F90199E2
:109B3000054608B1012076E022683D48032A98BF17
:109B4000514658F82220FFF779FB3A4A1368181A51
:109B50006368106001336360374B83F882500EE016
:109B60000D9A92B103FB07F20D99895C01228A409C
:109B7000324909680A4208D1636801336360636847
:109B80000C9A2A4D9342EBDB34E003FB0BF5236880
:109B900006EB050A2BB970590FF09BF900F1050887
:109BA00001E04FF00308404601F016F90028C1D14A
:109BB000204A214B1068C8EB0000106093F8822007
:109BC0001AB12C20FFF7CEFB02E0012283F882209D
:109BD000236843B97059FFF7C7FA9AF904104B1C70
:109BE000CAD0174803E09A4416489AF80410FFF7C1
:109BF00025FBC1E710D1012001F0EEF860B90D4A54
:109C00000A201368013B1360FFF7ACFB2B6801339C
:109C10002B604FF0FF336B60206848452CBF00205D
:109C2000012000E0002003B0BDE8F08F8C0D002083
:109C30006DD50108840D002044160020940D0020ED
:109C40007CD5010852D901088CB201082DE9F04FEA
:109C500000218DB00C22A9480FF0F7F8A84E002182
:109C60001422A8480FF0F1F8A74B377803F1180237
:109C7000012F94BF1F461746A04C002529460C22F1
:109C800004F1240084F8205084F821500FF0DDF80E
:109C90002320276305F03BFB752001210DF10F0206
:109CA000FDF718FBA0B1994B2846A362984B012100
:109CB000E36204AA432384F82430FDF70BFB9DF8EC
:109CC000103003F07E038DF81030002844D14CE0B2
:109CD00094F834305BBB8F4A8F4D93694FF48057B3
:109CE00043F00803936110238DF81A3028460323AC
:109CF00006A98DF81B30ADF8187008F070FF874A80
:109D00002F61138823F040031B041B0C138013885E
:109D100023F038031B041B0C43F008031380138843
:109D20009BB243F040031380012384F83430752044
:109D3000012106AAFDF7BCF89DF81830703B012BF5
:109D40005AD8052384F82030432384F82430744BF8
:109D5000A362744BE3624FE0682B06D1012384F8C1
:109D600020301D2384F8243046E09DF80F3003F0A6
:109D70007E03682B8DF80F3039D10223062084F83A
:109D8000203006AAA36A014698479DF81B309DF82B
:109D90001D2003F001035B0002F0010243EA82028E
:109DA0009DF8193003F00103134312D05AB2012A6F
:109DB00001D1002302E0022A03D1012384F82130DB
:109DC0001AE003F00303032BF7D0032005F016FB82
:109DD00012E04A4B0C209B6A012105AA98479DF886
:109DE000143013F00F03F0D0042BE6D1E1E7702B11
:109DF00004BF042384F8203094F820204A4F002028
:109E0000022A38703D4B0AD14849D9604849196146
:109E1000484999614849D96101233B701DE0012AF5
:109E20000CD146493A70D96041490422196144492C
:109E30005961404999614049D9610EE0043A012ACB
:109E400000F242833F4ADA60394A1A61394A9A611C
:109E5000394ADA6101233B7007223B4BD4F8C490A6
:109E600098461A7094F8385049F00102C4F8C4209A
:109E7000002384F83530082D00F2B680DFE805F0C5
:109E80000BB40B296E8D29A4A400012D40F2B680DD
:109E9000002583F835503378012B1AD84FF0000A8B
:109EA0000CAB03F818AD532051460122FDF730F9F1
:109EB00078B19DF81830E52B0BD1244B0422236098
:109EC000234B84F836A063600C4B83F835200223C3
:109ED0008EE094F82020094B022A3FD11D4A1A60D7
:109EE0001D4A5A6093F82130002B0CBF6F236E235C
:109EF000A372012384F83530032379E0C8160020CB
:109F0000D93A0020D4160020A4B20108D572000866
:109F10006175000800100240000C0140003800404C
:109F2000B16E0008DD6E0008DA3A00208570000886
:109F3000AD6D0008996D000890C1793DFD6E000877
:109F4000616D0008F96F00086800002019760008AC
:109F500089730008E9700008F56D00083378012B5B
:109F60001BD800220CAB03F8182D1C200D21012258
:109F7000FDF7CEF888B19DF818302A2B01D01A2BA6
:109F80000BD1D24A84F837302260D14AD14B62607B
:109F9000022283F8352004232AE000210CAB03F8C9
:109FA000181D18200122FDF7B3F868B19DF818308C
:109FB000FB2B09D1C84B01222360C84B6360C54B02
:109FC00083F83520052313E094F82020C14B043A90
:109FD000012A3FF65AAFC24A1A60C24A5A600122A9
:109FE00083F83520082303E0012D07D900253FE73A
:109FF00088F8013049F00303C4F8C430337894F88A
:10A000003A50012B05D109F0ABFFB74B4FF400528A
:10A010005A61042D00F2D381DFE815F00500DC0160
:10A020006800050099010A2005F071F97720A02148
:10A03000012205ABFDF76CF8002857D01E21012244
:10A040007720FDF709FA4FF42F6005F055F9002548
:10A05000A5F160014FF00009C9B2022206AB7720DA
:10A060008DF818908DF81990FDF752F89DF8193079
:10A070009DF8182043EA0222964B03F13C016A52F4
:10A080000235102DE4D1B3F84A104A4601F00F0E04
:10A0900001F47F41A3F84A104B46012522F001004C
:10A0A0002044808F002818BF002512F0010F03D034
:10A0B000C0B24340082002E083EA1023FAE713F419
:10A0C000004F18BF83F4C05301384FEA4303F6D161
:10A0D0000132102AE2D141EA0E017E4AA4F84A1068
:10A0E00025B9C3F303339E4500F0D18194F84C9019
:10A0F000784DB9F1000F40F0E581DFF8ECA109F0EF
:10A100002FFF4FF4804B2823504605A9ADF814B01B
:10A110008DF81630019308F062FD019B4FF4005258
:10A120001846CAF81020714905F0B6F90E21022030
:10A1300008F040FD0822CDF818B006A84FF0010B3A
:10A140008DF81D208DF81C908DF81EB00BF0CAF80C
:10A15000019B4FF0030C04A88DF810308DF811C04E
:10A16000CDF804C08DF812908DF813B009F090FE70
:10A17000142005F0CCF8D02177205A4605ABFCF727
:10A18000C7FF5146002800F0BF809DF81430DDF86D
:10A1900004C0552B85F86730A5F870C040F0B48036
:10A1A000D1215A4605AB7720FCF7B2FF9DF8143059
:10A1B000772003F00F021B0985F8682085F86930C5
:10A1C000162206ABAA21FCF7A3FF9DF818209DF8E4
:10A1D000193043EA0223A5F850309DF81A209DF863
:10A1E0001B3043EA0223A5F852309DF81C209DF84D
:10A1F0001D3043EA0223A5F854309DF81E209DF837
:10A200001F3043EA0223A5F856309DF820209DF820
:10A21000213043EA0223A5F858309DF822209DF80A
:10A22000233043EA0223A5F85A309DF824209DF8F4
:10A23000253043EA0223A5F85C309DF826209DF8DE
:10A24000273043EA0223A5F85E309DF828209DF8C8
:10A25000293043EA0223A5F860309DF82A209DF8B2
:10A260002B3043EA0223A5F862309DF82C209DF89C
:10A270002D3043EA0223A5F8643041F27073A5F84B
:10A28000743046F67813A5F87630194BAB67194B46
:10A29000EB67194BC5F88030184BC5F88430184B64
:10A2A000C5F8883095F84C304BB9FDF74FF942F6B8
:10A2B000E06005F021F8DAF80830C3F38039114B7B
:10A2C00083F80090012384F84C30FBE06B750008A4
:10A2D000E9720008C8160020F975000843730008E9
:10A2E00075700008F56D0008001001405D6E0008F3
:10A2F0004D750008A1720008297500085572000804
:10A30000856C00080B000020714A136823F4804319
:10A31000136000236F48DA0000F18C0505EB020E94
:10A32000DEF804C0DFF8E4E1F4450AD115F9335052
:10A33000282D06D183180022C3F8902083F88C20A2
:10A3400002E00133032BE5D14FF400534B6194F845
:10A35000A490604DB9F1000F40F0AE80142004F0DD
:10A36000D6FF05F1A5037620D0210122FCF7D0FE0F
:10A3700095F8A530582B2DD105F1A8038821182276
:10A380007620FCF7C5FE7620F4213122FDF764F833
:10A39000012385F8A430504BA5F87490EB674F4B20
:10A3A000AB6745F6D813A5F876304D4BC5F880302D
:10A3B0004C4BC5F884304C4BC5F888307CE0012DFF
:10A3C00008D02B4688F80230D4F8C43043F0040398
:10A3D000C4F8C430D4F8C4303E489B0704D54FF4C9
:10A3E0008073038103689847E36894F8C90098472D
:10A3F0003E4B367803F11802012E94BF1E461646D6
:10A4000094F839500023042DDFF8C89084F8CC303C
:10A4100001D91D46F6E7012202FA05F313F01A01ED
:10A420004CD113F0050F49D00CAB03F8181D1E20BA
:10A430000A21C9F8D060FCF76BFE00283ED09DF8D9
:10A440001830482B3AD12A4BC9F8D430294BC9F8D7
:10A45000D830032384F8CC30022388F80330D4F8B2
:10A46000C43043F00803C4F8C43094F8DC3003B1BE
:10A470003B7094F8DD3013B1164A82F8353094F809
:10A48000DE3013B1134A82F8CC3001201CE042F2D6
:10A490001073A2F87430A2F87630174B9367174BFD
:10A4A000D367174BC2F88030164BC2F88430164B76
:10A4B000C2F88830032385E7042383E7012DD4D92C
:10A4C00000259FE702237DE70DB0BDE8F08F00BFB8
:10A4D00000040140C8160020C56A0008C76A0008C9
:10A4E00011750008C171000805690008D4B201089F
:10A4F00065B00008CDAF000821750008457200085E
:10A500001975000835720008C96A00085D6E0008F8
:10A510002DE9F84303460D4600685968584C023A45
:10A5200003C4986844F8E809062A05D8DFE802F071
:10A530000A101822292F3500D4F8E0302B60D4F807
:10A54000E43013E0D4F8E4302B60D4F8E03005E0D8
:10A55000D4F8E0305B422B60D4F8E4305B4205E095
:10A56000D4F8E4305B422B60D4F8E0306B60D4F870
:10A57000E8301DE0D4F8E0305B422B60D4F8E430E2
:10A5800012E0D4F8E4302B60D4F8E0300CE0D4F8DA
:10A59000E0302B60D4F8E43005E0D4F8E4305B42DE
:10A5A0002B60D4F8E0305B426B60D4F8E8305B425B
:10A5B000AB60344B5B78002B5FD128680BF0BEFD9D
:10A5C000804668680BF0BAFD0746A8680BF0B6FD38
:10A5D000D4F8EC10064640460BF004FED4F8F81010
:10A5E000814638460BF0FEFD014648460BF0F2FC72
:10A5F000D4F80411814630460BF0F4FD014648467C
:10A600000BF0E8FC0EF03AFED4F8F010286040465B
:10A610000BF0E8FDD4F8FC10814638460BF0E2FD63
:10A62000014648460BF0D6FCD4F808118146304666
:10A630000BF0D8FD014648460BF0CCFC0EF01EFE98
:10A64000D4F8F410686040460BF0CCFDD4F800114B
:10A65000804638460BF0C6FD014640460BF0BAFC7A
:10A66000D4F80C11074630460BF0BCFD01463846C5
:10A670000BF0B0FC0EF002FEA860BDE8F88300BF4E
:10A68000A81700200B0000202DE9F34105690646BC
:10A690000F46002D5BD1D0F80080C8F3090353B1F9
:10A6A00000234FF40050D6F80080019309F072FFA8
:10A6B00004284AD120E04FF4302009F06BFF042831
:10A6C00002D04FF0FF3542E0234C4FF43020236995
:10A6D00043F002032361C4F81480236943F040036C
:10A6E000236109F057FF41F6FD732269042803EA4C
:10A6F00002032361D4D0E4E7174C4FF400502369E0
:10A7000043F001032361BBB2A8F8003009F042FF17
:10A71000042815D108F102030193019B3F0C1F800F
:10A720004FF4005009F036FF41F6FE732269042809
:10A7300003EA0203236108D133680433336006E07F
:10A7400041F6FE732269134023616FF0010528462C
:10A7500002B0BDE8F08100BF00200240064B10B5FA
:10A760001A881C4622EA00009042188002D001207C
:10A7700004F02CFE208810BD622F0020064B10B57F
:10A780001A881C4610439042188002D0012004F021
:10A790001DFE208810BD00BF622F002008B5104BA1
:10A7A0001A780023D9B2914207D20E49002051F8FD
:10A7B0002310013309680880F4E7322004F0A7FD74
:10A7C000094B1B685A0309D5084B1B685B0305D46A
:10A7D000BDE8084040F2DC5004F099BD08BD00BF60
:10A7E0006C2500203C2500207036002060310020C0
:10A7F0002DE9F04F8BB0FEF74DF94FF00309714C86
:10A800000021A046182204A80EF01FFB6E4B6F4AD1
:10A810001B1B05936E4B04945A6002F188325A60F8
:10A82000342101228DF82420D96000238DF80730CF
:10A830000AA9702301F8243D04A803F027F89DF825
:10A8400007209DF80430634D53408DF80730624B6C
:10A850000DF1080B9D4264D26A880024C2F30B06F6
:10A86000B31DADF808302B888DF80D40C3F30B01F4
:10A870001B0B8DF80C301304ADF80A1021D404A87A
:10A880005946062203F002F89DF807301BF8042011
:10A890000134062C83EA0203F8D1324604A8696821
:10A8A0008DF8073002F0F2FF6B689DF807201E4418
:10A8B000B34203D013F8011B4A40F9E78DF8072093
:10A8C0002DE0A2460AF1010A06225FFA8AFA04A8DC
:10A8D00059468DF80DA002F0D9FF9DF807200023FE
:10A8E0001BF803100133062B82EA0102F8D16F68CE
:10A8F0008DF807202744324604A8394602F0C6FFE7
:10A900009DF80730BA19974203D017F8011B4B4046
:10A91000F9E7BAF1030F8DF807303444D2D110357E
:10A9200095E759460222002404A8ADF8084002F039
:10A93000ADFF9DF807209DF808300AA953409DF807
:10A94000092004A85340DB43012201F8213D02F015
:10A950009DFF079A72B104AB02F10800184421462A
:10A96000C2F104020EF071FA04A80699FFF78CFEFA
:10A97000079408909DF8243023B1154A136943F0D9
:10A9800080031361089BB9F10109B3FA83F34FEA1D
:10A99000531303D0002B3FF432AF04E01BB9052062
:10A9A00004F02CFD08E098F80030702BF7D100205F
:10A9B00002F02CFF0028F2D0FEF758F80BB0BDE8EB
:10A9C000F08F00BF00F00108000002082301674576
:10A9D0000020024098E4010878E701082DE9F047DB
:10A9E000FEF758F8994B1B78702B03D0042004F025
:10A9F00005FD04E0012002F009FF0028F6D0944B89
:10AA0000944C187802F084FE2368934A1B780C213A
:10AA1000032B28BF00231370904A914E01FB0323A0
:10AA2000904A136046F2090233681A4012B943F49F
:10AA3000005333603368DF0703D546F2080002F0A5
:10AA40005FFE33685D0403D542F2090002F058FE50
:10AA50003368180703D546F2010002F051FE33684F
:10AA6000990403D544F2090002F04AFE7E4B1B789C
:10AA700023B17E4B5A780AB100225A707C4DAB78D4
:10AA80003BB1EB78012B04D833681A0644BF02238C
:10AA9000EB7033685B0603D54FF4803002F030FE74
:10AAA0004FF0000E7646734B73449F88790801F08F
:10AAB0007731BB0803F03333781AC11AFB0803F06F
:10AAC0001133CB1A03EB231303F00F32FF2392FB56
:10AAD000F3F317F0010CC3EB032318BF0136A2EB0D
:10AAE000030318BFF6B2012B0ADD022B40F0A98048
:10AAF000BCF1000F00F0A58017F4DE7F00F0A1800C
:10AB00000EF1080EBEF1280FCDD1013E012E00F24C
:10AB1000988004F041FB04F025FB04F0D9FA3022C0
:10AB2000002155480EF091F9544B0021186804F0AB
:10AB300075FB534E534B80F00100187033684FF093
:10AB40006408987F07F0C6FA3068FDF745F94E4A69
:10AB50004E4B1278DFF8889108FB02F2C8325A6037
:10AB600000229A60DA601A615A619A61DA6183F8A8
:10AB7000202083F82120464A464B1A60464B1A682B
:10AB8000464B1A60464B1B6813F0080F1BD0454B11
:10AB90001B68B3F9007097FBF8F630460BF0CEFA5D
:10ABA000824608FB167000B20BF0C8FA3E490BF063
:10ABB00019FB014650460BF00DFA3C490BF012FB15
:10ABC000C9F8000002E00023C9F80030A8880BF0A3
:10ABD000B5FA37490BF0BAFBE060E8880BF0AEFA43
:10ABE00033490BF0B3FB334BA0601B6832491A7931
:10ABF0000C3322719A7862712A7A22742F4A53F8A0
:10AC0000040C126814882E4A11602E4A2E491360D3
:10AC10000BF0E8FA01464FF07C500BF097FB2B4B02
:10AC2000186020460BF08AFA014629480BF08EFB8B
:10AC300028490BF0D7FABDE8F047274B1860FDF71D
:10AC400015BF264802F0C3FD63E700BF00F001080E
:10AC500018310020D8170020D8130020F43000202D
:10AC600060310020F0300020B10E00205031002073
:10AC7000D00300209A360020CC0E0020F4220020C1
:10AC80008027002006000020A93900201C15002084
:10AC9000B0270020E4380020081F0020C832002020
:10ACA0008C170020DC0300208988883C00002041AC
:10ACB00000401C4610160020DC1700206C0B002002
:10ACC000E00A00202C0B0020DB0F4940280B00205D
:10ACD000000061444C3D0F44700B002048E7010820
:10ACE000180B0020022888BF002008B5034B1870FD
:10ACF000FFF77EFDBDE8084070E600BF1831002078
:10AD000008B5FFF775FDFFF769FEBDE808400120B3
:10AD100004F05CBB38B5264C264DAC4219D2B4F9D0
:10AD20000230002B04DB2046616802F00BFD0EE0D0
:10AD30000025638861681A0444BFC3F30B0305FB55
:10AD400003112046013502F0FDFC032DF1D1103432
:10AD5000E2E70024184B20461C7002F0D9FC174B88
:10AD6000174A1C70174B18481A6009F076FA174AF0
:10AD7000174B0F4C1A60AC4214D2B4F90230002BBE
:10AD80000EDA62886168C2F30B0288180EF0FAF8D6
:10AD900062886168C2F30B0201EB42000EF0F2F828
:10ADA0001034E8E70B4B01225A7502229A7538BD20
:10ADB00098E4010878E7010818310020D813002032
:10ADC000F4300020F0300020A0D501080221080056
:10ADD00060310020D817002038B5134B05461B689A
:10ADE000984219DD114B9C7814B1012C09D017E061
:10ADF0000F4B1B68186988B1A842CCBF0120022004
:10AE000038BD7F280CDCFDF771FAC0F17F00854268
:10AE100008DDFDF749FA05E0002038BD012038BD06
:10AE2000022038BD204638BD840D0020E1030020FB
:10AE3000800D0020074B9B78012B08D1064A074B59
:10AE4000D0681B68834234BF002001207047002077
:10AE5000704700BFE10300201C000020B009002063
:10AE6000064B9B781BB1012B05D1FDF71DBA044B96
:10AE7000186804F085BB0020704700BFE103002084
:10AE8000800D0020F8B5011F06460023083051F858
:10AE9000042F02F120043F2C3BD802F108040F2CB0
:10AEA00006D80232032A04D9002B08BF012300E090
:10AEB00002238142EBD1012B30680ED0022B1AD035
:10AEC000736800F0030003F003039B0043EA0010E3
:10AED000B36803F00303184317E000F00F0040F0DD
:10AEE0004000FEF73FFAB068736800F00F0040EAD8
:10AEF0000310C0B209E000F03F0040F08000FEF710
:10AF000031FA3079FEF72EFA307ABDE8F840FEF7D4
:10AF100029BA06F10C0734463A46002552F8043D9A
:10AF2000AD0003F18001FF2910D903F50041B1F50F
:10AF3000803F02D245F0010508E003F50003B3F1BC
:10AF4000807F34BF45F0020545F00305B242E5D1EC
:10AF500065F03F00C0B2FEF705FA05F00303022BCF
:10AF6000207807D0032B0CD0012B13D1FEF7FAF970
:10AF700060780FE0FEF7F6F96078FEF7F3F9A07855
:10AF800008E0FEF7EFF96078FEF7ECF9A078FEF73D
:10AF9000E9F9E0780434FEF7E5F9BC424FEAA5058B
:10AFA000DBD1F8BD10B504467F2C06D964F07F00D4
:10AFB000C0B2FEF7D7F9E409F6E7E0B2BDE8104009
:10AFC000FEF7D0B9430083EAE070EBE737B50446FB
:10AFD00003211E2006226B46FCF79AF870B39DF8F9
:10AFE00001309DF80000164D43EA002000B20BF03E
:10AFF000A5F829680BF0F6F80BF0BAFA9DF80330C3
:10B0000020809DF8020043EA002000B20BF096F881
:10B01000A9680BF0E7F80BF0ABFA9DF80530A080BB
:10B020009DF8040043EA002000B20BF087F869683D
:10B030000BF0D8F80BF09CFA6080012003B030BD13
:10B040001000002010B5054C236818690AF07AF941
:10B0500018B123681A69024B5A6110BD9817002075
:10B06000000401402DE9F0437D4A87B01368904603
:10B0700093B11A681AB17B49886902438A619A8838
:10B080009868ADF8002002228DF80320694604225A
:10B090008DF8022007F0A3FD322004F038F90021DA
:10B0A00011221E20FCF7D8F9012160221E20FCF796
:10B0B000D3F9642004F02BF9002402A8FFF786FFDF
:10B0C000274626460A25022101221E20FCF7C4F944
:10B0D000322004F01CF902A8FFF778FFBDF9082020
:10B0E000BDF90A1014448A42A8BF0A46BDF90C30C3
:10B0F0000F4493421E44A8BF134613F5805F0BDD37
:10B100005949013D8A688989D36883EA0103D3607C
:10B11000D9D14FF0010901E04FF000091E200021B4
:10B120001222FCF799F90A25022101221E20FCF7C0
:10B1300093F9322004F0EBF802A8FFF747FFBDF9BE
:10B140000820BDF90A10A41A8A42A8BF0A46BDF910
:10B150000C307F1A9342A6EB0306A8BF134613F5E3
:10B16000805F09DD4049013D8A688989D36883EAA7
:10B170000103D360D8D101E04FF0000920460AF066
:10B18000DDFF014639480BF0E1F8394D20F0004071
:10B19000286038460AF0D2FF014634480BF0D6F852
:10B1A00020F00040686030460AF0C8FF0146314890
:10B1B0000BF0CCF820F00040A860002170221E2087
:10B1C000FCF74AF9012120221E20FCF745F91E2038
:10B1D00002210022FCF740F9642004F098F8B9F14C
:10B1E000000F04D14FF07E532B606B60AB60D8F83A
:10B1F00000301B4C1A7B002A2FD01A7D6AB31949E4
:10B2000000268A69012542F001028A61187B197DB6
:10B2100007F0D0FC2368184993F9150004F03CF9B5
:10B220002368164A1B6904A8536104930C238DF804
:10B2300015308DF814608DF816500AF053F8236815
:10B2400001A85B7D8DF806608DF8043003238DF82E
:10B2500005308DF8075008F01BFE07B0BDE8F083FD
:10B2600098170020001002404415002000406F464F
:10B270001000002001C05E4645B0000800040140F7
:10B28000024640213C20FCF7E7B8024680213C20E2
:10B29000FCF7E2B8012828BF01202DE9F04F06464F
:10B2A000142000FB06F3764F89B0F918FC58754B53
:10B2B0000A691C601E71744BB1F80880DD69B1F831
:10B2C0000AA02A43DA61A2884D6822F4407212046F
:10B2D000120C4AEA0809A28003A9C5F810900222BC
:10B2E0008DF80E0028460193ADF80C908DF80F20D4
:10B2F00007F075FC019B00971F464FF0080BAA68EA
:10B3000018EA020F03D10A2003F0F6FFF7E70A203C
:10B31000C5F8148003F0F0FFC5F810800A2003F090
:10B32000EBFFBBF1010BEAD1C5F814A00A2003F032
:10B33000E3FFC5F814800A2003F0DEFFC5F8108093
:10B340000A2003F0D9FF0222C5F810A028468DF884
:10B350000F2003A91C228DF80E20ADF80C9007F0E9
:10B360003EFC4A4A4A4994423A6903A80BBF42F458
:10B37000001242F480023A613A610BBF3A693A69BD
:10B3800022F4001222F480023A61A38823F440736D
:10B390001B041B0CA3803F4B93F800803E4BB8F17D
:10B3A000000F14BF9846884623889BB243F00103E0
:10B3B0002380A58809F0A4F8059A384825F03F05B0
:10B3C000B2FBF0F02D042D0C0543ADB2A580218811
:10B3D00008EB480321F001010904090C21804FF416
:10B3E0009671B2FBF3F301FB00F24FF47A7192FB1A
:10B3F000F1F29BB2002B08BF0123013243F400435A
:10B4000092B22284A3832388009A9BB243F0010363
:10B4100023802388002523F4816323F002031B0487
:10B420001B0C23804FF480432381142303FB062647
:10B43000737B012403A88DF80C308DF80D508DF826
:10B440000E508DF80F4008F023FD337B9DF80F2040
:10B450008DF80C308DF80D508DF80E501AB103A8F0
:10B4600008F016FD08E05A0903F01F039C4002F1A2
:10B4700020030B4A42F8234009B0BDE8F08F00BF1B
:10B4800004B30108F01700200010024000540040EF
:10B49000801A0600D604002000350C0040420F0040
:10B4A00000E100E0914B70B51A68908A80B2C1B299
:10B4B000CE072ED5118821F400610904090C1180F2
:10B4C000118889B241F48061118000215971997904
:10B4D00099B1D97911B9197AFF290ED10121D97100
:10B4E000597A022901BF118889B241F400611180A3
:10B4F000997A41F001011182E2E0997A01F0FE01AE
:10B5000011821A7AFF2A00F0DB80784AFF215171FC
:10B51000D6E08D073AD5BFF35F8F587AC0B20128C5
:10B5200013D1997989B1D97979B1118821F48061E0
:10B530000904090C1180BFF35F8F118B1188D87239
:10B5400089B241F4007111801BE0118BBFF35F8F52
:10B55000587A664902280AD1887940B1C97931B14F
:10B56000118821F480610904090C1180A2E0587A45
:10B570005E49032805D1887918B1C979002940F0BE
:10B580009980918889B241F4806198E04C0757D541
:10B590000121D9729979002938D0D979002935D07B
:10B5A000597A1088022959791ED920F48060000444
:10B5B000000C1080148ADD68C8B2E4B249B26C5441
:10B5C0001188DC6889B241F4007111801968821C0D
:10B5D0005A710A8A0130D2B240B222548A8892B299
:10B5E00042F480628A8026E080B240F400701080CD
:10B5F000148ADD68C8B2E4B249B26C54128A411CA4
:10B6000049B2D2B203306A54587114E0D97937483C
:10B6100009B9017C41B1118889B241F400711180EE
:10B620005A7901325A7106E0118889B241F4807169
:10B6300011800122C27119680A88D205FCD43FE04A
:10B6400001F0400101F0FF04E1B15879168ADD688C
:10B65000C4B2611C40B2F6B22E54C9B25D7A5971BF
:10B6600049B2C81C854201BF908820F48060000464
:10B67000000C08BF90805A7A8A4221D11B4A0234BA
:10B6800054711DE006061BD5597948B2451C0AD0F5
:10B690005C690131205CC9B21082587A597149B293
:10B6A00088420DD106E0197A5C711182997909B945
:10B6B000597A29B9918821F480610904090C918093
:10B6C000597A93F9050001318842084A0CD10021CA
:10B6D000D171D17A31B111688A8822F44072120492
:10B6E000120C8A8000221A7670BD00BFF01700206D
:10B6F00010B5204C2368998A89B211F4706F1CBF71
:10B700000122627611F4E06F2AD01A8B9A8889059B
:10B7100022F480624FEA02424FEA12429A801FD41A
:10B720001A8892051CD41A88D0050ED51A88D1051E
:10B73000FCD41A8892B242F400721A801A889205D8
:10B74000FCD42079FFF7A6FD0AE01A8892B242F4F1
:10B7500000721A809A8822F440721204120C9A80A5
:10B760002268938A23F470631B041B0C93820023CA
:10B77000237610BDF0170020026D70B515880446C1
:10B78000ADB2A90613D5036B8BB9C36A1BB1908800
:10B7900080B298470BE0E169928840694E1CD2B2B2
:10B7A000E6614254E169E268914228BFE3612B06F9
:10B7B00013D5636AA26A9A42236D0AD0511CA0690C
:10B7C000A162825C9A802369994206D30023A36216
:10B7D00070BDDA6822F08002DA6070BD026B034649
:10B7E000C16810B5406942B11A6C8C1A013A08BFA1
:10B7F0000A46005D1A64C0B210BD1A6A805C01324C
:10B800008A4228BF0022C0B21A6210BD436B13B136
:10B8100090F844007047836A406A1B1A58425841A6
:10B820007047426A816A03698A4238BFD218521A45
:10B83000416B21B149680A44591E8A4203D2013B37
:10B84000981AC0B2704700207047036B13B15B6851
:10B85000016C01E0C369016A8B423CBFC2689B185E
:10B86000581AC0B27047836A8169426B1944D1602B
:10B87000416A994297BF0169CB1ACB1A536096BFB0
:10B880000023536083624FF0000380F84430136854
:10B8900088BF816243F0010313607047436A826985
:10B8A000D154436A02690133934228BF00234362A3
:10B8B000436B1BB11B68DB0705D4D4E7026DD3686B
:10B8C00043F08003D3607047417105F0F1BC8160A3
:10B8D00005F0EEBC2DE9F04105460E46078A838946
:10B8E0009BB21F40002F37D0B7FA87F24FF00043CA
:10B8F000D340DB4399B21F40A2F11B032982042BE2
:10B90000F0D8DFE803F0221F1C190300746A24B189
:10B91000013C0023A4B2736201E0AC8DA4B2D6F85E
:10B920002080B8F1000FDDD0D8F800304046214625
:10B930009847D8F80480F4E73068A98E08E070686A
:10B94000298F05E0B068A98F02E0F068B5F84010D3
:10B95000036889B29847C5E7BDE8F0814FF08040A1
:10B960000049B7E79825002001480249B2E700BF27
:10B97000002C01407025002001480249AAE700BFC1
:10B98000002C014070250020254B10B55A43254B53
:10B99000254C1B680139B3FBF2F20388013AA0423F
:10B9A00089B292B29BB212D004F50064A0420ED0CC
:10B9B000B0F1804F0BD0A4F59834A04207D004F525
:10B9C0008064A04203D004F58064A04202D123F039
:10B9D00070039BB2154CA04206D004F58064A042CF
:10B9E0001CBF23F440739BB203800F4B81859842A8
:10B9F00002850FD003F5006398420BD003F5406336
:10BA0000984207D003F58063984203D003F5806322
:10BA1000984201D1002303860123838210BD00BF19
:10BA200040420F0064000020002C01400010004044
:10BA300073B505460068FFF7A7FF2A68012413883D
:10BA400000269BB243F001031380EB7A01A88DF826
:10BA500004308DF805408DF806608DF8074008F039
:10BA600017FAEB7A1B2B0BD1192301A88DF80430A0
:10BA70008DF805408DF806608DF8074008F008FA4B
:10BA800002B070BD0C4B800A98420CD004D8B0F5BF
:10BA9000801F0CD101207047084B984205D04933D4
:10BAA000984206D003E00220704703207047FE2032
:10BAB00070470020704700BF010010000200100016
:10BAC0002DE9F84304680746204688469146FFF76B
:10BAD000D9FF03284BD8BA7A9108B8F1000F06D1E4
:10BAE000A589AEB202258D4026EA0505A5810A2367
:10BAF00003FB00131F4A42F82380043342F82390CB
:10BB0000B8F1000F07D0BD7AA189AD080223AB4080
:10BB10000B439BB2A3812823434303F1200111442B
:10BB2000EFF31286502585F3128803F10C051C33C0
:10BB30001544134455F8047F17B10F602968043188
:10BB40009D42F7D100230B60F3B283F311882823C1
:10BB500003FB0020036A23B1A3899BB243F00103D6
:10BB600004E0A38923F001031B041B0CA381BDE89F
:10BB7000F88300BF702500200048FDE50C18002068
:10BB80000048F9E5601800200048F5E5B4180020E9
:10BB90000B4B4FF400525A604FF6FE730948D0F831
:10BBA000DC2011680B401360D0F8CC20D0F8D030E6
:10BBB0009A4201D0A83056E6012380F8EC30704755
:10BBC000000002400C1800202DE9F0431D46AC4B4C
:10BBD0008DB09842884617469DF8506060D1A94BB9
:10BBE000A94AAA49C3F8A82003F1FC02C3F8BC2063
:10BBF00003F5FE72C3F8C0204FF48072C3F8B4207E
:10BC0000C3F8B820A24AC3F8B070C3F8D820A2F590
:10BC10004842543AC3F8F420C3F8F02002F55742E2
:10BC2000FC32C3F8F800C3F8DC10936943F4804396
:10BC300043F004039361536943F00103536102230A
:10BC40008DF803304FF40073ADF80030330701D5A1
:10BC50001C230FE0AC0706D518238E4869468DF8E3
:10BC6000023006F0BCFFE8070AD54FF48063ADF858
:10BC700000304823874869468DF8023006F0AFFF50
:10BC80000E238DF804300022012301A88DF8053021
:10BC90008DF806208DF807307F4C08F0F9F8A5E004
:10BCA0007E4B984252D1774B774ADF655A654FF405
:10BCB00080721A665A6603F53F729A6603F57F72C0
:10BCC000DA66774AC3F8A400C3F89C20C3F8A02022
:10BCD000744B3107DA6942F40032DA619A6942F052
:10BCE00004029A619A6942F001029A614FF00203DC
:10BCF0008DF803304FF00403ADF8003001D51C235C
:10BD00000EE0AA0706D51823624869468DF802306E
:10BD100006F065FFEB0709D50823ADF8003048238E
:10BD20005C4869468DF8023006F059FF26238DF8ED
:10BD300004300022012301A88DF805308DF806207B
:10BD40008DF80730584C08F0A3F84FE0574B984255
:10BD500040F0F5804B4B4C4A9F601A6003F2FC4266
:10BD60005A6103F2FC529A614FF48072DA601A61F0
:10BD70004F4A18659A64DA644A4B3407DA6942F428
:10BD80008022DA619A6942F008029A614FF0020358
:10BD90008DF803304FF48063ADF8003001D51C23DB
:10BDA0000FE0A80706D51823424869468DF80230EF
:10BDB00006F015FFE9070AD54FF40063ADF800302F
:10BDC00048233C4869468DF8023006F008FF2723D7
:10BDD0008DF804300022012301A88DF805308DF87C
:10BDE00006208DF8073008F053F8264C4FF0000974
:10BDF000012384F84430C4F82090C4F81C90C4F89F
:10BE00002890C4F82490C4F82C806571A760A671AE
:10BE1000204605F04DFAEA0756D5236B002B4BD090
:10BE200001A808F0C9FAE36C206B01934FF480532A
:10BE30000A9380230693E368CDF82C900493202383
:10BE400009936369CDF814900293CDF81C90CDF856
:10BE50002090CDF80C9008F0DAFA01A9206B08F0D8
:10BE6000B8FA226B216D136843F0010313608B8ACB
:10BE70009BB243F040038B8253689BB2236423E060
:10BE8000003801400C1800202CB301084400024087
:10BE90005800024000080140B4180020004400404F
:10BEA0000444004000100240601800200048004098
:10BEB00004480040000C01404FF6DF72236D1A80E9
:10BEC000DA6842F02002DA60AB0730D5636B002BF2
:10BED00028D001A808F070FAA36C002501934FF454
:10BEE00080530A93802306932369606B0493102385
:10BEF00003930B95059507950895099508F087FA22
:10BF0000606B01A908F065FA636B1A6842F00202DF
:10BF10001A60226D5D605D60938A9BB243F080037E
:10BF2000938204E0226DD36843F08003D360226DD6
:10BF3000204693899BB243F40053938100E0002094
:10BF40000DB0BDE8F08300BF08B50848FCF782FEDD
:10BF5000FCF7DCF906F0CCFF18B9642003F0D7F940
:10BF6000F8E70348BDE80840FCF774BEA9D501080E
:10BF7000B6D501082DE9FF410A480688856844883E
:10BF8000B0F80480C768FCF7B9F8CDF800800290DB
:10BF90000197054831462A462346FCF75BFE04B06C
:10BFA000BDE8F0811C000020BED50108F0B5047882
:10BFB0008BB005460CB1002430E0464B19680E23C7
:10BFC00003FB0411B1F90400B1F90020B1F902300A
:10BFD0000090C8790190087A029091F906000390C8
:10BFE00091F909103C48049121460134FCF732FED6
:10BFF000082CE2D16BE02D2B14D1072C1BDC28463A
:10C000000CF0BCFF0AAB661C03EB440424F8100CD4
:10C0100015F8013F303B092BFAD934462B78002B19
:10C02000E9D104E0A3F13002092A09D8E5E7082C98
:10C03000BDF8182009D00BB0BDE8F04001F076BD86
:10C04000202BF8D101352646E7E7072AF3D840F23E
:10C05000DC55204BBDF81A001C68A0F2EE239BB201
:10C06000AB42E8D8BDF81C10A1F2EE239BB2AB4264
:10C07000E1D8BDF81EE003B20FFA8EF69E42DADB7D
:10C080000DB2AE42D7DC9D42D5DBBDF8246006F18F
:10C0900064039BB2C82BCED8BDF826502BB2112B0F
:10C0A000C9DCBDF820C0BCF1B40FC4D8BDF8227003
:10C0B000B42FC0D80E2312B25A43A318A0525980ED
:10C0C000A3F804E083F807C01F729E715D720BB085
:10C0D000F0BD00BF081F00201BD601087FB5047803
:10C0E000E4B92B4E062303FB046600252A46735D44
:10C0F000284821460135FCF7ADFD062DF6D1013467
:10C10000062CEED10024244B22461B5D214806213B
:10C110000134FCF79FFD082CF5D136E01F490CF0E7
:10C120003DFF002460B1032C10D00CF027FF01ABC1
:10C1300043F82400194900200CF030FF0134F1E7E6
:10C14000032C03D101A90EC90F2B04D904B0BDE8FB
:10C15000704001F0EBBCC8B2052808D8052AF5D814
:10C160000F4C062505FB00401044037107E006282C
:10C17000ECD1072AEAD80A48104480F8283005484C
:10C1800004B0BDE87040FCF765BD04B070BD00BFF1
:10C190000C1F00203BD60108301F0020C0D601082C
:10C1A000081F0020F0B504468FB020460CF091FE29
:10C1B000C5B20DBBA74806F0F1F8A74C217809B924
:10C1C000A6484EE049B214F8022C14F8013C009144
:10C1D0006178A348019194F902100734029114F98F
:10C1E000041C039114F8031C049129460135FCF743
:10C1F00031FD102DE2D1E3E720469A4905220CF0EB
:10C2000071FE054698B92946974870220CF01DFE2C
:10C210002846964B19680E2303FB001301300022B9
:10C2200008289A72DA721A735A73F4D10FE1204611
:10C230008F4904220CF056FE05462046002D45D1BC
:10C2400020210CF038FE002800F00181461C304609
:10C250000CF03FFE2C460746864B53F824502DB970
:10C2600085480FB0BDE8F040FCF7F4BC30462946E5
:10C27000FAB20CF037FE01340028EDD17F4A02F10A
:10C2800070010023137002F8043C02F8053C02F828
:10C29000063C07328A42F4D1794A12F834108B42B4
:10C2A0000FDA02EBC4025268C3EBC3010A441768F9
:10C2B0006D4E01338F5188199188818092798271F6
:10C2C000EAE770482946FCF7C5FC91E06E49072271
:10C2D0000CF008FE05462046002D49D120210CF027
:10C2E000EAFD06460CF0F5FDC4B26CBB6748FCF7EE
:10C2F000B1FC214666480134FCF7ACFC0E2CF8D1A9
:10C300005648FCF7A7FC002462482146FCF7A2FC33
:10C310000025564A012311680E2202FB0412D2F8AE
:10C320000A20AB4013425C4B5C495D4808BF19468C
:10C330000135FCF78FFC0E2DEBD148480134FCF79A
:10C3400089FC082CE0D182E0304656490CF026FEEC
:10C350002C4600284ED0022C51D00CF00FFE06AB1C
:10C3600043F824004F4900200CF018FE0134F0E798
:10C370004C490CF013FE002460B1082C3AD00CF0AC
:10C38000FDFD06AB43F82400464900200CF006FEF4
:10C390000134F1E7082C2DD1069B0F2B2AD8DDF8AC
:10C3A0001CC0BCF1070F25D8089F0D2F22D8099E6D
:10C3B00006F16402C82A1DD80A9DFF2D1AD80B98D1
:10C3C000642817D80C99642914D8884212DA0D9C75
:10C3D000032C0FD8DFF890E0C3EBC3020EEB02038F
:10C3E0000EF802C05F709E70DD70187159719C71FB
:10C3F0002D4CDAE60FB0BDE8F04001F097BB069B8C
:10C40000072B20D807990D291DD80278722A0DD044
:10C410006E2A18D1154A0E20126800FB0323012250
:10C420008A40D3F80A1021EA020209E00F4A0E20DE
:10C43000126800FB032301228A40D3F80A100A4342
:10C44000C3F80A2001E001F071FB0F4CADE60FB01C
:10C45000F0BD00BF59D601085A32002062C9010858
:10C4600084D60108A0D6010858320020081F0020F9
:10C47000A6D60108ECBD010841C901085E320020C2
:10C4800054B30108ABD6010851D601088DDB010871
:10C49000B7D6010852D901083ACD010880CC01086D
:10C4A000BCD60108C0D601088BC40108F7B50478D2
:10C4B000054684B92C4D2E46E97836F82420AB7811
:10C4C0002A48009121460134FCF7C4FB102C05F1E9
:10C4D0000405F1D145E00CF051FD0F28064638DC8B
:10C4E000284620210CF0E7FC70B3441C00252046B0
:10C4F0000CF044FD1E4BB70033F8153098421DDC9C
:10C500001C4B012D3B4403D0022D04D0188604E0BF
:10C5100083F8320001E083F8330020462C210CF030
:10C52000CAFC044610B10134012302E0AA1E5342A2
:10C530005341013513B1032DD9D112E00A4A00232A
:10C54000174422F826307B8003B0BDE8F04001F0AC
:10C55000EDBA094800210F2203B0BDE8F04001F018
:10C5600068BA03B0F0BD00BF381F0020C2D6010872
:10C5700024B40108081F0020D6D601082DE9F04791
:10C5800004788EB00546002C48D16D4D2E461422FD
:10C5900009A800210CF059FC06AA17466888062352
:10C5A00040FA03F1C90742BF6649C91811F8061CD1
:10C5B00003F1010344BF11700132102BF0D10023AD
:10C5C000137004AA114640FA03FE1EF0010F1CBFAF
:10C5D000DFF880E113F80EE003F101031CBF82F8DD
:10C5E00000E00132062BEED10023137016F8243040
:10C5F0008DE882006A785449029209A81A0903F06A
:10C600000F0300F01CFF2146504809AA0134FCF733
:10C6100021FB202C05F10405B9D18DE00CF0AEFC16
:10C620001F28074600F38380284620210CF043FC96
:10C63000002879D0424B0024BE0023F82740A246B0
:10C64000A0462746A1469A19451C5480404BE2B2A9
:10C6500014F803E00023284615F8011B39B1714591
:10C6600005D00A2B03D009A819540133F3E70EAD06
:10C670002B4471454FF0000503F8145C54D1531E50
:10C68000451C032B09D8DFE803F00D0502350DF139
:10C6900023012AE00DF1230115E009A80CF06EFC3E
:10C6A00081462FE009A80CF069FC07462AE0013317
:10C6B000062B08D02748185C9042F8D1012202FAD4
:10C6C00003F34AEA030A11F8012FDAB10023F1E774
:10C6D00001330A2B09D01B48185C9042F8D106336D
:10C6E000012202FA03F34AEA030A11F8012F4AB1C0
:10C6F0000023F0E709A80CF041FC0F28D4BF8046C6
:10C700004FF000080134052CA0D1134B07F00F07A0
:10C710001E4447EA091986F8709086F87180A6F8D9
:10C7200072A003F08BFF07E001F000FA04E00B4871
:10C7300000211F2201F07DF90EB0BDE8F08700BF97
:10C74000781F00202AB40108DCD60108EBD60108C6
:10C750003AB4010834B40108081F0020D6D60108F5
:10C76000F8B5047806466CB9284B214603EB8405DE
:10C7700033F8242026486B880134FCF76BFA042C2C
:10C78000F2D1F8BD23490CF069FB20B9BDE8F840AF
:10C79000214801F01CB830460CF0F0FB0328054698
:10C7A0002CD8304620210CF086FB044630B10134F1
:10C7B00020460CF0E3FB0126074600E00646204633
:10C7C00020210CF078FB18B9BDE8F84001F0AEB9B3
:10C7D00001300CF0D3FB012EF6D140F2DC53A7F26E
:10C7E000EE229A42F0D8A0F2EE229A42ECD8074B01
:10C7F00023F8257003EB85035880F8BD0748002116
:10C800000322BDE8F84001F014B900BFFE15002076
:10C81000F7D60108A0D6010888E50108FCCA01087E
:10C820002DE9FF4104780546002C36D16D4805F00E
:10C83000B5FD6D4D55F8040C002109F067FE002888
:10C8400040F0CD8021466948FCF704FA55F8040C05
:10C85000694600F08FFC01466548FCF7FBF9286843
:10C86000694600F087FC01466148FCF7F3F9686807
:10C87000694600F07FFC01465D48FCF7EBF9A868CB
:10C88000694600F077FC013401465A48FCF7E2F9AA
:10C890000C2C05F11005CDD1A1E0574905220CF073
:10C8A00021FB30B9554B0022C2501030C028F9D1BD
:10C8B00095E02846524904220CF014FB0446284611
:10C8C000002C3FD120210CF0F6FA002800F08780E0
:10C8D000451C28460CF0FDFA07464A4B53F82460E5
:10C8E0001EB9494805F05AFD79E028463146FAB2AA
:10C8F0000CF0F8FA01340028EFD1404B0022C2506E
:10C900001030C0289E46F8D1404BE4001A19D2F8E6
:10C91000F0809C46B8F1000F04D13D483146FCF749
:10C9200099F953E000250CEB040393F8EC309D4299
:10C93000F3DA2B010EEB030743440FCB013587E8F5
:10C940000F00F0E70CF01AFB0B28064642DC2846E5
:10C9500020210CF0B0FA054640B10135284600F020
:10C9600073FB264A3301D050012400E004462846D8
:10C9700020210CF0A0FA054640B10135284600F010
:10C9800063FB1E4B013403EB06135860284620213D
:10C990000CF091FA054640B10135284600F054FBF1
:10C9A000164B013403EB06139860284620210CF047
:10C9B00082FA10B901F0BAF811E0013000F044FB3E
:10C9C0000E4B032C03EB0616F060F3D11148FFF772
:10C9D00027FF04E0104800210B2201F02AF804B0E0
:10C9E000BDE8F0810AD701089C31002025D7010855
:10C9F0002BD7010818DB0108A0D6010898310020C8
:10CA0000A6D60108ECBD010841C9010854B30108CC
:10CA1000ABD601088BC40108D6D60108F0B504785E
:10CA200087B00646F4B9062363434A4AD2F8F010A9
:10CA3000C8184578CB5C19214D4305F561754279DD
:10CA400000958578694301F561710191C178029182
:10CA500001794148039121460134FCF7FBF80C2C85
:10CA6000E1D175E00CF08AFA0B2804466BDC394BF7
:10CA7000701CD3F8F050202100238DF817300CF0F3
:10CA80001AFA064678B1013630460CF077FA0328D8
:10CA90009FBF062303FB045358719DF817309CBFBA
:10CAA00001338DF81730304620210CF004FA064689
:10CAB00070B1013630460CF061FA0D289FBF062395
:10CAC0006343E8549DF817309CBF01338DF817304D
:10CAD000062707FB04573046791C0DF1170200F0BA
:10CAE0007DFF20210CF0E7F9064658B101363046AB
:10CAF0000CF044FA26289FBF9DF81730F8700133D8
:10CB00008DF81730304620210CF0D5F970B1013086
:10CB10000CF034FA0D289FBF062303FB0453187151
:10CB20009DF817309CBF01338DF817309DF81730F2
:10CB3000062B0DD0062202FB045000210CF085F9D3
:10CB400000F0F4FF04E0054800210B2200F071FF23
:10CB500007B0F0BD081F00202FD70108D6D6010866
:10CB6000F8B50E4D06462F4600242B7903F030030E
:10CB7000B3420CD104EB0413F9580948FCF76AF8E6
:10CB800028460021FCF76AF9064805F007FC013445
:10CB9000A72C05F11105E8D1F8BD00BF9CA601083E
:10CBA0004FD7010862C90108164810B5046854B18E
:10CBB000154964220B685343B3FBF4F3134A138003
:10CBC000002303600B60002213461148016851B135
:10CBD0000C7C062C03D0096A8B4238BF0B4601320D
:10CBE00050F82210F3E70B49092B0A6005DDB3F575
:10CBF000967FA8BF4FF4967300E00A23064A1933C4
:10CC0000136010BDFC090020000A0020F815002068
:10CC1000B4090020F809002000000020F0B501242C
:10CC2000B0FBF4F58D4201D34C43F9E70026D4B1B3
:10CC3000B0FBF4F504FB1500B4FBF1F41EB9002DB4
:10CC400001DC002CF3D1092D03F1010EEFB204DD5C
:10CC5000002A14BF3725572500E030253D441D70BC
:10CC600001367346E3E71C70F0BDF0B50124B0FB5C
:10CC7000F4F58D4201D34C43F9E70026D4B1B0FB63
:10CC8000F4F504FB1500B4FBF1F41EB9002D01DC32
:10CC9000002CF3D1092D03F1010EEFB204DD002ABF
:10CCA00014BF3725572500E030253D441D7001365F
:10CCB0007346E3E71C70F0BD03685A1C02601970EC
:10CCC00070472DE9F843089E002B07468846144616
:10CCD000334614BF4FF030094FF0200913F8012BF1
:10CCE0000AB9254603E0002CFBDD013CF6E7002DE8
:10CCF00004DD38464946C047013DF8E7354624EA99
:10CD0000E474A01B284415F8011B11B13846C04734
:10CD1000F7E7BDE8F88303884888C3F30B02904225
:10CD200006D10A79B2EB133F0CBF012000207047F7
:10CD300000207047014B186802F05CBCB003002073
:10CD400030224243124B70B59D189A580A60114A1E
:10CD500014680022A24206DA0F4E56F82260AE4254
:10CD600003D00132F6E7002200E001220A713022EE
:10CD700002FB0030C3688B60037C0B73836A0B611A
:10CD8000C36A4B61036A8B61436ACB6170BD00BFAC
:10CD90006C000020F4090020B4090020194B2DE993
:10CDA000F0411C6880460E2C1F4627DC0023A3425E
:10CDB00006DA154A52F8232042451FD00133F6E720
:10CDC0000025A5421ADC104EA90056F82530681C33
:10CDD0006BB9621B06EB80003144920001340CF009
:10CDE00019F846F825803C600120BDE8F0811A7CE6
:10CDF00098F810309A42ECD30546E2E70020BDE8EF
:10CE0000F08100BFF4090020B4090020102870B59B
:10CE100002D00E2803D970BD144B186803E0144BE0
:10CE2000302202FB003009B1836823B9114B002284
:10CE30001C681D4603E0BDE87040AFE70A46A24209
:10CE400012DA0D4B53F8221003EB8206814202F1F5
:10CE50000101F3D1A21A304603EB81019200013C9B
:10CE60000BF0D8FF2C6070BD70BD00BF34270020D0
:10CE70006C000020F4090020B4090020036810B5FC
:10CE80005A1C02601A4612F8024BD91C02605A78EA
:10CE900001609978090441EA0222191D0160D878DD
:10CEA000224342EA006010BD03685A1C02601A4621
:10CEB00012F8021B0260587841EA0020704738B52A
:10CEC0000446154600680CF05DF823681D44256093
:10CED00038BD03685A1C0260197003685A1C02604E
:10CEE0000A0A1A7003685A1C02600A0C1A70036856
:10CEF000090E5A1C02601970704703685A1C0260C0
:10CF000019700368090A5A1C0260197070472DE9EC
:10CF1000F0410C464E69CD690968074609F062F98F
:10CF200061688046304609F05DF90146404609F0E7
:10CF300051F8A1698046A06809F054F901464046BD
:10CF400009F048F8E1688046284609F04BF90146A7
:10CF5000404609F03DF8216A8046206909F042F90F
:10CF60000146404609F034F8A66167612562E06138
:10CF7000BDE8F0812DE9F8430C463049164609F02A
:10CF800031F90546304609F0D5F82D4909F02AF95E
:10CF900001464FF07E5009F0D9F90146284609F0C4
:10CFA000D5F9064600F02EFB0546304600F09EFB04
:10CFB00024490746304609F015F9294609F0C6F913
:10CFC00000F020FB0146284609F00CF939460646D8
:10CFD0004FF07E5008F0FCFF4FF07E518146304606
:10CFE00008F0F8FF05464FF07C51484609F0FAF882
:10CFF000294609F0ABF9294680462060484609F0E9
:10D00000A5F94FF040416060C4F80880384609F047
:10D01000E9F8294609F09AF93146E0604FF07E5070
:10D0200008F0D6FF294609F091F900232061A36199
:10D0300063612362E361BDE8F88300BFDB0FC94091
:10D04000BD378635CA92283F2DE9F0410278034664
:10D05000202A00F10100F9D0092AF7D02D2A02D1A7
:10D060000346414D04E02B2A08BF03464FF07E558E
:10D070001C460026234614F8012BA2F13007F9B212
:10D0800009290DD83949304609F0ACF8064638462A
:10D0900009F054F80146304608F09CFF0646E9E7DF
:10D0A0002E2A17D1314F234614F8010B3038C2B263
:10D0B000092A0FD809F042F8394609F047F9014624
:10D0C000304608F087FF29490646384609F08AF8B5
:10D0D0000746E8E71A7802F0DF02452A39D15A7884
:10D0E0002D2A02D10233012704E02B2A14BF013379
:10D0F00002330027013B002413F8012F303AD1B24C
:10D10000092903D80A2101FB0424F5E7B4F59A7F25
:10D1100028BF4FF49A74A0464FF07E53B8F1070F22
:10D1200007D91846124909F05DF8A8F10808034626
:10D13000F4E704F0070434B118460C4909F052F83A
:10D14000013C0346F7E719462FB1304609F0FEF8D7
:10D1500004E04FF07E51304609F044F8014628467D
:10D1600009F040F8BDE8F081000080BF00002041D8
:10D1700020BCBE4C30B5054687B00C4603A8002144
:10D180000C220BF062FE2846002109F0E7F920B1DD
:10D190002846284908F01EFF03E02846254908F0E4
:10D1A00017FF254909F01EF809F0E2F9054680EA63
:10D1B000E0706946A0EBE57007F06CF8002DACBF9D
:10D1C00020232D2368468DF80C300BF082FE0128B9
:10D1D00007D130238DF80D308DF80E308DF80F30DB
:10D1E0000CE0022805D130238DF80D308DF80E307B
:10D1F00004E0032804BF30238DF80D30694603A8EE
:10D200000BF04AFE03A80BF064FE0338C5B22A46B1
:10D2100003A920460BF088FE0023635520460749EA
:10D220000BF03AFE03AB204659190BF035FE2046B1
:10D2300007B030BD6F12033A00007A4459D7010895
:10D2400070B50646B6FBF2F40846154614B1204602
:10D25000FFF7F6FF05FB1464024B1B5D00F8013B72
:10D2600070BD00BF5BD701082DE9F04F81468A46AB
:10D2700016461C4689B000253178002900F0DB8075
:10D28000252902D00136484674E072784FF0000834
:10D29000302A0CBFB278B71CA2F1300312BF4FF096
:10D2A000000BF71C4FF0010B092B19D8A2F130032A
:10D2B000D9B2092905D80A2202FB083817F8012B30
:10D2C000F4E7A2F16103052B02D8A2F1570305E0B0
:10D2D000A2F14103052B03D8A2F137030A2BEADDA3
:10D2E0006C2A30D13A787E1C642A00F083800BD8F7
:10D2F000252A3DD003D8002A00F09D80BCE7582A9B
:10D300000CD0632A19D0B7E7732A22D002D86E2A2C
:10D3100037D0B1E7752A5CD0782AADD1271D2068B7
:10D32000A2F1580462424FF01001624155E02CD93D
:10D33000582A32D0632A2AD13E4648462178271DF2
:10D34000D04701350FE0642A63D00ED9732A14D177
:10D350003E46236848460093514642460023FFF765
:10D36000B0FC271D05443C4686E7252ADFD13E4612
:10D3700048462521D04701357EE70AD86E2A06D1D6
:10D380003E46236804341D6076E7002A53D03E46AB
:10D3900072E7752A26D0782AF9D1A2F1580304F150
:10D3A000040C5A422068CDF80CC04FF010015A41CD
:10D3B00005ABFFF733FCDDF80CC03E46644605AB19
:10D3C00000934846514642465B46FFF77AFC0544C7
:10D3D00052E72068271D0A21002205ABFFF745FC14
:10D3E0003C46ECE704F1040CCDF80CC020680A219F
:10D3F0000022DDE72068271D002808DA2D238DF89C
:10D40000143040420DF115030A210022E6E705AB76
:10D41000FAE7206804F1040C00280ADA2D238DF8BD
:10D42000143040420DF11503CDF80CC00A21002242
:10D43000BFE705ABF8E7284609B0BDE8F08F0EB4AA
:10D440000FB505AB53F8042B0190064901A80393CF
:10D45000FFF70AFF019B00221A7004B05DF804EB8D
:10D4600003B07047B9CC000880EAE073A3EBE07327
:10D470008B4206DB002801DD401A704702D00844C9
:10D4800070470020704770B520F0004421460546E3
:10D490004FF07E5008F09CFD0CF0B6F8134906469C
:10D4A000204608F09FFE124908F094FD01462046F0
:10D4B00008F098FE0F4908F08BFD0146204608F061
:10D4C00091FE0D4908F086FD0146304608F08AFEBF
:10D4D00000210446284609F023F820B121460748D8
:10D4E00008F076FD70BD204670BD00BF306E99BC5F
:10D4F0002716983D8434593EA40DC93FDB0F49409F
:10D500002DE9F84321F0004520F000460746884603
:10D510002846314609F022F808B9344600E02C4686
:10D520002046002108F0F2FF60B92846314608F095
:10D53000F7FF08B9304600E02846214608F006FF0C
:10D54000044600E000242046254908F04BFE25490A
:10D5500008F03EFD214608F045FE234908F038FD5D
:10D56000214608F03FFE214908F032FD214608F02F
:10D5700039FE1F4908F02CFD1E4900F100492046E4
:10D5800008F030FE1C4908F025FD214608F02AFE6F
:10D590004FF07E5108F01EFD0146484608F0D6FEC9
:10D5A00029460446304608F0D9FF20B121461348E9
:10D5B00008F00EFD04464046002108F0B1FF20B1FE
:10D5C00021460F4808F004FD04463846002108F0C3
:10D5D000A7FF08B104F100442046BDE8F88300BF6E
:10D5E00039094E3DE3B59E3E88FA163E45FE7F3F23
:10D5F000A7DFA83499FB243F69A2163EDB0FC93F81
:10D60000DB0F494070B5044608F0B2FF20304028D7
:10D6100057D820462C4908F0A1FF28B120462B49B5
:10D6200008F0D6FC0446F4E72046294908F078FFC4
:10D6300028B12046254908F0CDFC0446F4E72046F1
:10D64000244908F08BFF30B12249204608F0C0FC85
:10D65000014620480AE020461F4908F061FF40B11A
:10D660001C49204608F0B6FC01461B4808F0B0FCF7
:10D6700004462146204608F0B5FD054620462946C9
:10D6800008F0B0FD15490646284608F0ABFD1449E0
:10D6900008F09EFC0146284608F0A4FD114908F058
:10D6A00099FC0146284608F09DFD0F4908F090FCC2
:10D6B0000146304608F096FD0146204608F08AFCF7
:10D6C00070BD002070BD00BFDB0F4940DB0FC940BB
:10D6D000DB0F49C0DB0FC93FDB0FC9BF9A7C2E3679
:10D6E000FAAF4F393587083CA4AA2A3E08B503494A
:10D6F00008F070FCBDE80840FFF784BFDB0FC93FAE
:10D70000024A136823EA000010607047603100206D
:10D7100010B50A4B0A4A93420ED25A8810331104AC
:10D7200041BF53F80C4CC2F30B0200FB024253F80A
:10D73000081C48BF0A60EDE710BD00BF98E401086F
:10D7400078E7010870B5064644880D46C4F30B041B
:10D750000846224600210BF078FBF368094A934201
:10D7600009D3094A934206D228462246BDE87040B2
:10D7700019460BF007BC23B128462146BDE870408E
:10D78000184770BD78E701084AE80108F8B5044673
:10D7900015461F460E4640886168020444BFC0F328
:10D7A0000B0003FB00112046FFF7CCFF6388606885
:10D7B000C3F30B018D422A46A8BF0A461B0448BF8B
:10D7C00007FB01003146BDE8F8400BF0DBBB034628
:10D7D000B0F90220002AB6BF836841681968B1E732
:10D7E00070B505460E46074C074B9C4205D22046B5
:10D7F0003146A84718B91034F6E7002070BD20461E
:10D8000070BD00BF98E4010878E7010870B50646CE
:10D810001B4C14F8015B23882BB31A49E2188A4287
:10D820002CD2052B2AD92346934203D013F8011B8F
:10D830004D40F9E7A6B114482146FFF7D1FF78B172
:10D84000B0F90230A11D002BB7BF6379002303F0AC
:10D85000030303F1FF33B8BFDBB22288FFF796FF63
:10D8600023881C44D7E722786378A07853406B4024
:10D87000DB43DBB2C31A5842584170BD002070BD73
:10D8800000F001080000020817CD0008F8B50446B2
:10D890000E4617460D46F3199D4210D0E368591CF9
:10D8A000E16015F8012B234404291A72F3D12046B4
:10D8B000A168FCF7E9FE00232061E360EBE7206943
:10D8C000F8BD00BF2DE9F04101F0FAFC054600F17A
:10D8D000FA08234C26783601A3195A685B899268A6
:10D8E0001A420DD001F0ECFCC8EB00000028F0DD7E
:10D8F000FF2031E001F0E4FCC8EB00000028F7DC79
:10D90000A3195A685B899268154F1A42F2D001F048
:10D91000D7FCD7F8C830401B9842C7F8C4001AD8C3
:10D9200005F5FA75A3195A685B8992681A420AD0FC
:10D9300001F0C6FC401B0028F4DDD9E701F0C0FC73
:10D94000401B0028D4DCA3195A685B8992681A42EC
:10D95000F4D0002000E0012040B2BDE8F08100BF1B
:10D960002422002038B500252C46FFF7ABFF002805
:10D970000DDBA84001350443082DE4B2F5D1054A7A
:10D98000204692F8CC30634082F8CC3038BD4FF05E
:10D99000FF3038BD2422002038B5800040F4806478
:10D9A00001F08EFC054644F001040B4B14F0010F0E
:10D9B0001A7805F1340503EB02135A685B8914BF2A
:10D9C00013615361640805D001F07AFC401B002804
:10D9D000FADBEAE738BD00BF24220020F8B5044690
:10D9E0000E4617460025204620210BF064FA044617
:10D9F000D0B1013420460BF0C1FAB0F5617F05DBF0
:10DA000040F634039842A8BF184601E04FF4617015
:10DA1000A0F56170192390FBF3F00DB9307000E0B0
:10DA200070703B7801333B700DB90125DBE7204670
:10DA3000F8BD30B505460C46134629462246BDE8DA
:10DA400030400148FBF706B980D701087FB504785C
:10DA50000546D4B9324B1921D3F8D03003EB8405F5
:10DA6000A87813F82420484300F561706B78009083
:10DA7000E878414301F5617101912A48214601345A
:10DA8000FBF7E8F8142CE5D148E00BF077FA1328FF
:10DA900004463EDC224B681CD3F8D06020210023D2
:10DAA0008DF80F300BF007FA054660B101352846B6
:10DAB0000BF064FA1B289FBF06F824009DF80F3076
:10DAC00001338DF80F30284620210BF0F4F9A40023
:10DAD000054668B1013528460BF050FA0D289FBF66
:10DAE000331958709DF80F30013398BF8DF80F30FF
:10DAF00034442846A11C0DF10F02FFF76FFF9DF87B
:10DB00000F30042B0AD02046002104220BF09DF98F
:10DB100004E0054800211322FFF78BFF04B070BD1D
:10DB2000242200209FD70108D6D60108014804F01E
:10DB300035BC00BFB4D70108F0B5027887B04B4CB4
:10DB40007AB904F12806A2780023494950B25956FF
:10DB5000814273D00C333C2BF7D10834B442F2D15C
:10DB600081E0002504950595471C0BF007FA2B462C
:10DB7000C0B204EBC306B278904204D18DF8100015
:10DB80000236012404E00133052BF2D1002634468D
:10DB9000384620210BF08FF9054638B1013528466B
:10DBA0000BF0ECF90134ADF81200E4B2002728467E
:10DBB00020210BF080F9B0B3451C28460BF0DEF9AC
:10DBC00000222C495FFA82FE51F82230834204D0B1
:10DBD0000132082AF5D1002300E0734651F82320D2
:10DBE000824220D1022F0FD0032F12D05A1E012FB4
:10DBF000D2B204D0042A13D88DF814300EE0042ACF
:10DC00000ED88DF8153009E0052B09D88DF817309E
:10DC100004E09A1E052A03D88DF816300134E4B2C8
:10DC20000137042FC3D1052C03D807B0BDE8F0405D
:10DC30007CE704AB03CB3060716014E0E0790D4BFE
:10DC4000A57953F82000A2880090607A53F820004C
:10DC50000190207A53F8200053F8253002900648AE
:10DC6000FAF7F8FF79E707B0F0BD00BF9A36002059
:10DC7000C436002034A50108C2D701082DE9F743B6
:10DC8000047806464CB9204601A906F003FB01348E
:10DC9000FFF7F4FF122CF6D16DE00BF06FF9C4B270
:10DCA000112C63D8701C20210BF005F9334D03466D
:10DCB00015F81470324E18B9BA1E574257413FE05A
:10DCC00000F10109597830460BF0F5F860B1032CEA
:10DCD0008CBF03230023801BC0B23344184490F848
:10DCE0000480B8F1030F02D1FFF720FF43E0A8F151
:10DCF00002035F4248464FF020015F410BF0DBF822
:10DD0000D0B1002FF0D001300BF038F940F2ED2304
:10DD100080B2984205DD40F6CA039842A8BF184673
:10DD200001E040F2EE20A0F2EE20192290FBF2F08A
:10DD300005EB4403587001E0002FD5D105F814809D
:10DD400015F81430F25C67B10C4B0E4803EB44033A
:10DD5000597819234B43214603F2EE23FAF77AFF51
:10DD600009E009482146FAF775FF04E00748002159
:10DD70001122FFF75EFE03B0BDE8F083EC14002033
:10DD80008DBA0108E1D70108F3D70108FCCA0108E0
:10DD900008B5044804F002FB034B1868BDE80840CE
:10DDA00001F062BA02D80108F41500202DE9F84309
:10DDB000364C602394F8D4708046152F8946C4F8F9
:10DDC000C83006D0122F04D0012F0CBF02258C259D
:10DDD00001E044F62065FFF775FD002802DA013DF9
:10DDE000F9D14FE00A25FFF76DFD00284ADB013D20
:10DDF000F9D1D4F8C420530803EB9203C4F8C83017
:10DE0000FFF760FD00283DDBFAD184F8CC00FFF776
:10DE1000A9FD1B2836D1FFF7A5FD002832DB1B4BDF
:10DE200093F8D53098422DD1FFF79CFD0602FFF7FD
:10DE300099FD0643731EB3F5817F23D8FFF792FD4A
:10DE40000E281FD1FFF78EFD00281BDBB84219D129
:10DE5000FFF788FDB0B90025B31E9D4209DAFFF730
:10DE600081FD00280EDB4D45B8BF08F805000135DF
:10DE7000F2E7FFF777FD94F8CC00B0FA80F04009A4
:10DE8000BDE8F8830020BDE8F88300BF242200200D
:10DE90002DE9F04180461C4C082694F8D6304340CA
:10DEA00084F8D630257818F0010F04EB05156B685F
:10DEB0006A891A6107D0402001F01EFA6B686A89EE
:10DEC00040205A6115E0202001F016FA2378202026
:10DED00004EB03135A685B89536101F00DFA6B6818
:10DEE0006A8920201A6101F007FA6B686A8920208C
:10DEF0005A61013E01F000FA16F0FF064FEA580899
:10DF0000D0D1BDE8F08100BF2422002070B50A4DB9
:10DF100095F8D600FFF7BCFF2B7820201C012E19A6
:10DF2000736872891A6101F0E7F9314670680C3143
:10DF3000BDE8704004F053BE2422002038B5154CD3
:10DF4000054621780901631819465868103104F014
:10DF500046FEFF20FFF79CFFFF20FFF799FF7F2081
:10DF6000FFF796FF00231B2084F8D630FFF790FFC1
:10DF700094F8D5000130C0B284F8D500FFF788FFCF
:10DF8000280AFFF785FFE8B2FFF782FFBDE83840B7
:10DF90000E207DE7242200204FF6FF73028870B523
:10DFA0009A4204461ED0104D0626052085F8D460FE
:10DFB000FFF7C4FF3046FFF76BFF0020FFF768FF55
:10DFC0000020FFF765FF2088000AFFF761FF207837
:10DFD000FFF75EFFFFF79AFF05F1D7001021BDE8BC
:10DFE0007040E3E6012070BD2422002038B50124F2
:10DFF000084D204685F8D440FFF7A0FF2046FFF7E4
:10E0000047FFFFF783FF05F1D7001021BDE8384037
:10E01000CCE600BF2422002038B504460088002545
:10E020000A3080B2FFF78AFF184B93F8D400FFF74D
:10E030002FFF2088000AFFF72BFF2078FFF728FF2B
:10E040000020FFF725FF0020FFF722FF0020FFF749
:10E050001FFF0020FFF71CFF0020FFF719FF002023
:10E06000FFF716FF0020FFF713FF23889D4205DA14
:10E070006368585DFFF70CFF0135F6E7FFF746FFD1
:10E08000BDE838400248102190E600BF242200205D
:10E09000FB22002010B504460420FFF74FFF0B4B76
:10E0A00093F8D400FFF7F4FE2088000AFFF7F0FE93
:10E0B0002078FFF7EDFEA020FFF7EAFEFFF726FF2E
:10E0C00060682188BDE8104070E600BF242200206F
:10E0D000082380EA010212F0010F4FEA50001ABF34
:10E0E00080F4204080F0010080B2013B4FEA5101F2
:10E0F000EFD170472DE9F74F8146194F8B463C7899
:10E1000007F1040824013B1908EB040158680C319D
:10E1100001924E4604F063FD0025C9EB06035B4502
:10E120000BDAB24616F8010BFFF736FC28469AF8D0
:10E130000010FFF7CDFF0546EFE7019B33B1E8B2D2
:10E14000FFF72AFCC5F30720FFF726FC274404F15C
:10E1500008017868414403B0BDE8F04F04F03FBDCA
:10E16000242200202DE9F04101F0AAF800F5FA651B
:10E170001A4F3E783601BA19536854899B681C407F
:10E1800007D001F09DF8A842F2D34FF0FF30BDE870
:10E19000F08101F095F8254600F11B0801F090F898
:10E1A000C8EB00000028F9DBBB195A685B8992684C
:10E1B00008F134081A421EBF0120A040054304F1B3
:10E1C000010418BFADB20A2CE8D140F201232B4064
:10E1D000B3F5007FD9D16808BDE8F0812422002082
:10E1E00010B50446FFF7BEFF002803DA013CF9D55D
:10E1F000FF2010BDC0B210BD4FF6FF73984207B5A7
:10E2000017D0FF238DF8043000238DF805308DF8EA
:10E210000700030A042101A801228DF80630FFF748
:10E2200069FF0220FFF7DCFFA0F13003584258419C
:10E2300000E0012003B05DF804FB2DE9F341054641
:10E2400048880C46FFF7D8FF00283ED0278801A851
:10E25000022101228DF804508DF80570FFF74AFF66
:10E26000D4F8048000254646C8EB0603BB420EDA0C
:10E27000FFF778FF002801DAFF2022E0C4B2214630
:10E28000A8B2FFF725FF06F8014B0546ECE7FFF7BC
:10E2900069FF011EF0DBC9B2A8B2FFF719FF0446FF
:10E2A000FFF760FF011EE7DB2046C9B2FFF710FF52
:10E2B0000446FFF757FF0028DEDB0CB9C0B200E0D0
:10E2C000C220A0F130035842584102B0BDE8F081AD
:10E2D000F7B5074648880D461646FFF78DFF08B983
:10E2E00000202FE02C88FE238DF8043000238DF8C9
:10E2F000053001A8230A042101228DF806308DF88B
:10E300000740FFF7F7FE0220FFF76AFFFF28E7D17B
:10E31000686821460122FFF7EDFE2820FFF760FF25
:10E320003028DDD1012201A802218DF805208DF8C9
:10E330000470FFF7DFFE3046FFF752FFA0F1300315
:10E340005842584103B0F0BD0023044A52F823203C
:10E3500040F8232001330E2BF7D17047ECC301089E
:10E3600030B5184A58B113780133DBB2132B88BF8C
:10E37000002313700B6803F5C333A0330B601378CD
:10E38000D90704D4032B8CBF0023012300E0002312
:10E390000D4C00205178884212DAB4F9021000299D
:10E3A0000BDA0A490BB1657801E0094D2D7901EBD3
:10E3B00085010D68074941F8205001300434E9E730
:10E3C00030BD00BFFC230020781F0020381F002034
:10E3D000301F00201239002070B5274CF0B1A3780F
:10E3E00003B9E378013BDBB2A370244B1B785B07D6
:10E3F00043BF234B5A22B3F906300A2341BFA3F58A
:10E400007A7353434FF47A7293FBF2F31D4A48BF79
:10E410000A3392FBF3F30A6813440B6000210846A9
:10E42000194D6378144A994225DA6B881E051FD569
:10E43000124B1B785B070BD59378D678034493FB7C
:10E44000F6F206FB1233012BCCBF0023012303E0BD
:10E4500000F0010383F0010323B16A780B4B03EB57
:10E46000820300E00A4B1A680A4B013043F821206E
:10E4700001310435D5E770BDFC230020DB3A0020D4
:10E480000034002080841E00781F0020381F0020E8
:10E49000ECC301081239002030B5224B224CA0B148
:10E4A0001A790AB1013A09E05879257885428BBF7B
:10E4B00001305A715871042288BF01221A710A680A
:10E4C00002F5C32202F520720A6021781748184A23
:10E4D00019B1184909688D0601D441790FE01979FD
:10E4E000154CB1FA81F124784909A40704D509B182
:10E4F000C17904E0C17802E00029EED0817902EB15
:10E5000081020021587881420BDA0C4800EB81002F
:10E510004088800442BF1468094840F82140013116
:10E52000F0E730BDFC230020F80F0020301F002052
:10E53000381F00208C170020882F0020781F002013
:10E540001239002008B509480AF0C3FCC0B20928F6
:10E550000246074905DC431CD8B20A4420239371C4
:10E56000F5E708440023837108BD00BF02240020A2
:10E57000FC23002008B508480AF0ABFCC0B2142800
:10E58000064B05D8421C184420238371D0B2F6E70D
:10E5900018440023837108BD02240020FC230020BE
:10E5A000014908220AF0EEBC98BA01080149242268
:10E5B0000AF0E8BCA0BA01082DE9F0412E4D2F4E1B
:10E5C00020B32F4B08681B782BB900F5433303F5B4
:10E5D000A0730B601AE0B5F90030B5F90220002BEA
:10E5E000B8BF5B42002AB8BF52429342B8BF13463D
:10E5F0001933322B234AB8BF322392FBF3F303447F
:10E600000B60337FB3FA83F35B0933771E4B96F8C5
:10E610001C80A3F10C02B8F1000F14BF984690467D
:10E62000B5F90030192B04DC1A33CCBF0024C02408
:10E6300000E03024B5F90230192B02DD44F050041B
:10E6400003E01933B8BF44F0A004002573789D425D
:10E6500010DA0E4BAF003B445B885B0608D52846BA
:10E6600001F03CFF20421EBFD8F80020084BFA50B2
:10E670000135EBE7BDE8F081642F0020FC2300208A
:10E68000040E002080969800F8C30108781F00202F
:10E6900012390020022803D0431E584258417047C7
:10E6A000064B1B7823B1064B1868C0F3C040704777
:10E6B000044B1878C0F38000704700BF940F00200F
:10E6C000842F0020DB3A0020642928BF6421F8B59C
:10E6D00001FB00F5642495FBF4F40646E4B2002740
:10E6E000FBB2A34204D29F2004F0CBFC0137F7E732
:10E6F000B4420BD2142195FBF1F5C4EB8410663DB6
:10E70000C4EB80002844C0B204F0BBFC0134E4B286
:10E71000B44201D29A20F7E7F8BD2DE9F0438DB05D
:10E7200000F0CEFDAA4C0546236AC31A002BC0F2A6
:10E73000D78300F5433303F5A0732362A54B94F808
:10E7400024201F78C7F38007BA1A18BF012284F863
:10E7500024704FB1002A00F0C3839F4B5A789A70FF
:10E7600001225A701A704DE09B4B2AB1DA7842F0C0
:10E770000202DA709A785A70D97801F0020000F03B
:10E78000FF0238B994488068281A002803DB01F09A
:10E79000010200E0012202F00100DFF83CE2187003
:10E7A00082B3C8072ED59EF804008C4A411CC9B21A
:10E7B0008EF80410114491F82C101646022908D145
:10E7C000874A116840F602020A4012B902308EF8F8
:10E7D00004001A79B11891F82C10072906D1804944
:10E7E000096809065EBF7C4901320A71197906225F
:10E7F000B1FBF2F002FB1011CAB21A71324492F866
:10E800002C205A70744EDFF820923378002B3AD0C7
:10E81000F378AE2023F00203F370724B2B44B36005
:10E8200005F5F42303F59073F36000233374FCF7CC
:10E830002CFD08B104F0B6FB89F80000002800F0B8
:10E840004F83B020FCF721FD4020FCF71EFD002087
:10E85000FCF71BFD1020FCF718FD4FF4806808F151
:10E86000FF3800201FFA88F8FCF70AFDB8F1000F06
:10E87000F5D1404604F029FC7278584B03EB820333
:10E88000586B04F019FC99F80030002B00F0288335
:10E89000F368514AE91A0029A1BF03F5F423117C5A
:10E8A00003F59073D3607378A4BF01311174072B03
:10E8B00000F2E282DFE813F00800E00219006900CC
:10E8C0001A013701890106024749484A484B49481D
:10E8D000FEF7B5FD012004F0F8FB464804F0ECFB20
:10E8E000022004F0F2FB4448C4E23D4B1A681D4686
:10E8F00012F0020F23D0414B3E4819880A23B1FB86
:10E90000F3F203FB12133E4992B209789BB20091D5
:10E910003C49FEF794FDFFF72DFE012004F0D5FBE6
:10E92000344804F0C9FBFAF725F80646022004F043
:10E93000CCFB31461520FFF7C7FE032600E0012679
:10E940002B681B0540F198822F4B30491D686423CA
:10E9500095FBF3F2096803FB1253009125482C49FB
:10E96000FEF76DFDFFF706FE304604F0AEFB2148D2
:10E9700004F0A2FBF9F7DAFF0546701C04F0A5FBD2
:10E9800015202946FFF7A0FE76E20120214E04F073
:10E990009CFB214804F090FB33689D0746D51F4A35
:10E9A0001448B2F90210B2F900300091B2F9042013
:10E9B0001B4901921B4AFEF742FDFFF7DBFD0220D7
:10E9C00004F083FB0B4804F077FB03252FE000BF26
:10E9D000FC230020DB3A00203C31002098BA0108DB
:10E9E00070360020404B4C0007D801080AC80108C7
:10E9F000E3C401080224002005C80108AC1400206B
:10EA00006100002010D80108F00F0020A814002099
:10EA100028D801088C1700203DD80108CE0F00200F
:10EA200053D8010886D40108450600200225336822
:10EA3000D80717D58A4B8B495A688B4800929A6839
:10EA400005F1010801921B68884AFEF7F8FCFFF700
:10EA500091FD284604F039FB5FFA88F8824804F0FB
:10EA60002BFB45463368190717D5814B7D495A68FA
:10EA70007D4800929A6805F1010801921B687D4A61
:10EA8000FEF7DDFCFFF776FD284604F01EFB5FFA7B
:10EA900088F8754804F010FB4546774A7248B2F989
:10EAA0000210B2F900300091B2F904200A2192FB61
:10EAB000F1F26C490192714AFEF7C1FCFFF75AFD71
:10EAC000284604F002FB684804F0F6FA3368DA06D8
:10EAD00040F1D2816A4B6B496B4A1B686248FEF772
:10EAE000AEFCFFF747FD681CC0B2C0E10025674ED1
:10EAF0003378AB4240F2C0810E2D00F0BD81680832
:10EB0000013004F0E2FA284605F0C8FA3378AB4247
:10EB100006D9202004F0B5FA681CC0B205F0BEFA90
:10EB20000235EDB2E3E75A4B5A491A784E48FEF7E0
:10EB300086FC012004F0C9FA4B4804F0BDFA002518
:10EB4000554B49481A68535D2A44917A0091127DC9
:10EB500052490192524A52F82520FEF770FCFFF705
:10EB600009FDA81CC0B204F0B0FA01353E4804F01B
:10EB7000A3FA032DE4D14B4B4B491D783A482A4662
:10EB8000FEF75DFC052004F0A0FA374804F094FA83
:10EB90000C236B43454E4649F5186A78F35C3248BE
:10EBA000FEF74DFCFFF7E6FC062004F08EFA2E4837
:10EBB00004F082FAA9792A796B792B4800913D49B2
:10EBC000FEF73DFCFFF7D6FC50E1012004F07DFA92
:10EBD000394804F071FA00250226E8B204A9FEF7CC
:10EBE000AFF89DF81430002B36D0032D34D00B989D
:10EBF00007F0A0FA0146314807F0A8FB07F0B8FC7F
:10EC000042F21073DDF820800A9A08FB00F10092AE
:10EC1000424301F59C5102F59C5008310830B1FB8C
:10EC2000F3F1B0FBF3F02A464346019102902449E8
:10EC30000D48FEF704FC06F10108FFF79BFC304687
:10EC400004F043FA5FFA88F8074804F035FAB8F19F
:10EC5000080F00F21181464601350F2DBDD10BE1A1
:10EC6000782F002053D801080224002062D8010820
:10EC7000A02700209DD401085C2F002066D8010841
:10EC8000502700206AD801087DD80108943600205A
:10EC90001831002081D80108802700208DD8010874
:10ECA000ECBA0108D8130020A2D80108F4300020E3
:10ECB000B3D80108C4D80108D6D801080024744983
:10ECC000ECD80108E16A226BA36A914203D1EB1AE6
:10ECD000002BC0F2D180636B2163A16B824A8B420F
:10ECE0001CBF936392F83C3005F574251CBF0133BB
:10ECF00003F003034FF0010105F510754FF000001C
:10ED000018BF82F83C30A56204F0ECF994F83C306E
:10ED1000764A0025D05C04F0B4F90220012104F009
:10ED2000E1F9734B3620EB5C0135C3EBC30393FB76
:10ED3000F0F0C0B2062828BF06206038C0B204F048
:10ED4000A0F9102DEDD16B4B674D1B786A4913F07C
:10ED5000020F6A4B05F106001A7814BF59234E239F
:10ED6000FEF76DFBFFF706FC022004F0AEF9A81DCC
:10ED700004F0A2F96249634BD1F804E00A68A81DC7
:10ED800092FBF3F260499EFBF3F3FEF758FBFFF7AB
:10ED9000F1FB032004F099F9A81D04F08DF95B4BF9
:10EDA0005B491A88A81DFEF74AFBFFF7CBFB04203E
:10EDB00004F08BF9A81D04F07FF9564B56491A88C8
:10EDC000A81DFEF73CFBFFF7BDFB04210A2004F061
:10EDD00089F9A81D04F070F95049E26AA81DFEF7F0
:10EDE0002EFBDFF86481FFF7ADFB052004F06DF921
:10EDF000A81D04F061F9D8F804204949A81DFEF7C0
:10EE00001EFBFFF79FFB05210A2004F06BF9A81DEC
:10EE100004F052F9D8F81030D8F80C204149D21A31
:10EE2000A81DFEF70CFBFFF78DFB062004F04DF943
:10EE3000A81D04F041F9337CA81DDB0747BF3A4900
:10EE4000D8F8082039492A6CFEF7F9FAFFF77AFB5F
:10EE500006210A2004F046F9354804F02DF9354919
:10EE6000152233480AF060F8FFF76CFB072004F026
:10EE70002CF92F4804F020F9002F31D12E4B00211E
:10EE800093F820301220052B97BF2C4A3F259B1862
:10EE900093F8605004F026F9284604F0F2F81320A5
:10EEA000002104F01FF9264B1B78002B254B18BFBF
:10EEB00072201B7808BF2120002B18BF522004F0BD
:10EEC000E0F81420002104F00DF994F84450074BA9
:10EED000585D013505F0030504F0D3F884F844507B
:10EEE0000DB0BDE8F08300BFFC230020FCD8010872
:10EEF00031040020882F002001D90108F80F0020DC
:10EF0000FC0F00208096980012D90108F40F002011
:10EF10001FD90108C010002027D901082ED90108E7
:10EF200035D901083ED9010845D901084DD9010854
:10EF3000022400204C0600201C15002098BA01086D
:10EF4000040E0020990E0020CC2700207047044BAF
:10EF50004FF4805208B11A6170475A61704700BF80
:10EF600000080140034B4FF4805208B15A617047CA
:10EF70001A6170470008014030B50022074B811824
:10EF800003F10C0453F8045BA34241F8045BF9D18C
:10EF90001B880E32702A0B80F0D130BDFEBA0108FA
:10EFA00037B5054600212A2209F04FFF052200232C
:10EFB0000421019300938DF804208DF806208DF82C
:10EFC0000510AA1C6C4603CC516007491060595CBF
:10EFD0000133052B02F8081BF4D10123AB80522327
:10EFE0002B7003B030BD00BF0CBB010810B500236F
:10EFF0000549C4180A68C2504A680C3362608A68BE
:10F00000242BA260F4D110BD12BB010830B5094910
:10F0100000220B78084C1557854202BFFF25155575
:10F0200003F1FF3302F10C0208BFDBB23C2AF1D13D
:10F030000B7030BD44240020C43600200022084953
:10F040000C2303FB02135968814204D10022C262DF
:10F050001A815A6070470132052AF0D1704700BF0B
:10F06000C43600200023084A02EBC30292F90210C2
:10F07000814204D19088003018BF012070470133CD
:10F08000052BF0D1002070479A36002038B1438814
:10F0900011EA030003D08B420CBF0120022070470D
:10F0A00010B509490022042A0BD81446531CDAB2C1
:10F0B000064B03EBC4039C882042F4D00A70981CD2
:10F0C00010BD0A70002010BDF01500209A360020F7
:10F0D0002DE9F043204B00211B689D7893F803E055
:10F0E0001E4BAAB25F88988802EB8204C5F16406C1
:10F0F0005242F6B26400CEF1640CC01B92B293B2DD
:10F100000FFA83F9B9F1000F04DC002B14BF2B4672
:10F11000012300E0334609FB09F85B4308FB0EF8C6
:10F1200098FBF3F3634403FB09F34FF00A0893FBE6
:10F13000F8F323441BB243434FF47A7893FBF8F37C
:10F14000DFF81C803B4428F8113001310A320C29C9
:10F1500092B2D4D1BDE8F083F030002044240020E6
:10F16000522400200A4B00221B68187A02FB02F38B
:10F17000193B434303F6C4135343192193FBF1F3A3
:10F18000044921F812300132072AEFD1704700BF3D
:10F19000F03000206A24002010B50C4B00221B68C0
:10F1A0005C78187840F6C41102FB02F3193B634304
:10F1B00003F6C4135343434393FBF1F3044921F88B
:10F1C00012300132072AEDD110BD00BFF03000200F
:10F1D00078240020104B043033F91000B0F5617F23
:10F1E00005DB40F633039842A8BF184601E04FF410
:10F1F00061700A7819235A4302F28332824208DA94
:10F200004A78534303F283338342B4BF0020012082
:10F2100070470020704700BF0034002010B500F197
:10F22000500302788A4203D18478C278944204D38E
:10F2300004309842F5D1002010BD012010BD1FB54B
:10F24000084B1B681B0309D58DF8040002910023AD
:10F250000D2001A98DF80530FAF73AF905B05DF8EF
:10F2600004FB00BF7036002010B5427A044632B16C
:10F27000036804F10A01406898470023637210BDD7
:10F28000014B02481B6D18474424002080000240B7
:10F29000014B0248DB6C1847442400206C000240FC
:10F2A000014B02489B6C1847442400203000024068
:10F2B000014B02485B6C1847442400201C000240AC
:10F2C00010B50A4A0A4B11689B6800BF1268914248
:10F2D000F7D1084A4FF47A70546D00FB04F2D31A48
:10F2E000B3FBF4F300FB013010BD00BF1815002084
:10F2F00010E000E04424002038B50446FFF7E0FFAA
:10F300000546FFF7DDFF401BA042FAD338BD10B51C
:10F3100004462CB14FF47A70FFF7EEFF013CF8E79A
:10F3200010BD024A1368013313607047181500209E
:10F3300010B50024054AA3185B681BB1A256282A01
:10F3400000D198470834182CF4D110BD5417002070
:10F35000014B1B68184700BFB439002010B50020CE
:10F36000FFF7F6FF064B00241C70F9F7B9FB054BBD
:10F3700083F85840DC65A3F860405C6610BD00BFB0
:10F38000401500204424002010B510B9BDE81040FD
:10F39000E4E700230C225A430A4C1119125D824201
:10F3A00003D00133102BF5D110BD074B586E18B1A7
:10F3B0004A784078824204D200225966A3F860203D
:10F3C000DA6510BD2CBD01084424002010B54000B2
:10F3D0001428A8BF14200023074A022199540B4483
:10F3E00099181424834201F8014CF5DBFF21D15414
:10F3F0000F20BDE81040C7E7CC3200202DE9F843CC
:10F4000081460B26013E3CD0204C09F10107A36840
:10F41000A2894FF032085A612368A28805251A6133
:10F42000A268A189D36801204B40D3602268A188DB
:10F43000D3684B40D360FFF78BFF4046FFF767FF71
:10F44000A268A189D36800204B40D3602268A188BC
:10F45000D3684B40D360FFF77BFF4046FFF757FF71
:10F4600045B1013DDCD14FF4FA70FFF750FF4FF08A
:10F47000FA08D5E7013FD3D14FF47A70FFF747FF81
:10F48000C0E7034A034BDA60BDE8F8834415002067
:10F490000400FA0500ED00E00A4B10B55A6832B1DD
:10F4A000DA681AB15A6942B9022200E0012203EB7C
:10F4B000C204616003F8320010BD0020BDE81040B6
:10F4C0009CE700BF5417002003685B6A03B118472C
:10F4D000704703681B6A03B11847704703689B694C
:10F4E00018472DE9F743064689469DF828801146BE
:10F4F0001A469DF82C3000250C2068431C4FC41977
:10F50000C057B04202D1208920B12BE00135052D32
:10F51000F2D127E0022E0FD005DC56B1012E21D109
:10F52000009314480AE01E2E0DD01F2E1AD1012080
:10F5300009E00093104801E0104800934346FCF7AF
:10F5400043FB044605E001F047FF41460446FFF750
:10F55000C5FF4CB10C2303FB05752671A5F8089077
:10F560006C6001E0002000E0204603B0BDE8F083BD
:10F57000C4360020004400400038014000480040EC
:10F5800003685B69184710B504462046FFF7F8FF8B
:10F5900018B90A20FFF7BBFEF7E710BD03681B6927
:10F5A00018470368DB68184703685B68184710B59D
:10F5B0000E4C2068FFF7F8FF0028F9D02068FFF70D
:10F5C000F0FF0B4A0821138883EA00239BB213F44F
:10F5D000004F4FEA43031CBF83F4815383F00103C0
:10F5E00001399BB2F3D1138010BD00BFE03300207E
:10F5F000E433002003681B68184710B504460C4B21
:10F6000021461868FFF7F6FF0A4B0822188880EA9F
:10F61000042010F4004F4FEA40001CBF80F48150DA
:10F6200080F00100013A80B2F3D1188010BD00BF14
:10F63000E0330020EC33002003682DE9F041DB6962
:10F6400004460E46174693B90D467B1B3344002BE8
:10F650000BDD236820469B6898470028F9D0204698
:10F6600015F8011BFFF7C6FFEFE7BDE8F081BDE825
:10F67000F0411847E0E770B5124D0024214605F12E
:10F680006900702285F8684009F0DFFB2146D5F853
:10F69000DC300C4A0B4493F9020088B11E6802F179
:10F6A00069040E5108199C88073184809B79702960
:10F6B000837192F8683003F1010382F86830E6D173
:10F6C00070BD00BF44240020094B1A680E2303FBC1
:10F6D0000020437AFF2B07D0064A12789A4203D9BA
:10F6E000054A32F8130000E0808800B2704700BF7E
:10F6F000C832002094360020003400202DE9F84361
:10F700000024274BE0B293F82861B04211D203EBFA
:10F71000400203EB8003D3F8F830B2F8E01033B1C5
:10F720000B2804D81F4A12780AB1DB6898470134C5
:10F73000E7E71D4B1B685B032FD500242346E2B28D
:10F74000B2422AD2DFF858904FEA840809F1F8074C
:10F7500057F8242055689D4217D02846FCF792F9A7
:10F76000EFF31283502282F312882821AA8C01FB26
:10F77000009092B20132C0F85021AA8ADBB292B254
:10F7800042F00102AA8283F3118857F80830002260
:10F790001B6801341A802B46D1E7BDE8F88300BF0F
:10F7A00044240020380000207036002008B50D4B9E
:10F7B0001B6813F4805F0C4B14BFB3F8D021DA88B8
:10F7C00093F828110023D8B2884204D2074820F8C1
:10F7D00013200133F7E7FFF791FFBDE8084032201F
:10F7E00095E500BF70360020442400202425002029
:10F7F0000A4B30B51A680A4B02F48052B3F8D04174
:10F80000DD880023002A0CBF28462046054921F840
:10F81000130001330C2BF5D130BD00BF7036002032
:10F82000442400201A3100202DE9F74F494B4A4C5F
:10F83000D3F80080D4F8D4514046294606F0D2FCD3
:10F84000D4F8D87100903946404606F0CBFCD4F885
:10F85000DC6101903146404606F0C4FC39468246E0
:10F86000284606F0BFFC31468346284606F0BAFC1F
:10F8700031468146384606F0B5FC39468046384662
:10F8800006F0B0FC014606F0A5FB314607463046BF
:10F8900006F0A8FC014606F09DFB064639464FF0EF
:10F8A0007E5006F095FB314606F092FB5146C4F8B7
:10F8B000E001584606F08CFB014606F08BFB0199EF
:10F8C000C4F8E401484606F085FB014606F082FBD9
:10F8D0005146C4F8E801584606F07CFB014606F0A4
:10F8E00079FB2946C4F8EC01284606F07BFC01466A
:10F8F00006F070FB01464FF07E5006F069FB314682
:10F90000054606F065FB0099C4F8F001404606F094
:10F910005FFB014606F05EFB0199C4F8F40148461E
:10F9200006F056FB014606F055FBC4F8F8010099B5
:10F93000404606F04FFB014606F04CFB3946C4F842
:10F94000FC01284606F044FBC4F8000203B0BDE801
:10F95000F08F00BF2C00002044240020F8B52F4B6E
:10F960001B685B0758D52E4C2E4D2678012E07D0EC
:10F97000AB689847EB689847012323706B8845E094
:10F980002B6998476B6898476B69201D26499847F3
:10F990002169E2680978501C8842A16908BF267570
:10F9A00001F1010608BF0020032E04BF1C4E4FF0DA
:10F9B000010E636808BF86F81CE004EB81010B624E
:10F9C000217F08BF0026A768DFF854E0A66181B157
:10F9D000DEF82060DEF82410DEF828308E42DEBF2C
:10F9E0008E4631467646B342A8BF33468B42B8BFF7
:10F9F0000B4604EB8202D36204EB8002D26AE06021
:10FA0000BA1A1344A360002323702B88D4F8EC2087
:10FA1000642B38BF6423D360F8BD00BF8C1700206F
:10FA2000482600203C170020DC0F0020034B1B68F9
:10FA30009B0301D5FEF771BE704700BF70360020F2
:10FA40002DE9F04FB54B85B01B685A0702D5B44A73
:10FA5000127D12B9DB0640F14582B24B1A68B04BF9
:10FA6000D3F8F070D11B009146F2A71100981F4601
:10FA7000884240F23782AC4CC3F8F02025885DB351
:10FA80001A69D3F8F4101278013D501E9A68B2FB3F
:10FA9000F0F2082091FBF0F6891B0A44C3F8F42029
:10FAA00092FBF0F006F04AFBA04906F04FFCA0499B
:10FAB00009F020FC01464FF07E5006F089FA9D497E
:10FAC00006F090FB06F054FD0022C7F8F8002580F0
:10FAD000C7F8FC20C7F800213A69B8681278964D3B
:10FAE000013AB0FBF2F006F025FB904906F02EFC3F
:10FAF0008F4909F0FFFB01464FF07E5006F068FA8F
:10FB00008C4906F06FFB09F0B9FB3A698246D2F8DE
:10FB10000480286806F012FB414606F063FB81462C
:10FB2000D7F8F8007E4EC0EB0A0006F007FB41460E
:10FB300082464FF07E5006F04BFA0146504606F0E2
:10FB400051FB0146484606F045FA09F097FB28604C
:10FB500004F010FE794A8146D2F82080D7F80411CB
:10FB6000404606F0E7FC20B14FF0FF32C6F808210E
:10FB700009E0484606F0E2FA414606F033FB06F09B
:10FB8000F7FCC6F80801D7F808B16548BBF1000FCB
:10FB90000BDDB0F90C118B4507DA2968C5F800B008
:10FBA000CBEB0101C0F8101139E02E68D7F8101125
:10FBB000BBF1000FA6EB0106DFF864812E602EDD9D
:10FBC000B8F91451AB452ADCCBEB050006F0B6FAC8
:10FBD0008146B8F90C01281A06F0B0FA01464846E9
:10FBE00006F0B4FB0546584606F0A8FA294606F08A
:10FBF000F9FA8046304606F0A1FA294606464FF04B
:10FC00007E5006F0E5F90146304606F0EBFA014673
:10FC1000404606F0DFF906F0ABFC4749086048496A
:10FC2000086806F087FA4749064606F0DBFAD7F877
:10FC30001851019075B13A49D1F8240106F07EFAC5
:10FC40008046284606F07AFA0146404606F07EFBDA
:10FC5000054600E00025D7F82811284606F0C2FA2C
:10FC6000314606F0BFFA344902900E684FF07C51DD
:10FC700006F0B8FA019906F0B5FAD7F8FC900199A8
:10FC80000390484606F0AEFAD7F81080DDF80CC0B5
:10FC9000D8F80CA00146604606F09CF9D7F8001190
:10FCA00006F098F9514606F09DFA0390304606F0AA
:10FCB00045FA514601904FF07E5006F089F9DDF883
:10FCC00004C00146604606F08DFA039B01461846C3
:10FCD00006F080F90299C7F800018246484606F00E
:10FCE00079F98146C7F8FC0015480021C7F81C11B6
:10FCF000C7F82011C7F82411C7F81811016021882E
:10FD0000002940F0EF80BBF1000F0F4C1EDD0449CD
:10FD1000B1F90C118B4519DA26601BE08C17002015
:10FD200048260020B8390020D239002080E6C54797
:10FD3000B1DC423ED048874AD80F0020242600205C
:10FD4000BC390020BD378635A8100020504606F08B
:10FD50000FFC2060D7F82C01DFF8ACA1301A06F0B8
:10FD6000EDF9624906F03EFA8346009806F0E2F9A2
:10FD70000146584606F0EAFA06F0FAFB40F2DC5279
:10FD80009042A8BF1046A2F6B8329042B8BF1046C3
:10FD90000A21C7F82C61FDF767FBD8F80860834695
:10FDA0003146484606F01EFA8146584606F0C6F926
:10FDB000314680464FF07E5006F00AF90146404633
:10FDC00006F010FA0146484606F004F9C7F8FC00B0
:10FDD00009F054FA05210646FDF746FB40F23E6164
:10FDE000434AD7F8308110604248028802F21F323D
:10FDF00092B28A4205D8428802F21F3292B28A42F7
:10FE000005D90020C7F84001C7F830516AE09AF8D8
:10FE100044210ABB2068DAF834210A21121AB2F50B
:10FE2000FA7F3548A8BF4FF4FA729042B8BF104627
:10FE3000FDF71AFBDAF838214FF0800ED2782F49FF
:10FE4000504390FBFEF2B2F5967FA8BF4FF4967236
:10FE50008A42B8BF0A4601E0294A1268D7F8380139
:10FE6000C6EB020E447A20260EFB04F494FBF6F651
:10FE7000C17CD7F83C21B6F5967F0EFB0122A8BFC6
:10FE80004FF496761F49B2F5C81FA8BF4FF4C812A9
:10FE90008A42B8BF0A464FF40054C7F83C2192FB8F
:10FEA000F4F2164C407FA642ACBF9419141906F028
:10FEB00045F941460646284606F08CF8014630468C
:10FEC00006F090F94FF06C5106F08CF906F050FBFB
:10FED0009628A8BF96206FF095029042ACBF201ADA
:10FEE000A01A8FE705B0BDE8F08F00BF0024744969
:10FEF000D40F00205C2F00200CFEFFFFD4FEFFFF7C
:10FF0000C03900200000E7FF482600200D4B10B547
:10FF10001B68DB0614D50C4B19680C4BD3F8482131
:10FF20003C3291420CD3D3F84C41C3F8481122889B
:10FF300063680B201A61FFF7DFF9636822885A6152
:10FF400010BD00BF8C170020181500204826002087
:10FF50004B4B70B51B681B0740F19080494C4A4BD6
:10FF600004F5A8705B689847B4F9503104F5AC709B
:10FF7000C4F85831B4F952310146C4F85C31B4F9CF
:10FF80005431C4F86031414B1A78FAF7C1FA404B4A
:10FF90001878194610F0040F17D03E4B1B68C4F8B0
:10FFA000643100233C4A0026D518EE80A2F11005EA
:10FFB00035F8135002F10C0612329D539D52023354
:10FFC000062BEFD120F00400087094F880212D4B0F
:10FFD000A2B1B3F96E11D3F85821521AC3F85821BF
:10FFE000B3F97011D3F85C21521AC3F85C21B3F94C
:10FFF0007211D3F86021521AC3F86021D4F8641149
:020000040801F1
:10000000204A00293AD0234B02F5BA741B6802F546
:10001000BD705B1A21498B421AD821490A68898828
:10002000D3684B40D36000231E4934F9136051F864
:1000300023205D001C31B242B8BF21F81320415F7C
:1000400001338A42C4BF18496A52032BECD170BDF8
:100050000023C2F8643102F5B67234F9135030F956
:10006000131001332944022591FBF5F1032B22F8EB
:10007000021FF2D1BDE87040FAF742BE70BD00BF6A
:100080008C170020482600209C1700209417002081
:10009000882F0020B8390020B02700207FC3C90175
:1000A00044150020A0270020C22700209D4B2DE9E9
:1000B000F0411B681A0640F117819B4E3368B3B9B3
:1000C0009A4C94F88431013B042B00F20D81DFE857
:1000D00013F0140014001400FA00D700924B1868B3
:1000E000FFF75FFAF7F7F6FA08B100F0FFFA3068A9
:1000F000FFF75AFA0028F1D1E2E794F8A4718B4D8A
:1001000017B1012F11D0EFE0012B00F2ED8095F82F
:100110008521874B0C2101FB02335A78854B3068CF
:1001200053F82210FFF73AFA64E03068DFF8F881FC
:10013000FFF726FA002800F0D78095F88431022BCB
:1001400045D0032B53D0012B40F0CE807A4B196859
:10015000D5F89C31CB1AC72B40F2C680D5F8983120
:10016000042B32D8724A0C20964600FB0323C5F8B4
:100170009C11D8F800505E78AF6800236D49D8B262
:1001800051F82320BA4204D00133082BF6D10023C2
:1001900000E00346B34205D0284651F82610FFF789
:1001A000FDF9A1E094F885310C2101FB03E25668CA
:1001B00016F8011B19B12846FFF71CFAF8E7D4F826
:1001C00098310133C4F898318EE002208AE095F826
:1001D0008521574B0C2101FB02335A78554BD8F837
:1001E000000053F82210FFF7D9F903207AE095F8C0
:1001F000A6310BB9042075E095F8A0310BB985F84C
:10020000A07194F8A031494D012B16D1D5F8983141
:10021000B22B0CD8464A3068134493F83C10FFF7D1
:10022000E9F9D5F898310133C5F8983105E0002394
:10023000C5F89831022385F8A03194F8A0313B4DE0
:10024000022B18D1D5F898210F2A11D895F8A5318D
:10025000374903EB03130B44134493F8F010306851
:10026000FFF7C8F9D5F898310133C5F8983102E0A5
:10027000032385F8A03194F8A031022B34D9B9E7D3
:10028000D4F88C3129490133C4F88C3194F8A73162
:100290005BB191F8853105220133DBB2B3FBF2F299
:1002A00002EB82029B1A81F88531234B00221B68E6
:1002B0000120C4F89031214B1A70214A137823F0A1
:1002C000020313700EE01C4BD4F890211B689B1A9C
:1002D00040F6C412934207D91A4A0520136823F046
:1002E00020031360F7F7D0FC164B1B689B0617D54D
:1002F000154B0E491B68D1F8A8219A1A002A0FDB6A
:100300000E4A1278042A0BD903F5123303F5F87359
:10031000C1F8A8310D498A688989D3684B40D360F8
:10032000BDE8F081703600203831002048260020DA
:1003300020BB010834A5010818150020F80F002083
:10034000882F00208C170020B83900204415002089
:1003500010B5324B50B31A7830480132D2B2132A5A
:1003600088BF00221A701A78DAB942702C4A1268D3
:10037000940704D52B4C24780CB102244470D40586
:1003800006D5294AD2781AB15A7842F004025A7036
:10039000264A127812F0050F02BF5A7842F0010285
:1003A0005A700A6802F5C332A0320A605A78002AED
:1003B00032D01A4B1B7899080A41D0071AD503F09E
:1003C0000103012983F0010210D008D3022911D1C1
:1003D000174B03F11801002A08BF0B460BE0154B21
:1003E00003F11801002A18BF0B4604E0114B03EB80
:1003F000C20300E00F4B00220F4909788A420BDA52
:100400000E4901EB82014988090642BF18680C4970
:1004100041F822000132EFE710BD00BF982800200C
:1004200070360020FA1500201C150020DB3A002051
:10043000FCC30108ECC30108FD230020781F002045
:1004400012390020F0B5891A782461439B1A91FB78
:10045000F3F10F4B063001221F78824001F22B117D
:100460000020B84213DA0B4B03EB80035B88134286
:100470000BD0094D4FF4B47635F820300B4493FB84
:10048000F6F406FB143325F820300130E9E7F0BD1F
:10049000FD230020781F00201239002010B50A4BE0
:1004A0000420B3F906104FF47A724FF4FA63FFF7A1
:1004B000C9FFBDE81040054B0820B3F90010002229
:1004C00040F2FF33BEE700BF00340020AC10002034
:1004D0000149702208F056BD64BC01081B4B1C4941
:1004E00013F82020887802F00F03834205DDC878D6
:1004F0008342ACBF0223002300E0012309791209E3
:100500008A4202DB43F0040305E0114949798A423B
:10051000D8BF43F008039A0710D013F00C0F0DD08A
:1005200013F0020F14BF0521042113F0080218BFB5
:1005300002220A4401209040184301E043F4007075
:10054000030708BF40F4807080B27047781F002016
:1005500098280020F8B52E4E00242E4B1B789C4284
:1005600054DA758828050AD415F4805F08BF2A4A32
:100570002A4B14BF7278D27803EB820300E0002389
:10058000E9052CD5264A178800222648910030F824
:10059000220040B9244B2046194491F87270FFF7AD
:1005A0009DFF002305E0384215D0F3E70433182BF4
:1005B00029D01E4AD1189A5C498845FA02FE1EF0DD
:1005C000010FF3D00142F1D0062303FB0727184B9C
:1005D000DA5D124B0FE00132062AD6D10EE0AA05F1
:1005E0000CD5144B0C4A1B7813F0040F18BF52782B
:1005F0000A4B08BF127803EB820300E01BB11A68B4
:100600000D4B43F8242001340436A6E7F8BD00BFA3
:10061000781F0020FD230020301F0020381F0020FD
:10062000622F0020D4BC010864BC0108ECBC0108A6
:100630000C1F0020DB3A0020123900200023F0B507
:100640001C46264A02EB84014988174611B912F864
:10065000242032B1090504F1010448BF0133202CE4
:10066000EFD11F4A0025D9B214702B462A461D48E7
:100670008171A5420DD017F8256001354FEA161E8D
:10068000734506F00F06B8BF7346B242B8BF324694
:10069000EFE70132D2B25408013302720132DBB209
:1006A0005210C371C2705A0801335B10013A0371D2
:1006B00006234271B1FBF3F203FB1212013C12F06C
:1006C000FF0F847006D00B46062B03DDDA0701D43A
:1006D0005B10F9E7044A1370F0BD00BF781F0020DB
:1006E000FD23002098280020FF230020924B2DE9B5
:1006F000F04FDA68914D1A612A6891B0DA60904A39
:100700000295136843F0200313608E4B1A78012A78
:100710000CBF002201221A708B4B1A78910740F10E
:100720004E838A490978042940F249838849097827
:1007300001F0040101F0FF0011B922F001021A706A
:100740001B78DB0702D408B1F7F796FB81494A7A98
:10075000531C052293FBF2F202EB82029A1A7E4BA3
:100760004A721F7892000023DFF81082DFF810929F
:1007700058F82310794C91FBF9FE04F1080040F879
:1007800023E0774844F8231000FB0E1142F210706A
:1007900091FBF0F004F1100680B226F813004FF040
:1007A000140C04F114060CFB036C04F13C0A5AF817
:1007B00023605CF802504CF80210761B3144052689
:1007C0004AF8231091FBF6F109FB0E114434012F76
:1007D00044F823104FEA830B444605D10238B0F5A4
:1007E000797F98BF4BF808100BB90123BCE7594E2D
:1007F000029BB2461868B36DC01A05F09BFC5949BC
:1008000005F0A4FD029B4FF07E511B680746B365BF
:1008100005F086FE08B94FF07E574B4BCAF85C7066
:100820001B78514E13F00103504D12D00DAA0092C7
:100830004F4B0EAA01920CCB94E80300F7F732FA63
:100840000D9A6421B2FBF1F20E9B328093FBF1F31F
:1008500000E033802B809AF860303E4D002B35D07D
:10086000E96D4FF07E5005F071FD07466B6E206814
:10087000C01A05F063FC394605F0B4FC05F078FEBB
:10088000AB6E86B2606836B2C01A05F057FC394BC1
:10089000196805F0A7FC394605F0A4FC05F068FED0
:1008A000B5F96E2000B28118B5F96C200220B3189A
:1008B00091FBF0F193FBF0F389B29BB2A5F87210B3
:1008C000A5F87030A5F86E10A5F86C3001238AF8F1
:1008D0006030294B61681B88206803F030031D4E8F
:1008E000264DCAF86810CAF86400002B00F0678231
:1008F00006F17C03009306F180030193726FB36FDE
:10090000F7F7D0F96B68B06FC01A05F017FC194BF8
:10091000196805F067FC05F02BFE736F2A68C6F8AE
:1009200088009B1AC6F884300B4B1B78012B29D00A
:10093000022B00F0E58042E2CC27002018150020B1
:100940008C170020E4030020882F0020F80F0020DF
:10095000DB3A002098280020020F0020A428002065
:10096000806967FF00007A446A1000206C10002044
:10097000B010002030000020622F0020FC0F00206B
:1009800080969800D6F88C30D6F8A8400293D6F816
:100990009C3004F100400393D6F8A030F76D059326
:1009A00005F0E6FD8146204605F0E2FDD6F8A430CC
:1009B000BB4C0493BB4B06901B684FF0000B079396
:1009C000B94E4FEA4B0356F82B80A6F1140240466D
:1009D00032F81B50089305F0B1FB029905F002FCB8
:1009E00005F0C6FD401B1FFA80FA283626F81BA02A
:1009F0000FFA8AFA504605F0A1FB039905F0F2FBC5
:100A000005F0B6FD86B20AEB080005F097FB0599E4
:100A100005F0E8FB394605F0E5FB216805F0DAFA58
:100A200005F0A6FD484504DB069B9842A8BF184682
:100A300000E0484605F082FB206005F099FD079B29
:100A4000304486B2987805F075FB984905F0CAFBEA
:100A500001464FF07E5005F079FC394605F0BAFAB0
:100A60000146384605F072FC09906068D4F808A089
:100A7000C0EB080005F062FB394605F067FC514603
:100A800005F0A6FA099A0146104605F0ABFB0146AF
:100A9000504605F09FFA3135ADB2622D0146206116
:100AA000C4F80480A0600ED9049805F09BFB05F003
:100AB0005FFD7F4AB0F5FA6FA8BF4FF4FA6090422D
:100AC000B8BF104600E0002040F6B832064436B207
:100AD0009642A8BF1646774A089B9642B8BF16466C
:100AE000754A54F8140B9E52142202FB0BF2734900
:100AF0005050BBF1000F40F062814FF0010B5FE7F7
:100B0000684BB6F8B0401F68F36F3D8902935B08ED
:100B10009D4228BF1D4623B29D4202DC1FFA85F983
:100B20000AE06749F06D05F05DFB05F021FD20440A
:100B30001FFA80F9A6F8B090DAF88060DAF8B440CD
:100B4000341B2046F7F7F0F841F293130028D8BF82
:100B500040429842CCBF0020012078B3204605F0E7
:100B6000EDFA584905F03EFBFCF74CFD04460298AF
:100B700005F0E0FA0146204605F034FB05F0F8FCEC
:100B800040F6B83380B2AAF8B80000B29842A8BFC5
:100B90001846484B9842ACBF3018F01848F6A043AE
:100BA000984203DDA0F50C40A03804E00028BCBF4B
:100BB00000F50C40A030CAF8BC0001E0CAF8BC60E7
:100BC000DAF8BC300026C3F50C502830039305F04A
:100BD000B5FA3C4905F006FB0446FCF787FD0F908B
:100BE0002046FCF70FFDDAF8C030DAF8CC40059368
:100BF000DAF8C4300E9004F10040089305F0B8FC18
:100C00000490204605F0B4FCDAF8C830DAF85C80CD
:100C10002A4C09900793730048460A9305F08EFA10
:100C20000EAB53F8261005F0DDFADFF8A0A005465C
:100C30003AF9160005F082FA0146284605F0C8F98F
:100C400005F096FC05B2204BB5F57A7FA8BF4FF4AE
:100C50007A759D42B8BF1D460AF13C0AA8B22AF82F
:100C6000160000B205F06AFA0599824605F0BAFA54
:100C700005F07EFC089983B25046069305F0B2FA5F
:100C8000414605F0AFFA216805F0A4F905F070FCC3
:100C9000049B98421CDB099B9842A8BF184618E0A9
:100CA000440F0020040F00201C290020DB0FC94046
:100CB00030F8FFFF48F4FFFF160F00206C0F0020F4
:100CC0000000C842D302373918FCFFFF0829002072
:100CD000049805F033FA20608346B87805F02AFAC4
:100CE000384905F07FFA01464FF07E5005F02EFBA3
:100CF000414605F06FF90146404605F027FB0B9091
:100D00006068D4F808A0281A05F018FA414605F0E2
:100D10001DFB514605F05CF9DDF82CC0014660462C
:100D200005F060FA0146504605F054F96560014649
:100D30002061A060079805F055FA05F019FC069BA4
:100D40001434034458469A4605F012FC40F6B83273
:100D5000504400B29042A8BF10461B4A0A9B9042E2
:100D6000B8BF1046194A1A4998521422724342F8E1
:100D700001B00EB901264EE73B792BB1039A6423EB
:100D800092FBF3F3134A13803B88029A124C9A4267
:100D90000ED9D4F8B430D4F88000C01AF6F7C4FFE6
:100DA00042F2107380EAE072A2EBE0729A4206DD32
:100DB0000A4B01221A70B4F8D020064B1A8011B0E9
:100DC000BDE8F08FDB0FC94048F4FFFF160F00208D
:100DD000440F0020FE0E002098280020020F002063
:100DE000426A806A131A58425841704741717047ED
:100DF00043799B070AD5436A8269D154436A0169E2
:100E00000133B3FBF1F201FB1233436270474279C5
:100E100002F0020202F0FF0342B10369426A806AF3
:100E2000013BDBB2101A23EA0000704718467047F6
:100E3000437913F001031FBFC36803F1FF32C36995
:100E4000006A1DBF181A1040C0B218467047437997
:100E500010B513F0010304460DD0FFF7E9FF58B1B8
:100E6000236A6269E168D05C0133B3FBF1F201FBF4
:100E70001233236210BD184610BD90F83B3210B5F6
:100E80007BB990F83A3290F83942A34209D2B0F8CF
:100E9000401201229A400A430133A0F84022DBB2FB
:100EA000F3E710BD8379DB0748BFB1FA81F1D0F8D1
:100EB000343148BF49095A681B8909B11361704729
:100EC0005361704710F80A3C0133DBB20A2B84BF30
:100ED00010F8131C044A00F80A3C82BF002322F8D1
:100EE000113000F80A3C7047C0130020F0B55A4892
:100EF000142403780133B3FBF4F204FB1233012210
:100F0000037000EBC3031A719960544B5D681C6C4D
:100F1000A9429A680C4409D293F8485085B104F567
:100F20008034944211D94FF480350BE094420CD9AF
:100F300093F84850002D0CBF00254FF4803501E098
:100F4000944202D9A21A521B02E0C2F58032224416
:100F5000002583F8485090F8A45014279C606C1C1E
:100F600094FBF7F507FB1545DA6090F8F840DE686A
:100F700080F8A450013400EB8505C5F8A86094FB07
:100F8000F7F507FB154480F8F84000EB8400596042
:100F9000C0F8FC1040F68C218E42304A3CD91178C2
:100FA00092F945400846A1420CD10C1F082C09D8E3
:100FB00092F84640182C9ABF013482F8464082F8D5
:100FC000441002E0002283F8462093F94440234A6B
:100FD000A14219D192F84740B4B10C3200248C429E
:100FE00006DA52F8046F1E4D25F814600134F6E756
:100FF0000C2805D01A4A002422F810400130F7E7E7
:101000001848027801320270012283F8472000223A
:1010100083F845101A70F0BD92F84710D1B140F234
:10102000DA51A6F2EF20884208D811780B2905D8AA
:101030000B1D0131117042F82360F0BD002283F8CE
:101040004720094B03F13002002143F8041F93426B
:10105000FAD1F0BDF0BD00BF6C290020F8040020DB
:10106000C0130020B63300200405002010B50D4B3E
:1010700014241A780132B2FBF4F004FB10221A7027
:1010800003EBC20300221A71074A9960136C013303
:101090000B4413644FF6FF73994204BF012382F897
:1010A000483010BD6C290020F8040020024B53F892
:1010B00020301B68198070473C250020074BA1F5A4
:1010C0007A7153F820301A681B8959434FF47A73A8
:1010D00091FBF3F189B21180704700BF3C250020DD
:1010E0001FB50123ADF80830ADF80410002301A9A5
:1010F000ADF80A30ADF80C30ADF8062003F0DEFF95
:1011000005B05DF804FB38B5A0F513746379A579D3
:10111000DB0745D594F8383205F00105F3B1226BB1
:101120001068838DC3F34E03838494F83C3223B15B
:10113000B4F842320133A4F84232917A6A00FFF7E0
:10114000CFFF012384F83B32002384F8393284F83E
:101150003A3284F83832A4F8403238BD94F83B3241
:101160002046012B04BF94F8393284F83A32FFF755
:1011700084FE94F83B22236B3AB9012284F83B2287
:101180001868997A05FA02F207E0002284F83B22F7
:1011900095421868997A08BF0222BDE838409FE757
:1011A00038BD10B5A0F5127494F83C22BAB9A36A00
:1011B000616A994228D0591CA069A162C35C206968
:1011C000DBB25B0043F400738142A4F83E324FF07F
:1011D0000A0384F83D3228BFA262012312E094F989
:1011E0003D327BB1B4F83E1220464B08A4F83E32A3
:1011F00001F00101FFF756FE94F83D32013B84F8FF
:101200003D3201E084F83C3294F83832002B4ED164
:1012100094F839320133DBB2092B84F8393203D127
:101220002046BDE8104028E60A2B40D194F83B3216
:101230002BB9B4F8403243F00103A4F8403263798B
:10124000D9071CD5B4F84002820501D4C30705D4E0
:10125000B4F844320133A4F8443210E0E36AC0F336
:1012600047000BB198470AE0E3696269D054E3692B
:10127000E1680133B3FBF1F201FB1233E3610122B8
:1012800084F8382294F83B220023012A84F839326A
:101290000DD1A27984F83B32236B12F0010F18684C
:1012A000997A0CBF02220022BDE8104018E710BD59
:1012B000F0B5046D8279A389467923F4005312F0C6
:1012C000020F4FEA03434FEA13430CBF00214FF4D0
:1012D000005112F0040FA38114BF4FF4806E4FF041
:1012E000000E16F0010F8768054614BF0420002089
:1012F000B307238A48BF40F008029BB223F440534F
:1013000043EA01032382A18948BF90B289B221F444
:10131000B05121F00C014EEA010140EA0102A28124
:10132000A38A87B023F440731B041B0CA38201A87B
:1013300003F0E6F8039B049E254A944218BF1E461C
:10134000A389192272431BB2002BB4BF7E00BE00DA
:10135000B2FBF6F66427B6FBF7F00001010907FBC4
:101360001163A28912B2002AB7BFD9001A01323123
:10137000B1FBF7F2A7BF3232B2FBF7F302F007027C
:101380001043A8BF03F00F03AA79A8BF184380B287
:1013900012F0010F20812B6D06D00E498B4202BF47
:1013A000042001F54841086112F0080F9A8A0BBF2A
:1013B00022F0080292B2120442F0080208BF120C96
:1013C0009A829A8992B242F400529A8107B0F0BD93
:1013D00000380140004400402DE9F04F1E464FF414
:1013E000147343435A4D85B005F5A6748046914663
:1013F000E718A24610B92B44564A03E0012806D14B
:10140000554A2B44C3F87C211032C3F880224FF494
:10141000147303FB08F35148EC180AEB030203F5BD
:101420009C73343253444FF0010CC4F84C01C4F89F
:101430007811C4F86021C4F8643100224FF480713F
:10144000D4F88032032084F884C3C4F85811C4F857
:101450006C21C4F86821C4F85C11C4F87421C4F884
:10146000702184F8882384F88523A4F88E23A4F8B7
:101470009023C4F8549184F8510184F8526184F89F
:10148000928358681B8903A9ADF80C3010238DF89E
:101490000E300223CDF804C08DF80F30009301F018
:1014A0009EFBD4F87C21009B5068128903A9ADF8FB
:1014B0000C2048228DF80E208DF80F3001F08FFBA4
:1014C000DDF804C038466146FFF7ECFC3220FDF73A
:1014D0001EFF234BD4F880B21B681A46B2FBF9F109
:1014E000B1F5803F03D3012AF8D95208F6E71D4A27
:1014F0004FF41474B3FBF2F204FB08F8584689B2B7
:10150000D2B2FAF795FA05EB0809174B08F51278ED
:101510000AEB08040022C9F8943358462146FAF72A
:10152000CFFAD9F87C5116F0010F0CBF022200222D
:101530002868A97AFFF7D4FD0C4B2846C9F89833E0
:10154000211D0022FAF7BCFA384605B0BDE8F08F3D
:101550006C2900202CC501084CC5010804BD0108F8
:101560006400002040420F00A31101080711010888
:1015700003460A4690F84602D96A9B792CE71FB5C4
:101580000123ADF808300023ADF80C30ADF80A3077
:10159000094BADF8041093F8EC3501A9012B08BFF5
:1015A0000323ADF8062008BFADF80C3003F086FD2C
:1015B00005B05DF804FB00BF6C29002038B510F8B9
:1015C0000E2C044650F8043C52B9012200F80E2CAF
:1015D00020F80C1C997A18680222BDE83840CEE742
:1015E00030F80C2C20F80A1C891A89B220F8081C43
:1015F000074A10F80F0C002522F8101004F80E5CB2
:101600001868997A2A46FFF7BAFF04F8065C38BDD5
:10161000C0130020044B53F820301BB107289CBF97
:101620001B681980704700BF24060020F0B540F207
:10163000E6363B4DB5F90040241A04F2F317B742E1
:1016400003D8002CB8BF644201E04FF4FA74B5F936
:1016500002502F1A40F2E63007F2F315854203D804
:10166000002FB8BF7F4201E04FF4FA77BC42B8BF09
:101670003C462C48C4F5FA74052794FBF7F7B0F9FB
:101680000040B0F90260002CB8BF6442002EB8BF21
:101690007642B442B8BF3446012A21D1AE2939DCA2
:1016A0001220C1F1AF0141430A220C1B91FBF2F160
:1016B000544394FBF1F2642AA8BF6422002BC1BFFB
:1016C000A7F164006421484390FBF3F0D4BF0020ED
:1016D000401822EAE2724243642092FBF0F01BE0E1
:1016E00000290DDDC4F5E164122594FBF5F54D43A9
:1016F000642295FBF2F5501A2844584390FBF2F30C
:10170000002B07DDA7F164006424444394FBF3F04D
:10171000643001E00020F0BD20EAE070F0BD00BFC1
:10172000003400205C2F00202DE9F04F87B0039398
:1017300082460291019203F0EFFFBE4BDC8804F079
:101740000204A4B28CB1B3F90A40B3F90830002CFA
:10175000B8BF6442002BB8BF5B429C42B8BF1C4676
:10176000B4F5007FA8BF4FF400740AF10903DFF855
:10177000E8B200930025B0494FF0040E31F915305E
:10178000143151F825106A00002991FBFEFEB8BF04
:101790004942B1F5206F4FEA43034FEA8507DBF872
:1017A00000000FDCCEEB03010144B1F57A5FA348E2
:1017B000A8BF4FF47A518142ACBFCBF80010CBF8F0
:1017C000000002E00021CBF800109A48816A0E0167
:1017D0001AD590F82C1000F1300611F0200FDBF82C
:1017E000001002D190F82D0050B1F659704281429C
:1017F00003DB8E423046A8BF0846CBF8000003E06A
:101800000029B8BF4942F1510098DBF8006010F898
:10181000011FF6114E431AF8051000904B438549FD
:10182000B611B1F806C09B111CF0030F47D0083168
:10183000505E8349515E01EB40010198C0F1000800
:10184000414503DB8842A8BF08468046DFF8E491A3
:10185000039932F90900C0EB080031F915804044C2
:1018600009F13C0842F2107957F808100144494543
:10187000A8BF4946DFF8E4914945B8BF494647F853
:1018800008109AF8078008FB00F09AF81B80C01136
:1018900008EB8808C8F10009484503DB4045A8BFAC
:1018A000404681469AF81100C9EB030341430913EE
:1018B000761A6643634301EB662609EB6323DFF880
:1018C000A09119F8058008FB0EF8A3EBA81809F100
:1018D0000403D05E22F803E0BAF82230CEEB000019
:1018E0009BB10592CDF810C009F1080904F026FC5F
:1018F000242101FB0591FBF70AFB07F0BFFCDDF893
:1019000010C000EB4003059A0DE009F1740E09F1D7
:101910007C0957F80E1057F8093047F80E000B44B1
:10192000034447F8091047491CF4006F11F805906B
:1019300009FB03F34FEA631901F1040308EB060105
:101940004944D15206D0404B1B78590702D528464E
:10195000F6F7BCFA374B0BF1040B03F1D40247F84E
:10196000028003F1E002BE5003F1EC0247F802905E
:101970001E460DB90125FEE6B3F90C20029B042496
:101980009B79B0690F335B005343726A5B1192FB22
:10199000F4F2002BA3EB0202B8BF5B42322B9AF8A1
:1019A0000C100BDC01FB0201284B8B42A8BF0B463D
:1019B00027498B42ACBFB361B16101E00023B36141
:1019C0009AF80240234B54431B78A411032B0CD9E3
:1019D000BAF82030B3F5FA7F07D25A42944203DBBB
:1019E0009C42A8BF1C4600E01446B5696FF0FF0397
:1019F00045F34F35B5F5807FA8BF4FF480759D4204
:101A0000B8BF1D466319A6F8D030F3881A0506D56D
:101A10000D4B1B785B0702D50220F6F757FA00231F
:101A2000C6F8DC40C6F8E850C6F8F43007B0BDE8A8
:101A3000F08F00BF5C2F0020642F002080C1FFFFCB
:101A4000D439002024300020DB3A0020FEFFFF0FB5
:101A5000020000F06C2500206C2F0020F0D8FFFF62
:101A6000A02F00202DE9F04F87B0039383460C464A
:101A7000924603F051FE964BB3F8069009F0020926
:101A80001FFA89F35BB1109B9BF82410188A9BF80E
:101A900025209BF81B30FFF7C9FD019000E0019362
:101AA000D946E31CDFF8448202930025029A022DF6
:101AB00012F8013F8649029203F11B0304D1B1F9E8
:101AC0000C2053435B1132E001F1080232F915207A
:101AD000CC885343A6074FEA45004FEA231326D08C
:101AE0007C4E36F9156006EB4206CAF100029642BA
:101AF00003DB56453246A8BF5246095EE007A2EB1B
:101B00000102039948BF9BF8073031F915100A44C8
:101B100057BF9BF811105A434A4301994FBF131105
:101B20004A43642192FBF1F258BF03EB22136A4847
:101B30004FF0040E50F8251099F8004091FBFEFE7E
:101B4000CEEB03035C4300F586702F5C64217C437D
:101B500094FBF1F4022D4FEA85024FEAE4140ED112
:101B6000BBF8201059B15D480078032807D94842D6
:101B7000844203DB8C42A8BF0C4600E00446544874
:101B8000B0F82C6100F110017343515899F80A60C4
:101B9000DB1206FB0316524BB6F5001FA8BF4FF42D
:101BA0000016816A9E42B8BF1E46090118D590F8FA
:101BB0002C3013F0200F00F1300302D190F82D10DB
:101BC00039B199584B429E4209DB8E42A8BF0E465E
:101BD00006E086EAE671A1EBE671995000E01E4648
:101BE0003B4901F11003D65099F814307613002BBD
:101BF00048D001F59873D05842F803E04FF6FF73D0
